:020000040800F2
:10000000204001204905000845BE0708058F070864
:1000100041BE07081DF806088D17080800000000FB
:10002000000000000000000000000000550400086F
:100030002BFC060800000000B10400083DC60708BC
:1000400063050008630500086305000863050008F0
:1000500063050008630500086305000863050008E0
:1000600063050008630500086305000863050008D0
:1000700063050008630500086305000863050008C0
:1000800063050008630500086305000863050008B0
:1000900063050008630500086305000863050008A0
:1000A0006305000863050008630500086305000890
:1000B0006305000863050008630500086305000880
:1000C0006305000863050008630500086305000870
:1000D0006305000863050008630500086305000860
:1000E00063050008630500080000000063050008C0
:1000F0006305000863050008630500086305000840
:10010000630500086305000863050008630500082F
:10011000630500086305000863050008630500081F
:100120006305000801F90608630500086305000877
:1001300005F9060863050008630500086305000863
:1001400000000000000000000000000000000000AF
:1001500015F9060825F90608630500086305000877
:1001600063050008630500086305000863050008CF
:100170006305000859BE0708630500080000000079
:1001800063050008630500086305000863050008AF
:10019000630500086305000863050008630500089F
:1001A000630500086305000863050008630500088F
:1001B000630500086305000863050008630500087F
:1001C000630500086305000863050008630500086F
:1001D0006305000849BE07086305000863050008B9
:1001E000630500086305000863050008630500084F
:1001F000630500086305000863050008630500083F
:10020000630500086305000863050008630500082E
:10021000630500086305000863050008630500081E
:10022000630500086305000863050008000000007E
:10023000630500086305000800000000630500086E
:1002400063050008630500086305000863050008EE
:1002500063050008630500086305000863050008DE
:10026000630500086305000863050008F99907089D
:10027000451C00006305000863050008000000003D
:10028000630500086305000863050008000000001E
:10029000000000006305000800F002F800F0CAF852
:1002A0000AA090E8000C82448344AAF10107DA45D1
:1002B00001D100F0BFF8AFF2090EBAE80F0013F059
:1002C000010F18BFFB1A43F0010318478C93080075
:1002D0004C9408000A444FF0000C10F8013B13F056
:1002E000070408BF10F8014B1D1108BF10F8015B8F
:1002F000641E05D010F8016B641E01F8016BF9D182
:1003000013F0080F1EBF10F8014BAD1C0C1B09D1D8
:100310006D1E58BF01F801CBFAD505E014F8016B4A
:1003200001F8016B6D1EF9D59142D6D370470000DC
:10033000103A24BF78C878C1FAD8520724BF30C811
:1003400030C144BF04680C607047000000230024E3
:1003500000250026103A28BF78C1FBD8520728BFD5
:1003600030C148BF0B6070476E2900F0CB87702901
:1003700000F03583662904F0748D652904F0718DD1
:10038000672904F06E8D612904F06D8D03681B0AE6
:1003900028BF41F08001692900F0A682642900F09D
:1003A000A382752900F0A0826F2901F0508478297A
:1003B00000F00183E92901F0EB83E42901F0E883EF
:1003C000F52901F0E583EF2901F04D84F82900F0CB
:1003D00000830368DB0928BF41F08001632901F035
:1003E0005A83732901F05F83E32902F0F981F3292D
:1003F00002F0FE81002070471FB584F0C9FC9DE823
:10040000030000F0E5FE00F04CFD00F0C1FE04002A
:100410000020002184F0FAFA401C606000200021D6
:1004200084F00AFBE06002F067F81FBD10B502F02F
:10043000CCF810BD02F088FD1146FFF7DDFF03F098
:1004400083FC02F0D1FF03B4FFF7F0FF03BC82F09E
:10045000A5FA00002C4B19680868B0E8F04F80F34B
:100460000988BFF36F8F4FF0000080F31188704749
:100470000000000008480068006880F308884FF01A
:10048000000080F3148862B661B6BFF34F8FBFF3EC
:100490006F8F00DF00BF00BF08ED00E0DFF80C0049
:1004A000016841F470010160704700BF88ED00E011
:1004B000EFF30980BFF36F8F134B1A681EF0100F14
:1004C00008BF20ED108A20E9F04F106009B44FF00A
:1004D000500080F31188BFF34F8FBFF36F8F83F00D
:1004E0006DFD4FF0000080F3118809BC19680868A1
:1004F000B0E8F04F1EF0100F08BFB0EC108A80F388
:100500000988BFF36F8F7047FC010020EFF305806F
:10051000704700000B49D1F800C04A685CF8043B02
:100520001068184442F8040B8C4528BFA1F1DC0C7C
:100530008A4228BFA1F1DC02C1F800C04A6020F065
:100540000040704784B000200948804709480047B0
:10055000FEE7FEE7FEE7FEE7FEE7FEE7FEE7FEE773
:10056000FEE7FEE704480549054A064B70470000D0
:1005700051C60708990200082000012020400120F0
:10058000202001202020012010B500F001FE001DD8
:1005900010BD00BF7944080070B5064600F0F4FDB8
:1005A000056806F10B0020F00704B4429CBF002050
:1005B00070BD2B466A68BAB11068A04210D304F12E
:1005C000080188423CBF5068586007D35168101931
:1005D00041601168091B016058601460101D70BDF6
:1005E00013465268002AE7D12146284600F0DCFD78
:1005F0000028DED170BD70B50446051F00F0C4FDB3
:100600000068002C14BF446870BD002C18BFAC42B9
:100610003CBF20466468F8D301680A18AA4218BF94
:10062000456003D12A6805461144016028684119D4
:10063000A1421CBF6C6070BD61686960216808449C
:10064000286070BD53EA020C00F069802DE9F04B80
:100650004FF00006002B1FBFB3FA83F503FA05F431
:1006600024FA05F65E4012BF1643B2FA82F502FA8A
:1006700005F4C5F120051EBF22FA05FC44EA0C046E
:10068000203556EA044C4FEA144418BF641C4FF05E
:1006900000084FF00009904271EB030C39D3002998
:1006A00019BFB1FA81F701FA07F6B0FA80F700FA3C
:1006B00007F6C7F120071EBF20FA07FC46EA0C0622
:1006C0002037B6FBF4FCA7EB0507103F07F01F0B24
:1006D000CBF120060CFA0BFB2CFA06F644BFB3460E
:1006E0000026202FA4BF5E464FF0000B5BEA060CED
:1006F00008BF4FF0010B19EB0B09ABFB027C48EB79
:100700000608C01B06FB02CC0BFB03CC71EB0C01F3
:10071000C1E70B46024641464846BDE8F08B13B59B
:100720004FF000004FF00001AFF30080BDE81C4027
:100730007047B2F120030AD5C2F1200320FA02F07B
:1007400001FA03F321FA02F140EA0300704721FAAB
:1007500003F04FF000017047B2F120030AD5C2F157
:10076000200320FA02F001FA03F341FA02F140EA11
:100770000300704741FA03F04FEAE171704710B58A
:100780004C1084EA530404D54042C1F1000138BF43
:10079000491E1B4204D55242C3F1000338BF5B1E01
:1007A000FFF750FF14F0804F04D04042C1F1000128
:1007B00038BF491E14F0004F04D05242C3F1000369
:1007C00038BF5B1E10BD00000FB4044910B503AA6A
:1007D000029801F06DF910BC5DF814FB00AF002029
:1007E0000FB4044910B503AA029801F061F910BCD6
:1007F0005DF814FB00AF00200FB41CB5084B06AA2F
:100800007B4469460090059801F023F904460020D6
:10081000694601F031F920461CBC5DF814FB00006C
:100820007512000070B5044685690068C10601D5DF
:10083000302600E02026C00707D070BDD4E9012192
:1008400030469047206A401C20626D1EF6D570BD70
:1008500070B5044685690078C00707D170BDD4E93A
:10086000012120209047206A401C20626D1EF6D591
:1008700070BD09684A0501D540B27047C905FCD56D
:1008800000B2704709684A0501D5C0B27047C90572
:10089000FCD580B2704770B50C460546012A05D0DC
:1008A0002878800600D5EA69002302E0012305E0EC
:1008B0005B1C934202D2E05C0028F9D1A869E618DB
:1008C000C01AA861286A184428622846FFF7AAFFC0
:1008D00004E0D5E9012114F8010B9047B442F8D3A4
:1008E0002846FFF7B5FF70BD2DE9F041064600240C
:1008F00010687529314616A510D0FFF7BAFF0028F9
:1009000002DA404213A507E031688A0701D512A533
:1009100002E0490704D511A5012401E0FFF7B2FF69
:1009200000210A2206F1240709E0B0FBF2FCB0FB2B
:10093000F2F302FB1C00303078541846491C0028A2
:10094000F3D123462A463046BDE8F04100F081BC91
:10095000000000002D0000002B000000200000001F
:10096000F0B40D460188090502D5214C7C4402E013
:100970001F4C7C440E34002100F1240608E002F0F4
:100980000F071209E75D42EA03721B097754491CFD
:1009900052EA0307F3D102780023120704D5702D21
:1009A00006D009B1022311342246F0BC00F051BC3C
:1009B00001231034F8E770B504460D46214610684F
:1009C000FFF760FF024629462046BDE8704000233D
:1009D000C6E7D21D22F00703D3E90023C0E703686E
:1009E000126843F0200303600823C3610023B7E7C4
:1009F000334808002DE9F05F894604464FF0000AAD
:100A0000DFF874B1FB44C0F820A02046E1688847B5
:100A1000002874D0252806D0D4E901219047206A07
:100A2000401C2062F1E700265F462046E1688847C7
:100A30002028054607DB312D05D2781910F8200C47
:100A400008B10643F1E7B00701D526F00406C4F863
:100A50001CA00027C4F818A02A2D09D0284681F030
:100A600083FF38B304EB8708303DC8F8185019E00D
:100A700059F8041B204604EB87029161E16888471E
:100A8000012F054618D1E069002820DA26F020065B
:100A90001DE0D8F8180000EB800005EB400030386E
:100AA000C8F818002046E1688847054681F05CFFD9
:100AB0000028EED1012F0AD02E2D08D12046E16862
:100AC00088477F1C0546022F46F02006C4DBA0693C
:100AD000002803DA404246F00106A061F00701D089
:100AE00026F010066C2D0BD0682D09D04C2D39D076
:100AF0006A2D35D0742D35D07A2D33D016E038E0FC
:100B0000E1682F4620468847B842054609D16C2F38
:100B100026D04FF48060E1680643204688470546AA
:100B200004E06C2F1AD04FF4807006430DB3A5F18A
:100B30004100192802D8203546F400664A46294665
:100B4000204626604E46FFF70FFC80B101280BD0EF
:100B5000F61D26F0070000F1080956E74020E4E7FB
:100B60008020D8E70020D6E706F104094DE72846A3
:100B700052E7206ABDE8F09FC34708000FB400B5F4
:100B80008DB010A9099000910B904FF0FF300A90A2
:100B900000200C90064878440690064878446A463F
:100BA00007900F9909A801F0F9FA0DB05DF814FB50
:100BB000231600003B1600002DE9FF5F1D464FF095
:100BC000FF3B91464FF000085F46D5E90146A96911
:100BD00001987F1C8847296A824688470028F6D1F9
:100BE000BAF1FF3F0CD0002E24F4C06419DD60067A
:100BF00014D5BAF12B0F09D0BAF12D0F0ED103E0A5
:100C0000584604B0BDE8F09F44F48064A969019897
:100C10007F1C8847761E8246002E02DDBAF1300F17
:100C200003D0B9F1000F26D032E0A969761E0198F1
:100C30007F1C44F400748847002E824605DDBAF11B
:100C4000780F06D0BAF1580F03D0B9F1000F10D0C9
:100C50001EE0B9F1000F02D0B9F1100F18D1A96947
:100C6000761E01987F1C24F4007488478246102069
:100C700002E0082000E00A20814609E0A96908FB9B
:100C80000908761E01987F1C44F400748847824648
:100C9000002E05DD4946504600F0F0FF0028EDDA51
:100CA000E96901988847A00502D46FF00100A8E720
:100CB000E00725D1600613D5600502D5C8F1000014
:100CC00000E0404629680A1D2A600968220501D50E
:100CD000087015E0220701D5088011E008600FE0D8
:100CE0002868011D29600068210502D580F8008070
:100CF00006E0210702D5A0F8008001E0C0F80080DE
:100D000038467EE72DE9FF5F4FF00008994614460C
:100D100046469169D2E901A7DDF838B001988847C5
:100D2000054659EA0B0005D009E0A1690198761C37
:100D300088470546216A284688470028F5D1681C5F
:100D400003D05FEACA7005D015E04FF0FF3004B061
:100D5000BDE8F09F2068011D2160D0F800800AE006
:100D60005FEACA7001D108F8015BA169761C01989D
:100D70007F1E88470546002F1ADD681C18D0B9F180
:100D8000000F0DD0E81705EBD060421120F01F00D6
:100D900059F822102A1A012090400142E0D107E0C0
:100DA000BBF1000FDCD12846216A88470028D7D044
:100DB000E16901988847BBF1000F07D1002E05DDDE
:100DC0005FEACA7002D1002188F80010A068B8421A
:100DD00003DDBBF1000F03D017B16FF00100B6E7E0
:100DE0003046B4E770B5064600F0D6F9046805460B
:100DF00030460A22002101F053FA2C6070BD000039
:100E000070B50446C068810713D0800601D5A56A75
:100E100004E0A169606808442169451A204601F090
:100E200027FB002206462946204601F071FA30468B
:100E300070BD002070BD70B510B1BDE87040DFE737
:100E40000025074C6E1E07E02046FFF7D9FF00B1D2
:100E50003546206D20F00104002CF5D1284670BDE8
:100E6000ACAE0020021E71F1000204DA0023D0EBC8
:100E7000030063EB010170470B4910B5A1F17C023F
:100E80000A4CC2E93712372106E000EB104342F862
:100E90002130074B00FB03400B1EA1F10101F4DCE4
:100EA00010BD0120E8E7000024B00020E119D6665B
:100EB000CD0D0100014A01F0BBBB000084030020FE
:100EC000401ECAB210F8011F8A4202D00029F9D18F
:100ED0000020704730B505460B462A4613F8014BF3
:100EE00012F8010B08B1A042F8D01CB1002802D0C2
:100EF0006D1CF1E7284630BD40EA0103024630B5DB
:100F00009B0710D14FF0013400E008C208C91D1B37
:100F10009D4315EAC41FF8D013F0FF0102F8011B2E
:100F20000DD01B0AF8E711F8013B002B02F8013B3A
:100F300005D011F8013B002B02F8013BF3D130BD85
:100F400010B5431C02E010F8011B71B18107FAD102
:100F50004FF0013202C88C1A8C4314EAC211F9D046
:100F6000C01A0A0603D0C01E10BDC01A10BD0A0464
:100F700001D0801E10BD0902FCD0401E10BD421ED3
:100F800012F8013F002BFBD111F8013B002B02F8B6
:100F9000013BF9D17047032A40F2308010F0030C76
:100FA00000F0158011F8013BBCF1020F624498BFBC
:100FB00011F801CB00F8013B38BF11F8013BA2F159
:100FC000040298BF00F801CB38BF00F8013B11F0D4
:100FD000030300F02580083AC0F0088051F8043B74
:100FE000083A51F804CBA0E80810F5E7121D5CBFE1
:100FF00051F8043B40F8043BAFF30080D20724BF14
:1010000011F8013B11F801CB48BF11F8012B24BFA7
:1010100000F8013B00F801CB48BF00F8012B7047F6
:1010200010B5203AC0F00B80B1E81850203AA0E883
:101030001850B1E81850A0E81850BFF4F5AF5FEAB7
:10104000027C24BFB1E81850A0E8185044BF18C96A
:1010500018C0BDE810405FEA827C24BF51F8043B11
:1010600040F8043B08BF7047D20728BF31F8023B65
:1010700048BF11F8012B28BF20F8023B48BF00F8F9
:10108000012B70474FF000020429C0F0128010F0CD
:10109000030C00F01B80CCF1040CBCF1020F18BF54
:1010A00000F8012BA8BF20F8022BA1EB0C0100F0E7
:1010B0000DB85FEAC17C24BF00F8012B00F8012BBA
:1010C00048BF00F8012B70474FF0000200B51346EF
:1010D00094469646203922BFA0E80C50A0E80C5058
:1010E000B1F12001BFF4F7AF090728BFA0E80C5009
:1010F00048BF0CC05DF804EB890028BF40F8042B02
:1011000008BF704748BF20F8022B11F0804F18BF6E
:1011100000F8012B704700004FF0013C50F8042B01
:1011200051F8043B9A4215D1A2EB0C03934313EA06
:10113000CC130BD150F8042B51F8043B9A4209D13F
:10114000A2EB0C03934313EACC13E7D04FF000005B
:10115000704700BFD01A01BAB1FA81F101F018014D
:1011600022FA01F0CB40C1F12001DBB2C0B2C01ABB
:101170002CFA01F3D11A914311EAC311E6D1704759
:1011800070477047704700000048704794B00020D7
:1011900000487047ACB00020004870478CB0002079
:1011A000704770477047704738B504460A460020BC
:1011B0006946AFF30080002808BF38BD0246009999
:1011C000204601F05BFA012038BD012001F097BEF6
:1011D000F8B5AFF30080054600200C46102000BF94
:1011E0000646A819A0420DD9324669460020AFF341
:1011F0000080070008BF01F082FE0098A04218BFDF
:101200000546C419FFF7C0FF05600746F01D20F032
:1012100007004619284600F00AF8B44208BFF8BD96
:10122000A21B31463868BDE8F84001F027BA00211A
:101230000160C0E9011070471020704710B5FFF73A
:10124000ABFF006810BD10B50446FFF7A5FF0460B2
:1012500010BD2DE9F0470D4699469246044600F12F
:1012600024080168880604D5E06921F01001216096
:1012700000E00120A84201DD471B00E00027A16932
:101280007A1902EB0900081AA0612078C00602D47E
:101290002046FFF7C7FA002608E0D4E901211AF832
:1012A00006009047206A401C761C20624E45F4DB05
:1012B0002078C0060AD52046FFF7B4FA06E0D4E944
:1012C000012130209047206A401C2062381EA7F17F
:1012D0000107F4DC07E0D4E9012118F80500904784
:1012E000206A401C2062281EA5F10105F3DC20467F
:1012F000FFF7AEFA2078000602D50220BDE8F0879D
:101300000120FBE711680268006A530501D50870E7
:101310000AE0D30501D5088006E0130603D5C217FD
:10132000C1E9000200E008600120704770472DE924
:10133000FF4F0C461E464FF0FF378BB0D2E900013D
:10134000DDF860800A908A46C1F30A5505B93D462A
:10135000002108464FF00000BAF1000F00F44000F1
:1013600005DA00EB80004FF4400101EA50004FEA3B
:101370009059B9F1010F00DDB9460A9850EA4A00C8
:101380000ED044F61050A5F2FF3545432F14B8F1A6
:10139000000F1ED07542291E1EDDC9F100021CE09F
:1013A000B8F1010F4FF0000001D0302103E0F2430B
:1013B00005E02154401CB042FBDB304600220021F6
:1013C00021540B99C1F80880C1E900200FB0BDE895
:1013D000F08FBD1B6D1CDEE74A4600DA694206A8A5
:1013E00001F014FC06AB93E8070003AB83E80700A9
:1013F00050460A9902F074F88DE80700A0F50050F5
:101400001F3800900398002D0ADD42F21F014A4662
:101410000844002303A90390684602F01FFB09E07B
:10142000A0F500504A461F38002303A903906846E0
:1014300002F03EFB8DE807000004000C03D04FF0E3
:10144000FF30410800E01046B8F1000F03D0002241
:10145000009215461EE0751E05D401F029F93032C0
:1014600062556D1EF9D5B3460122084302D0002211
:101470007F1C04E02078302801D100227F1E002A42
:10148000099784D01DE0112D07DA01F011F93032EF
:1014900062556D1C50EA0102F5D1084302D0009854
:1014A000C8B10EE00021681E05E0235C625C635455
:1014B0002254401E491C8142F7DBAB46A81B401E4C
:1014C0000990002004F80B000B98099AC0F80880D6
:1014D000C0E9002B7AE711264FF0000857E72DE905
:1014E000F04F88460446D21D22F0070191B0D1E9A1
:1014F0000001CDE90A0180F04BF902460B98C00FBC
:1015000001D02D2007E02068810701D52B2002E0C3
:10151000202101EAC000032A099001D0072A05DB37
:1015200003464146204601F011F90BE12078800680
:1015300001D5E06900E00620B8F1650F814606D0CC
:10154000B8F1660F18D0B8F1670F70D131E0002004
:10155000B9F1110F009001DB112301E009F1010342
:101560000AAA01A90CA8FFF7E2FEDDE90C7000262B
:1015700009F10105834647E001204B4600904FF0FA
:1015800000470AAA01A90CA8FFF7D1FEDDE90DB0BA
:101590000C995D46002610B909F101000D18B9EB50
:1015A000050003D4C0F1FF3609F10105A5EB0900E0
:1015B0002BE0B9F1010F01DA4FF001090020B9F178
:1015C000110F0090484601DD112300E003460AAAEE
:1015D00001A90CA8FFF7ABFEDDE90C704D46002613
:1015E0008346207800070AD4AB4500DA5D4601A89F
:1015F000012D04DD411911F8011C302907D04F4598
:1016000002DA17F1040F04DA012082460FE06D1EA2
:10161000EEE7002F02DCED1B3E4403E0781CA842FD
:1016200000DD7D1CB81B00F1010A4FF00047207857
:10163000000703D4AA4501DB4FF0FF3A0021B7F1C0
:10164000004F0DF143088DF8431024D002202B23C6
:10165000002F01DA7F422D230A21021EA0F1010092
:1016600000DC5FB197FBF1FC97FBF1F201FB1C7C06
:1016700017460CF1300C08F801CDEEE7A8F1010097
:1016800003702188090501D5452100E06521A0F1FD
:10169000010800F8011C09980FA9A1EB0807FF1D1C
:1016A00000B10120411901EBEA70A1693844081A20
:1016B000401EA0612078C00602D42046FFF7B2F891
:1016C000099828B1D4E901219047206A401C206282
:1016D0002078C00622D52046FFF7A4F81EE0002E91
:1016E00004DBB34502DD01A8805D00E03020D4E9D1
:1016F00001219047206A401C2062761CAAF101005B
:101700005FEA000A0AD1FFF743FDC0680168405C48
:10171000D4E901219047206A401C2062281EA5F1CF
:101720000105DCDC07E0D4E9012118F8010B904742
:10173000206A401C2062381EA7F10107F3DC204616
:10174000FFF786F8032011B041E600002DE9F04FC5
:1017500004460D46D21D22F0070089B0D0E900975B
:101760004846394680F014F80246F80F01D02D2380
:1017700007E02068810701D52B2302E0202101EA40
:10178000C0038DF820300BB1012000E00020032AB7
:10179000824601D0072A04DB2946204600F0D6FF06
:1017A0003FE12078800601D40D2500E0E569C7F30C
:1017B0000A560D2D49DA00214FEA175B08464FF013
:1017C0000000002F00F4400007DA00EB80004FF427
:1017D000400100EBD07001EA60008115012901DDB4
:1017E0004FF0FF3100224FEA850CBCF1180F06D3F1
:1017F0001346ACF118004FF08052C24003E04FF4A2
:10180000801323FA0CF30CF10C0CBCF1200F04D361
:10181000ACF1200C09FA0CF001E007FA0CF00029F9
:101820004FF0004801DD18B90FE00ED140450CD350
:1018300019EB02095F4121B9404502D19F4329EAD2
:101840000209BBEB175F00D0761C2088000502D58B
:101850007B48784402E07A487844193808AA302353
:1018600002F80A30037C0AF10101002E0AF1020A93
:1018700053546A4602DC4FF0300101E04FF0310171
:101880004FF001088DF8001002D0A6F2FF3603E0F9
:1018900059EA470100D06B4E002D02DC2178090780
:1018A00004D54FF002082E218DF80110C446002106
:1018B0000BE0C7F303433F01C35C491C6D1E02F8F4
:1018C0000830052908F1010801DA002DF1DC0021BA
:1018D0000CE000EB1973491C1B786D1E082902F8F7
:1018E00008304FEA091908F1010801DA002DF0DC8F
:1018F00021688B0602D516E0A8F10108E04505DD58
:1019000002EB080313F8013C302BF5D0B8F1000FBF
:1019100009DD02EB080313F8013C2E2B03D1090764
:1019200001D4A8F10108002D05DD3E2102F80810C0
:101930006D1E08F10108407C002E02F8080008F135
:10194000010804DA2D20764202F8080002E02B207C
:1019500002F808000A214FF47A70864208F1010863
:101960000BDB96FBF0F3303302F8083096FBF0F314
:1019700008F1010800FB136601E0642E0CDB642013
:1019800096FBF0F3303302F8083096FBF0F308F1E1
:10199000010800FB136601E00A2E06DB96FBF1F05E
:1019A000303002F8080008F1010896FBF1F001FB65
:1019B0001060303002F80800A16908F1010808EB56
:1019C000050202EB0A00081AA0612078C00602D4C2
:1019D0002046FEF727FF216A08AE01EB0A002062CD
:1019E00004E0D4E9012116F8010B9047BAF1010A8D
:1019F000F7D22078C00602D52046FEF713FF6E46C8
:101A000009E016F8010B3E280FD0D4E901219047D8
:101A1000206A401C2062B8F10108F2D22046FEF78D
:101A200017FF09B00320BDE8F08F206A2844206228
:101A300003E0D4E90121302090476D1EEBD3F8E795
:101A40009939080002FCFFFF01694A1C026108780D
:101A5000704700B58FB0CDE90131002105910549EE
:101A60007944CDE9031011466846FEF7C3FF0FB075
:101A700000BD0000E5FFFFFF0A6802F8010B0A60E5
:101A8000704710B5436913B1AFF3008001E0FEF772
:101A900002FF012010BD127800F124010A7000221B
:101AA0004A700122EDE711684FF0FF32E9E70000CC
:101AB000074B70B50D467B44FFF7CBFF0446284625
:101AC00081F094F810B14FF0FF3070BD204670BD2A
:101AD0003B1108002DE9FF5F15468A460446DFF8F2
:101AE000AC80F8440027D8E900103E46CDE900104C
:101AF00010E03AF816106A4602A801F0D9F9411C24
:101B000007D02178890603D5E269391891420DD8AA
:101B10000744761C2078800602D5E069B84205DDCE
:101B2000AE42E6DB3AF816000028E2D1A069C01BFD
:101B3000A0612046FEF776FED8E90010CDE900103E
:101B4000002017E03AF818106A4602A801F0B0F930
:101B5000B0F1FF3F81460BD000250DF1080B05E0E9
:101B6000D4E901211BF8050090476D1C4D45F7D3C2
:101B700008F10100B0428046E4DB206A384420626C
:101B80002046FEF765FEBDE8FF9F00001E370800F7
:101B90002DE9F0418046D21D22F007020025D2E94E
:101BA0000002F52915A614D0011E72F1000106DA13
:101BB0000023D0EB030063EB020211A608E0D8F883
:101BC00000108B0701D50FA602E0490701D50EA62C
:101BD00001251146002408F1240704E000F068FD07
:101BE00030323A55641C50EA0102F7D12B46324696
:101BF00021464046BDE8F041FFF72BBB0000000046
:101C00002D0000002B0000002000000030B4002157
:101C100000F1240408E002F00705D208303542EA5A
:101C20004372DB086554491C52EA0305F3D104688A
:101C3000002310A2250707D5A40600D421B1C4694A
:101C400001230DA2641EC46130BCFFF702BB10B5B6
:101C5000044621461068FEF715FE02462046BDE800
:101C600010400023D2E7D21D22F00701D1E9002362
:101C7000CCE7000000000000300000003A2800D24D
:101C8000303820F02002412A01D3A2F137008842E7
:101C900001D34FF0FF3070472DE9FF4F06468BB060
:101CA0000878FF2806D0491C2D2805D000244FF0C5
:101CB000000908E000200CE00124F8E709EB8903A3
:101CC000491C00EB43090878FF28F7D114B1C9F18A
:101CD00000008146107800252C46AA4629462D286A
:101CE00001D02B2804D1521C2D2813D0002082466D
:101CF0008B461078FF280FD04FF0000C0A21521CA1
:101D0000A5FB017804FB018105FB0C11C5194BEB08
:101D10000104EEE70120EAE7002108464FF0000049
:101D2000BAF1000F02D000EB80004008C0F38157E9
:101D3000012F01DD4FF0FF370E9955EA040009EB42
:101D400001080BD04FF0020918F5FA7F16DA4FEAB6
:101D5000CA70002F706008DD012007E04FEACA70EA
:101D6000C6E900B00FB0BDE8F08F00203060FFF78B
:101D700013FAC0F800901821084616E0B8F5FA7F6B
:101D800018DD002F02DAF748784401E0F64878447D
:101D9000D0E90010C6E9001040EACA707060FFF791
:101DA000FBF9C0F80090142108460FB0BDE8F04FD1
:101DB00082F0F3BF002108464FF00000B8F10001A7
:101DC000099002DAC7F1000200E03A4601DAC8F1F0
:101DD000000106A800F01AFF06AB93E8070003AB6A
:101DE00083E8070044F23E005BEA04010090584695
:101DF00004D144F21E012C465D460091210C0904D9
:101E0000014306D10099240444EA15442D041039F5
:101E1000009104F07F41014306D10099240244EA75
:101E200015642D020839009104F07041014306D178
:101E30000099240144EA15742D01091F009104F052
:101E40004041014306D10099A40044EA9574AD00D5
:101E5000891E009104F00041084304D100986D19D7
:101E60006441401E00904FF001033A466846B8F1C5
:101E7000000FCDE9014503A902DD01F02EFE01E0CE
:101E800001F001FEBAF1000F04460D4601D084F0C6
:101E90000044002108464FF00000099940F2FF7706
:101EA000484010F00C0F07D124F00040284303D025
:101EB000C4F30A50B84212D1FFF76EF9C0F800908F
:101EC000C4F30A50B8420AD1A8487844D0E90010B7
:101ED000C6E9001004F000410843706042E7C6E91B
:101EE00000543FE72DE9FF4F1F464FF0000A4FF027
:101EF000FF38454691B0D7E90146CDF83CA0FFF741
:101F000047F9C0680168405C1090B96912986D1C6F
:101F10008847396A814688470028F6D1B9F1FF3FE2
:101F20000AD0002E24F4D06411DDB9F12B0F08D0B3
:101F3000B9F12D0F0BD102E0404615B013E744F480
:101F40008064B96912986D1C8847761E81466005C9
:101F500004A901D52D2000E02B20002E01F1010B5A
:101F60000DF130088DF810003FDDB9F1690F08D090
:101F7000B9F1490F05D0B9F16E0F02D0B9F14E0F8A
:101F80001CD13B4601A8009580E85002DDE9121201
:101F90006FF0020082F0CDFFC11CCED10EE0B96916
:101FA00012986D1C884781461398761E44F400747D
:101FB00005600F98401C002E0F9016DDB9F1300F10
:101FC000EDD0B9F1780F02D0B9F1580F0DD10F98BB
:101FD00001280AD13B46CDE90054DDE91212001F69
:101FE000029682F0A4FFC11CA7D1109989453ED169
:101FF00044F0800406E01399681CAAF1010A44F435
:1020000000740860B9696D1C1298761E88473028E4
:102010008146F0D02BE01099894505D1200603D4E4
:10202000761E44F0800418E0484680F09DFC08B31A
:10203000761E0DF123018B4544F4007408D2A9F1FA
:1020400030000BF8010B200607D5AAF1010003E0D0
:10205000200602D40AF101008246A00502D5139998
:10206000681C0860B96912986D1C88478146002E6B
:10207000D1DC53E0002E51DDB9F1650F02D0B9F18A
:10208000450F4BD1A00549D5B9696D1C1298761E34
:1020900024F440748847002E81460CDD2B2804D0A0
:1020A000B9F12D0F07D144F48074B96912986D1CF1
:1020B0008847761E8146E00501D52D2100E02B21C1
:1020C00008F8011BCDF8008021E0761E0DF13901E2
:1020D000884544F400740CD2A9F1300010F0FF00E0
:1020E00088F8000002D10099884509D908F1010853
:1020F00006E0E00501D51E4801E042F20F7082467D
:10210000B96912986D1C8847814613980560002EA6
:1021100004DD484680F028FC0028D6D1F9691298E1
:102120008847FF2053468BF8000088F80000002005
:102130000A900B9004AA0CA90AA8FFF7ADFDA00510
:1021400002D46FF00100F8E614F0240F12D0E0077B
:102150001CD13868DDE90A12031D3B600068C0E944
:10216000001213E094790800867908004A78080084
:10217000F1D8FFFF0AA9684680F08EFBE00705D181
:102180003868009A011D3960006802602846D4E66C
:10219000026811441378016018467047D160054900
:1021A0007944516104497944116200211161114659
:1021B00000F022BBEDFFFFFF91050000426842B135
:1021C000016811F8013B23B1521EC0E90012184604
:1021D00070470121C160881E704742685AB1C368C8
:1021E000016843B983688B4205D0491E521CC0E97F
:1021F0000012002070474FF0FF3070470FB40023EB
:1022000000B589B00CA900910B99CB60214B7B44A0
:102210000693214B7B44079304236FF00042CDE9E2
:1022200001321E4A7A446B4608920246002082F030
:102230007CFE09B05DF814FB70B506464FF0FF3028
:1022400015460C46324686B00091CDE9010169463B
:102250000020049004A8FFF7D1FF0246049821183B
:1022600025B108B1084600E02046286004980028FF
:102270000DD0002A02DD0098884208D03246081BA3
:1022800069460094CDE9010404A8FFF7B7FF06B042
:1022900070BD0000ABFFFFFFC3FFFFFF1305000091
:1022A0002DE9F04791460F4680460446002614F873
:1022B000015B2DB1FEF768F90068405DC007F6D1FB
:1022C0002B2D02D02D2D18D0641E4A4639462046AB
:1022D00000F04CFC27B13968A14201D1C7F8008059
:1022E0004FF0020471050BD54042002803DDFEF7D4
:1022F00053FF0460A007BDE8F08746F48066E4E77A
:102300000028F8DAFEF748FF04606FF00040F2E7BB
:102310002DE9F041044616460D464769007B8007CB
:102320002ED0384680F04EFB50BB3EB3012E02D07B
:10233000022E25D104E0204600F0DAFC05441DE021
:10234000384680F02DFBE168002841F01001E16083
:1023500005DA204600F058F80120BDE8F081C903F5
:102360000BD56268E16A914200D81146A269114416
:102370002269891A814200DD08460544002D01DAF0
:102380000220EAE7E16A6068E268814206D29103CE
:10239000E06203D522F4003141F01002A669002763
:1023A000AE4213DCE16A814201D90B4600E00346EC
:1023B00003EB060C2369ACEB030CAC4506DD814254
:1023C00001D98C4600E084469C4505D1A760276072
:1023D00042F02000A5620DE0AD1BE669AE1B814214
:1023E000A66000D90846C01A281A206058196060F3
:1023F00022F0200003490840E060002084F8487083
:10240000ABE70000BFCFD7FFC16821F4001141F056
:102410008001C16000218160016070472DE9F047B3
:10242000814614460E464FF0FF383248D56857694A
:10243000054209D03846A16980F00AFB002811DB6B
:102440002C48C0430540E5602B4632464946384695
:1024500080F014FBA16920F00042B21A1144002858
:10246000A16103D02046FFF7CFFF4046BDE8F087CB
:1024700070B504460569C06A6168884200D808469C
:10248000E16821F42011E160C90312D5A84208D007
:102490002246411B2846FFF7C1FF10B14FF0FF3025
:1024A00070BD0020E562C4E90150E06820F480308E
:1024B000E060002070BD10B50446C06820F0200028
:1024C000E060A16AA06988420DD02046FFF7D0FFE6
:1024D000E06820F4405040F01000E060A06AA06185
:1024E0002069E062606044F24001E0688843E06097
:1024F00010BD00001000020010B542485421FEF744
:10250000E3FD41485421FEF7DFFD40485421FEF72A
:10251000DBFD3F493B483C4A3F4B08603D490A6070
:102520003A491960531C0365481C10650120086571
:102530003B48344A39A1784400F01EFC20B93848A1
:1025400078440A3800F0D4FC37482F4A35A1784443
:1025500000F012FC20B9344878440A3800F0C8FC76
:1025600032482A4A2FA1784400F006FC20B92F48AF
:1025700078440A3800F0BCFC40232248DC000021EB
:10258000224600F0D6FB20B125487844543800F0AC
:10259000AFFC1D4822464023002100F0CAFB20B1B9
:1025A00021487844543800F0A3FC184822461023F0
:1025B000002100F0BEFB002806D01C487844BDE88E
:1025C0001040563800F094BC10BD104870B5006D36
:1025D00020F001040B4800F045FC0B4800F042FCE1
:1025E0000A4800F03FFC09E0206D20F0010520467C
:1025F00000F038FC2046FDF7FEFF2C46002CF3D1FE
:1026000070BD0000ACAE002000AF002054AF002031
:10261000780300207C03002080030020720000006B
:10262000522C080077000000412C0800312C0800D3
:102630002DE9F04115460E46040002D12C6804B97C
:102640000BA4204600F072FC0444207870B12746A9
:102650003146384600F05AFC0444207810B100207E
:1026600004F8010B38462C60BDE8F0810027F9E73B
:1026700000000000004870478CB00020034640680E
:102680008C46002818BF88423CBF03464068F8D3F8
:1026900018681844884207D00CF1030020F00700A6
:1026A000001D411A521A0146081D0A60FDF7A3BF1A
:1026B00030B5B0F10A024FEA900E71F100034EEA14
:1026C000817EB0EB0E0061EB91014FEA101E4EEAE5
:1026D000017E10EB0E0041EB11114FEA102E4EEA75
:1026E000016E10EB0E0041EB11214FEA104E4EEA45
:1026F000014E10EB0E0041EB1141401841F1000179
:102700004FEAD00040EA41704FEAD10110EB80055A
:102710004FEA810444EA907444EB01046D1944EBE0
:102720000404521BA3414FF0000348BF0A3200D5F6
:1027300030BD401C41F1000130BD10B50446FDF72D
:1027400023FF0068005D00F0010010BD2DE9F0419D
:102750001F46044603260168072A01F4006004DBD3
:1027600008B116A505E016A503E008B115A500E01F
:1027700015A521F010002060A069C01EA0610FB156
:10278000401EA0612046FEF74DF84FB1D4E901216B
:1027900038469047206A401C2062C01C206206E038
:1027A000206AFAE7D4E9012115F8010B9047761E5B
:1027B000F8D22046FEF74CF8BDE8F0814E414E00BD
:1027C0006E616E00494E4600696E660010B5436941
:1027D00013B1AFF3008001E0FFF77CF9012010BDD9
:1027E000128800F1240182840022C2840122EDE7D4
:1027F00011684FF0FF32E9E72DE9F34F4FF0000A7F
:102800000C4656468DB001200C9001F10C000B9047
:1028100062690B9801219047051E2DD0252D2CD0E3
:10282000216A8847C0B162690B9801219047216AEB
:1028300088470028F7D16269411E0B98904700E055
:10284000761CA1690D988847216A88470028F7D12E
:10285000E1690D988847DBE7A1690D988847A84290
:10286000074601D1761CD3E7E1690D9888477F1CA4
:1028700002D1BAF1000F6FD06CE162690B980027AA
:102880003D46394690472A2804D162690B980121B8
:1028900090470125DFF8D08262690B9801219047AB
:1028A000A0F130010A290AD24745E5DC07EB870190
:1028B00000EB4107303FDFD445F01005ECE7E906B7
:1028C00001D46FF000476C280AD04C2814D0682837
:1028D00015D06A280DD074281CD07A281AD01DE093
:1028E00062690B98012190476C2802D045F00405DD
:1028F00014E045F002050DE045F020050AE06269AC
:102900000B9801219047682802D045F0080505E0A2
:1029100045F4006562690B9801219047C4E90157AD
:1029200065283DD019DC58287AD00CDC452837D0F2
:1029300004DC252826D041289ED131E046282FD01E
:10294000472899D12CE05B2877D0612828D06328CC
:102950007CD0642823D15AE0F7E06F2848D008DC07
:1029600066281DD067281BD0692821D06E2816D173
:1029700027E0702845D0732868D0752847D078287C
:102980000DD14DE0A1690D988847252805463FF4F3
:1029900069AFE1690D9888476D1C3FF46AAFD9E0D3
:1029A0000D9923466A466FF0010082F0BEFAC6E038
:1029B00045F0400023464FF000026060A80736D47F
:1029C0003EE0E8077FF447AF2068011D2160006802
:1029D000290501D506701BE7290701D5068017E7F1
:1029E000A90703D5F117C0E9006111E706600FE7F9
:1029F00045F0400023464FF008026060A80716D457
:102A00001EE040F60E0125EA0100606016E045F088
:102A1000400023464FF00A026060A80707D40FE089
:102A200045F040006060A80708D5234610220D99A4
:102A30006FF00100AFF3008081E007E01022234631
:102A40000D996FF00100FEF7B7F878E04FF000093C
:102A500063284F46C8464B46CB4602D05B2807D07A
:102A600039E02079C00601D40120A060012732E0BE
:102A70006269D4F80CB00B98012190475E2807D109
:102A80004FF0010949466269D4F80CB00B989047A1
:102A9000216939B900210A4603AB43F82120491CBA
:102AA0000829FADBD8B3216949B308F10108626942
:102AB0000B98012190475D28F4D1B9F1000F09D09E
:102AC000002003A951F82020D24341F82020401CC7
:102AD0000828F7DB03AB2069002820794FEA407013
:102AE0001ED05B462246CDF80080CDE901970D99B6
:102AF00000286FF0010020DAAFF300801FE0C1175B
:102B000003AA00EBD1614B1121F01F0102EB8302FC
:102B1000411A13680120884003431360C7E719E096
:102B20000D99224600286FF00100009702DAAFF3FA
:102B3000008004E0FEF7E6F801E0AFF30080002833
:102B40000ADA401C06D10C9820B14FF0FF300FB0CC
:102B5000BDE8F08F5046FAE7E90701D10AF1010A12
:102B6000064400200C9053E6CCCCCC0C2DE9F05F51
:102B7000824615468B4600270AF10104B9460078C3
:102B8000302801D09DB113E014F8010B01277828FB
:102B900003D0582801D045B10AE00DB1102D07D15E
:102BA000002714F8010B102502E0082500E00A2593
:102BB0000026B0460EE005FB080005FB06F10127E4
:102BC0001FFA80F801EB1046B6F5803F00D3B946F6
:102BD00014F8010B2946FFF751F80028EBDABBF196
:102BE000000F05D00FB1641E00E05446CBF8004042
:102BF000B9F1000F06D0FEF7CFFA02210160C81E1E
:102C0000BDE8F09F48EA0640FAE700002DE9F047EA
:102C1000814616468AB0354878440DC88DE80D00C7
:102C200032487844801C03AC0DC884E80D0041F69E
:102C30009B300844372190FBF1F290FBF1F5A5F1B0
:102C4000800501FB12041B3C02D56442012000E018
:102C50000020DFF898A080460027FA44AAF1BE0AB7
:102C60000EE0E0070AD03246684607EB4701012331
:102C70000AEB810100F01CFF8DE8070064107F1C47
:102C8000002CEED1194F7F44AE3F19E0E80715D074
:102C900007EB04100DF1180A90E80E008AE80E0008
:102CA000C068F04201D1981908903246012306A964
:102CB00003A800F0FDFE03AB83E807006D10641C61
:102CC000002DE3D14FF0010332466946B8F1000F01
:102CD00003A802D000F0C2FE01E000F0E9FEC9E95D
:102CE0000001C9F808200AB0BDE8F08730280800C4
:102CF00010B50146C268900703D0900607D5886AD0
:102D00000AE0FEF749FA01210160881E10BD8B69B7
:102D1000486818440B69C01A91F848301BB191F803
:102D20004910401A10BD1103FCD50028FADD401EE1
:102D300010BD70B5C468A50713D0650211D4B2F5F3
:102D4000807F09D0B2F5007F06D0B2F5806F08D140
:102D5000012300F1240106E05D1E6FF07F46B542BD
:102D600001D3012070BD0161C361416024F4706131
:102D70001143C160002070BD2DE9F0410C460746AB
:102D80001646104600F06EF82078611C61280AD0C3
:102D9000722802D077283CD102E00125002405E00A
:102DA0000225042402E0082448F2020511F8010B70
:102DB0002B2806D0622809D011F8010C74280AD0FB
:102DC0000BE045F0030544F00204EFE745F004058D
:102DD00044F00104EAE744F01004384621467FF04D
:102DE00003FE411C15D00021316171604FF4007168
:102DF000F560F1617061200704D5304602220021A0
:102E0000FFF786FA306D40F0010030653046BDE8CE
:102E1000F0810020FBE72DE9F0410D460646104CFD
:102E2000206DC10704D0410804D020F00104F7E769
:102E300022460EE05420FDF7AFFB07000ED0206DB8
:102E400047F001010843542120653846FEF73CF95C
:102E50003A4629463046BDE8F0418DE70020D6E7E6
:102E6000ACAE00202DE9F04704464FF000094FF0CA
:102E7000FF37C568D4E90486A80707D02046FFF7C6
:102E8000F7FA30467FF077FD002802DA3846BDE8D1
:102E9000F087280502D54046FDF7ADFB4C212046C2
:102EA000FEF712F9206D20F0010020654846EEE79C
:102EB00070B516460C460546FDF766FB036893F8A9
:102EC0000101012806D0FF2C0FD8185D68B1012040
:102ED0002C7070BDD3F807013246214603F2071368
:102EE00003442846BDE8704018474FF0FF3070BDDE
:102EF00010B500F087FABDE8104000F07EBA10B5BA
:102F000000F09AFABDE8104000F077BA30B50346F9
:102F10001D781DB10A4603E0AC4201D1181A30BD3C
:102F200012F8014B002CF7D15B1CF1E730B50346DA
:102F30001D783DB10A4612F8014B1CB1AC42FAD1E2
:102F40005B1CF5E7181A30BD7546FFF793FBAE46DC
:102F500005006946534620F00700854618B020B5A5
:102F6000FDF700FBBDE820404FF000064FF00007E2
:102F70004FF000084FF0000B21F00701AC46ACE821
:102F8000C009ACE8C009ACE8C009ACE8C0098D468E
:102F9000704700002DE9FF4F1F464FF03C0987B0F6
:102FA0004FF00042DDE9141001F10108DDF858A0EE
:102FB00002EA4050039000200590834605460446EF
:102FC0000490B969461E08988847AAF1010A029040
:102FD000BAF1000F3BDD02982E2815D01021FEF724
:102FE0004DFE00282EDB4FF0010B0599014317D051
:102FF000B9F1000F0BDB4A46C11700F045FA054353
:103000000C43A9F1040905E0012004900BE008B18C
:1030100045F0010501200590049820B9361D02E015
:10302000049800B1361FB969089808F1010888476B
:10303000BBF1000FAAF1010A0290C9D00999C1F8A9
:103040000080C5E70298702808D0502806D0F9699A
:1030500008988847BBF1000F14D04FE00020029081
:103060000120BBF1000F049009D0B969089808F15C
:1030700001088847AAF10109B9F1000F07DCF969D5
:10308000089888476FF001000BB0BDE8F08F2B283F
:1030900004D02D280CD14FF0FF300490B969089866
:1030A00008F101088847A9F10109B9F1000FE6DD2F
:1030B000411CE4D00A21FEF7E1FD0028DFDB029984
:1030C00008F1010801EB810100EB41000290B969B0
:1030D000089888470A21FEF7D1FD099AA9F101094C
:1030E000B9F1000FC2F8008001DD0028E7DAF969C4
:1030F000089888470499029800FB016655EA040085
:1031000004D004F04041090002D006E0039898E0A2
:10311000A40044EA9574AD00B61E04F00041080016
:1031200002D16D196441761E159810F0240F03D05A
:103130004FF00B095C4803E04FF028096FF07D0069
:103140008246564507DAAAEB06018944B9F1410FD8
:1031500001DD4FF0410901200021A9F1010200F039
:1031600093F9024628400B462140084301D0012133
:1031700000E00021501E029143F1FF312840214020
:10318000084301D0012000E000200299834651EA63
:103190000B014FD0002108464FF00000039900F4C6
:1031A000400039B100EB80004FF4400100EBD070DB
:1031B00001EA60008015012802DD4FF0FF3000E0D9
:1031C00013D0401C36D0029860B3BBF1000F0CD175
:1031D0004A460120002100F057F9284021400843C9
:1031E00001D0012000E00020E0B101204A4600218A
:1031F00000F04AF9034640190A4661412D1A8C41F4
:1032000011D3B9F1400F09DD159810F0240F02D049
:10321000AAF1340603E0AAF1170600E0761C0025A7
:103220004FF0004406E05B1E42F1FF3220EA030546
:1032300021EA0204CAF10100B04206DA1B490398F0
:1032400008430190002000900EE0039AC4F3D321BC
:10325000E80A0A43164940EA44500A433146CDE998
:10326000000268467FF024FB159810F0240F0BD065
:103270001598C00715D13868DDE90012031D3B60C1
:103280000068C0E900120CE002A869467FF004FB68
:103290001598C00705D13868029A011D3960006889
:1032A00002604046F0E6000002FCFFFF0000F07FF5
:1032B0000000F03F2DE9FF4F92461D4685B04FF0CC
:1032C0000041DDE9124BDDE914727F1E01EA4B502B
:1032D000414940F0FF4940EA0108002122F0200066
:1032E0004928049102D04E2828D04CE03BA001266A
:1032F00007C88DE80700A9690698641C88477F1EE7
:10330000014606D41DF8060018B121F020018142C3
:103310000BD0E96906988847032E34D0082E32D0A6
:103320006FF0010009B0BDE8F08F761C032E01D0CC
:10333000082EE0D1601CCAF80000DCE7A9690698F5
:10334000641C88477F1E2AD420F02000412826D103
:10335000A9690698641C88477F1E20D420F02000AD
:103360004E281CD1A9690698641C88477F1E48F422
:10337000002849F48009CAF8004001D4282806D062
:10338000E969069888475FEACB7012D022E0A96904
:103390000698641C88477F1E01D4002803DAE96977
:1033A00006988847BCE72928F1D1641CCAF8004078
:1033B000E9E71BF0240F07D028680499031D2B6050
:1033C0000068C0E9001805E02868021D2A6000684E
:1033D000C0F800902046A5E70000F07F494E46491E
:1033E0004E4954590000000010B50446AFF3008068
:1033F0002046BDE81040FDF726B8002801D07FF038
:10340000CDBA704710B5014602A000F050F8012077
:1034100010BD000053494752545245443A2052656A
:103420006469726563743A2063616E2774206F70FB
:10343000656E3A200000000010B5012805D000217B
:1034400003A000F034F8012010BD09A1F8E7000046
:1034500053494752544D454D3A204F7574206F667D
:103460002068656170206D656D6F727900000000E5
:103470003A2048656170206D656D6F727920636FC9
:103480007272757074656400B2F120030AD5C2F1DE
:10349000200301FA02F120FA03F300FA02F041EAF4
:1034A0000301704700FA03F14FF00000704770B558
:1034B00005460C460A2000E06D1C7FF003FB35B189
:1034C00028780028F8D102E0641C7FF0FBFA14B1E0
:1034D00020780028F8D1BDE870400A207FF0F2BAC9
:1034E0005FEA400C08BF91F0000F4FEA8C234FEACF
:1034F000C12243EA51514FEA1C5018BF00F5F04079
:103500004FEA300018BF41F000415FEA6C5C00F008
:103510002980BCF1FF3F08BF40F080407047130C8A
:1035200006BF12044FF0100C4FF0000C130E04BF36
:1035300012020CF1080C130F04BF12010CF1040C61
:10354000930F04BF92000CF1020CD30F04BF520082
:103550000CF1010C11464FF00002A0F11F00A0EB8E
:103560000C00704711F0004F08BF704731F0004168
:103570003FF4D5AF0B0C06BF09044FF0100C4FF011
:10358000000C0B0E04BF09020CF1080C0B0F04BF5A
:1035900009010CF1040C8B0F04BF89000CF1020C23
:1035A000CB0F04BF49000CF1010CCCF12003A0EBC0
:1035B0000C0022FA03F302FA0CF241EA030100F1D3
:1035C0000100704720F07F4C80EA030023F07F4722
:1035D000ACEB070303F57C5300F0004003F1FF035D
:1035E0002DE980494FEA154B09B44FEA144325EA07
:1035F0000B4E24EA03480FF2042606EB1327490872
:103600003E785FEA320203FB0667C7F5000707FB57
:1036100006F64FEA54374FEAD64606F1020607FB94
:10362000066CCCF1005C4FEA1C472CEA074C07FB08
:1036300006F40CFB06F504EB15464FEA961634BF6C
:1036400000204FF000404FEAD13706FB07FC4FEA5D
:103650001C4C0CFB0BF7D21B03FB0CF761EB0701B7
:103660000CFB0EF7B0EB074072EB17420CFB08F7B0
:1036700034BFA2EB0742B2EB074261EB17414FEABE
:103680000C444FEA910706FB07FC4FEA1C4C0CFB6D
:103690000BF7B0EBC74072EB573203FB0CF734BFAC
:1036A000A2EBC742B2EBC74261EB57310CFB0EF7FE
:1036B000B0EBC70072EB57720CFB08F734BFA2EBFC
:1036C000C702B2EBC70261EB5771039F4FEA8161FA
:1036D00041EA921104EBCC044FEAD1374FEA8262FF
:1036E00006FB07FC42EA90124FEA80604FEA1C4C4E
:1036F0000CFB0BF7D21B03FB0CF761EB07010CFB78
:103700000EF7B0EB074072EB17420CFB08F734BF23
:10371000A2EB0742B2EB074261EB17414FEA8C552F
:103720004FEA910704EB9C2406FB07FC4FEA1C4C74
:103730000CFB0BF7B0EBC74072EB573203FB0CF7F7
:1037400034BFA2EBC742B2EBC74261EB57310CFB6F
:103750000EF7B0EBC70072EB57720CFB08F734BFE3
:10376000A2EBC702B2EBC70261EB577115EB4C2518
:103770004FEA816141EA92114FEA82624FEAD13702
:1037800042EA901206FB07FC44F100044FEA806015
:103790004FEA1C4C0CFB0BF7D21B03FB0CF761EB45
:1037A00007010CFB0EF7B0EB074072EB17420CFB66
:1037B00008F734BFA2EB0742B2EB074261EB1741B7
:1037C00015EB1C154FEA813141EA92414FEA8232F2
:1037D00042EA90424FEA80304FEA0C7644F100040E
:1037E00048EA03434EEA0B484FF0000EB2EB080CD8
:1037F00071EB030724BF624639464EEB0E0E4FF0C5
:10380000000B0018524149414BEB0B0BB2EB080C7B
:1038100071EB03077BF1000B24BF624639464EEB88
:103820000E0E4FF0000B0018524149414BEB0B0BB1
:10383000B2EB080C71EB03077BF1000B24BF62466F
:1038400039464EEB0E0E51EA020718BF46F001064C
:1038500016EB0E7655F1000254F1000103D5BDE8D8
:103860008901BDE80088BDE88901BDE80048B619B6
:10387000524141EB0101A3F10103704780807F7E3B
:103880007D7C7B7A797877767675747372717170D6
:103890006F6E6E6D6C6C6B6A6A6968686766666588
:1038A0006464636362616160605F5F5E5E5D5D5C16
:1038B0005C5B5B5A5A595958585757565655555587
:1038C0005454535352525251515050504F4F4F4EE7
:1038D0004E4D4D4D4C4C4C4B4B4B4A4A4A49494935
:1038E0004848484747474746464645454544444477
:1038F00044434343434242424241414146EA064631
:10390000A3F570534FEA164646EA42564FEAD222D2
:1039100042EA415210B54FEAD121A3F1010300F070
:103920002FF820F0004000F1020C00F0004701EBFE
:1039300000501146BCF5006F40EA070000D210BDF0
:10394000BAF1000F0AD01CB503B44FF004004FF0D9
:1039500004014FF000000FBCBDE810404FF0000123
:10396000BBF1010FB9BF04484FF0FF3103480021FC
:1039700040EA070010BD00BFFFFFEF7F0000F07FAF
:10398000002B9C4630D477002BD01CB54FEA37076C
:1039900003B44FF010004FF01001BAF1000F06D041
:1039A000BCF1000FDCBF40F0080040F008014FF010
:1039B00000000FBCBDE810400BF1010BBBF1010F83
:1039C00008BF5FEA170722BF12F1010211F10101DE
:1039D0004FF0004143F1000300F0004043EA0000D3
:1039E0007047F9D35708D0E746EA064613F1400F6F
:1039F0004FEA16461FDD13F1200FDFBF16430A46BC
:103A0000002120335B42BED0C3F1200746EA0646C0
:103A100002FA07F74FEA164646EA0706C3F12007FF
:103A200022FA03F201FA07F721FA03F14FF000033B
:103A300042EA0702A7E746EA020646EA06464FEAD6
:103A4000164646EA0106BCBF46EA0646360C4FF06B
:103A500000034FF000024FF0000194E72DE9804C85
:103A60009A46934670B491E8380007C831EA400C92
:103A700048BF34EA430C03D5FFF7A4FDFFF780FFEE
:103A8000F0BCBDE8008C2DE9804C9A46934670B49A
:103A900091E8380007C831EA400C48BF34EA430CCB
:103AA00003D5FFF78FFDFFF729FFF0BCBDE8008CC1
:103AB0002DE9804C9A46934670B491E8380007C8C7
:103AC00010F0804F08BF13F0804F03D100F01AF8B8
:103AD000FFF756FFF0BCBDE8008C2DE9804C9A46FC
:103AE000934670B491E8380007C810F0804F08BFC3
:103AF00013F0804F03D100F005F8FFF7FFFEF0BC94
:103B0000BDE8008C20F07F4780EA030023F07F4C63
:103B100007EB0C03A3F57C5300F00040A3F1FE0378
:103B200092F0000F00F0B38095F0000F00F0778066
:103B30002DE901494FEA11404FEA144621EA0048B5
:103B400000FB06FC24EA064708FB06F607FB08F81C
:103B500000FB07F718EB06484CEB164C4FEA124BEC
:103B600018EB07484FEA15464CEB174022EA0B4E7C
:103B70000BFB06FC25EA06470EFB06F607FB0EFECE
:103B80000BFB07F71EEB064E4CEB164C4FF00006F6
:103B90001EEB074E4CEB174B18EB0B0840F10000E7
:103BA00018EB0E0B58EB000840F100008F1A4FF095
:103BB00000013CBFC943661B14BFB5EB040C0021D8
:103BC0003CBFC943F61B4FEA17444EEA8E0E27EA64
:103BD00004454FEA1C4704FB07622CEA074C05FB2F
:103BE00007F70CFB05F604FB0CFC16EB074642EB53
:103BF000174216EB0C4642EB1C421BEB060658EB39
:103C00000202414146EA9E0601D5BDE80189B61986
:103C1000524141EB0101A3F10103BDE801894FEAE3
:103C200014454FEA114724EA054621EA074C05FBF3
:103C300007F406FB07F70CFB06F105FB0CFC11EB88
:103C4000074144EB17444FEA124711EB0C4144EB98
:103C50001C4422EA074C05FB07F206FB07F70CFBA6
:103C600006F605FB0CFC16EB074642EB174216EB7B
:103C70000C4642EB1C456A1854F1000148BF7047DE
:103C8000B619524141EB0101A3F10103704795F0D0
:103C9000000F37D04FEA11424FEA144721EA02469B
:103CA00024EA074C02FB07F106FB07F70CFB06F4BE
:103CB00002FB0CFC14EB074441EB17414FEA15479C
:103CC00014EB0C4441EB1C4125EA074C02FB07F5C1
:103CD00006FB07F70CFB06F602FB0CFC16EB07468F
:103CE00045EB174516EB0C4645EB1C42121951F1FA
:103CF000000148BF7047B619524141EB0101A3F1E1
:103D0000010370474FEA14454FEA114724EA05467C
:103D100021EA074C05FB07F106FB07F70CFB06F24F
:103D20004FF0000605FB0CFC12EB074241EB17417C
:103D300012EB0C4251EB1C4148BF7047921841EB0B
:103D40000101A3F10103704741F2ED4CC0F2000CF8
:103D5000604741F6350CC0F2000C604741F6713CFB
:103D6000C0F2000C604740F21D2CC0F2000C60470E
:103D70002DE9F04104460D4627462E46002F00DC73
:103D80000127002E00DC012617E0FE4840780428B9
:103D900002D1FD48806968B9FC48008848F20101F9
:103DA000084038B9F848808C20B902220021084622
:103DB00056F02FFE38467EF0D3FFF448008800F01E
:103DC00001000028E1D0F048806928B90420F049BA
:103DD00008700020BDE8F08130467EF0C1FFE94860
:103DE0004078042801D00020F4E70120F2E770B504
:103DF000054632207EF0B4FFE648007800F001006E
:103E000028B1E548007810B932207EF0A9FFE148DA
:103E1000007800F0010010B1DF48007808B90120F7
:103E200070BDDE48008800F0010008B90120F7E706
:103E3000052405B1142413E0D2484078042801D0A9
:103E40000020EDE70020D6490862C86132207EF0EC
:103E500087FFD348C06908B90120E1E7601EC4B2FA
:103E6000002CE9DC0120DBE72DE9F0412DED0A8B88
:103E700004460D4616461F46CA4890ED260BB0EE86
:103E8000409B90ED560AB7EEC00AB0EE408B90ED25
:103E9000520AB7EEC00AB0EE40CB90ED320BB4EE52
:103EA000C80BF1EE10FA03D290ED320BB0EE408B5E
:103EB000BC4890ED320BB4EECC0BF1EE10FA03D20D
:103EC00090ED320BB0EE40CB66B1B7EE000BB4EE26
:103ED000C08BF1EE10FA03DDB7EE000BB0EE408BB5
:103EE000B0EE48CBB04890ED000B20EE080BB7EEDB
:103EF000C0ABB5EEC0AAF1EE10FA03D19FEDAB0A4C
:103F0000B0EE40AAA049C96B681A002801DB01463F
:103F100000E0414200EE101AF8EEC0AA8AEE8ABA1A
:103F2000B0EE000AB4EEC0BAF1EE10FA03DD9D481F
:103F300080ED26CB02E09B4880ED268BAFB39C48FA
:103F400030C09C4890ED000AF2EE040A80EE201A80
:103F5000B7EEC11A944890ED002B954890ED010AF8
:103F6000B8EEC00B01EE420BBDEEC00B80ED010AB6
:103F700000234FF480621946012054F0FFFE0A210D
:103F80000846FFF7F5FE38B9864880ED269B0020ED
:103F9000BDEC0A8BBDE8F0810020FFF728FF28B9AF
:103FA000804880ED269B0020F2E702E07D4880ED0E
:103FB000268B7F4830C000234FF4806219460120D1
:103FC00054F0DCFE0A210846FFF7D2FE20B97548FE
:103FD00080ED269B0020DBE70120FFF708FF20B9DA
:103FE000704880ED269B0020D2E76E4880ED269B2E
:103FF0000120CDE71CB500200090019066490978AA
:10400000E9B36449097801F00101C1B36A4991F843
:104010004A1001F0010191BB6849897801F0010162
:1040200069B3614991ED000B9FED651B20EE010B1B
:10403000B0EE002B80EE021B63494868002801DBCC
:10404000014600E0414200EE101AB8EEC00BB4EE9B
:10405000C01BF1EE10FA15D20121002031F081F8D9
:10406000CDE900014848C06B0199411A4648406CAF
:10407000014445484164444ADDE9001000E001E0A4
:10408000C2E90E10474890F8240148B9454890F815
:104090003401032804D04D48007800F0010060B1DD
:1040A0009FED4B0A434880ED000A3E4890F82401FA
:1040B00040F080004749087007E09FED3C0A3D480A
:1040C00080ED000A002043490870364890ED260B29
:1040D000414880ED000B334890F810033F490870C9
:1040E0003048B0F810013E4908802E4890F8180179
:1040F0003C4908702B4890EDB20A3B4880ED000A1D
:10410000284890F8240139490870264890F8EC04B2
:10411000374908700020234981F8240181F8EC0414
:1041200081F810036420A1F81001002081F8180123
:10413000084690ED040BB2EE081BB4EEC10BF1EE95
:1041400010FA0DDD90EDB20AF7EE000AB4EEE00AC7
:10415000F1EE10FA04D2B7EE000A80EDB20A0DE0DB
:10416000104890EDB20ADFED110AB4EEE00AF1EE6C
:1041700010FA03D29FED0D0A80EDB20A18480088AC
:10418000642837E00006002020070020F00500200A
:10419000A69B0424B40500204C05002050050020F7
:1041A000D00900203006052458010024CDCCCC3D98
:1041B000E0080020189B042488030020B402002497
:1041C000000000A09999B93F58050020BA4200307C
:1041D000B4A29139A29B0424809A0424A09A0424B6
:1041E000A89A0424A49A0424B09A0424789A042453
:1041F0007C9A042402DA0A207EF0B2FDFE48407860
:10420000082821D10420FC4948700198E0B1FB48FE
:10421000007800F0010068B140F2E240F849C8843B
:1042200002E001207EF09CFDF548B0F9260001284F
:10423000F7DC09E0F148007830B1F249B1F8B0128A
:1042400001F10A007EF08CFD0120EF4908701CBDD1
:1042500010B5ED48007800B910BD002012F034FD13
:10426000EA480078E74981F82401E948007881F8B4
:10427000EC04E84890ED000B084680ED260BE6487C
:10428000007881F81003E548008800B2A1F8100119
:10429000E348007881F81801E24890ED000A0846EA
:1042A00080EDB20AE04890F8480020F01000DE49A6
:1042B00081F8480000BFCFE7D24890EDB60ADB484E
:1042C00080ED000ACD480078D9490870CD4890F8B3
:1042D000BC02D8490870CB4890F8C002D649087093
:1042E000C848B0F8B002D5490880C648B0F8B00256
:1042F0003F2803DA3F20C349A1F8B0024FF0FF3056
:10430000CF490860BF48D0F8AC02B0F51C7F08D890
:10431000BC48D0F8AC02086040F27120B949C1F83D
:10432000AC02C14890F8500000F0400058B1B548C8
:1043300090EDA00BB1EE001B20EE010BB7EEC00B11
:1043400080EDB60A10E0B84890F8500000F0040084
:1043500050B1AC4890ED8C0BB0EE001B80EE012B01
:10436000B7EEC20B80EDB60AA64890EDB60ADFEDB7
:10437000B50AB4EEE00AF1EE10FA03D29FEDB10AED
:1043800080EDB60AA94890ED000AF2EE040A80EE2C
:10439000201A9C4890EDB60AB4EEC01AF1EE10FA5D
:1043A0000ADDA24890ED000AF2EE040A80EE201A1F
:1043B000944880EDB61A17E0924890EDB60A9B48F3
:1043C000D0ED000AB2EE041A60EE810AB4EEE00A03
:1043D000F1EE10FA08DD90ED000AF2EE040A20EE8C
:1043E000200A884880EDB60A864890F8BC02022868
:1043F00003DA0220834981F8BC02824890F8C002A7
:10440000022803DA02207F4981F8C0027D4890F833
:10441000A402022811DA7B4890F8BC02142803DDBC
:104420001420784981F8BC02764890F8C00214281C
:1044300003DD1420734981F8C00202206F4908701F
:1044400070477F4800680021494071EA000004D0AD
:104450007B4800686B49C1F8AC024FF0FF307849E7
:104460000860764800886749A1F8B0026F4890ED6F
:10447000000A084680EDB60A6D4800785F4908706A
:10448000604890F8A40202280BDA694800780870A6
:10449000684800785B4981F8BC026748007881F879
:1044A000C002704770B505464DB96748007820B91D
:1044B000FF2065490870012070BD0020FCE74FF423
:1044C000FA76632400BF4C484078042801D00020CD
:1044D000F2E7301EA6F101010EB204DC0A205B49AE
:1044E00008700020E8E7584890F90000002803DA37
:1044F0000020554908701BE0534890F90000A04285
:1045000013D0514890F90040002C0CDB5048807DBE
:10451000A04208DD0120A0404E490978084010B1B2
:1045200040F26B3601E04FF4FA7628207EF018FC5A
:10453000454800780028C6D10120BDE770B5334852
:104540000078002800DD70BD2D48D0E90E452D48CB
:1045500090F8E40102282ADB3F4890ED140BB5EEF9
:10456000C00BF1EE10FA08D83C48D0F8800000F4F7
:10457000802010B900243A4D19E0374890ED141B03
:10458000384890ED002B21EE021B9FED372B21EEDA
:10459000021BB0EE410B51EC100B80F001FC241A11
:1045A00065EB0105324830C00120324908701548DA
:1045B00090F8C80100281ED12F4830C02F4830C0C5
:1045C0002F4830C00F4890F8EE0100F0010088B18C
:1045D0000C4890F8D001012872D00A4890F8E40104
:1045E00002286DDA27484068002869DD2248D0E9B2
:1045F000003049E064E09CE0000600204C0500200B
:104600002007002030060524CA9A0424789A04243E
:104610007C9A0424809A0424A09A0424A89A04244E
:10462000A49A0424B09A042488030020289B04241C
:10463000389B04243C9B0424409B0424449B042476
:104640004C9B042417B7D138A09B0424A69B0424B8
:104650004000002488420030300A052490340024B1
:1046600000000C8158010024000000000000F0410F
:10467000D89A0424CE9A042460060020A0060020C4
:10468000E006002048350024FA49D1E900219A18B3
:104690004841F949C1E9002003C9F84A03C2F64874
:1046A000D0E90010F64AC2E90010F34903C9F54AFF
:1046B00003C2F548407840F00100F349487038E003
:1046C000F24890ED000AB5EEC00AF1EE10FA30DDC6
:1046D00090ED001AB7EEC11AED4890ED002B31EEC7
:1046E000021BEC4890ED002B21EE021B1FED222B4C
:1046F00021EE021BB0EE410B51EC100B80F050FB91
:10470000DD4A03C20120E4490870DB48D0E900100B
:10471000DA4AC2E90010D84903C9D94A03C2D649C6
:1047200003C9D84A03C2D848407840F00100D649AE
:10473000487000BF07E72DE9F0412DED028BD74807
:10474000007850B10020D5490870D54991F8A812D9
:10475000490001F164007EF003FBD24890ED000BAC
:104760009FEDD11B81EE002BCD4880ED262BD0484C
:10477000D0E90E45CF4830C0C949B1F85010080300
:10478000C11700EBD161CB4A526802EB6111C94AF3
:10479000516000234FF480621946012054F0EEFA74
:1047A000FA210A20FFF7E4FA20B90020BDEC028BC1
:1047B000BDE8F081BE48C06BBE494968884201D05F
:1047C0000020F3E7BA48D0E90E10BA4AC2E9001057
:1047D00010464068B249B1F850104FF4805202FBC5
:1047E0000100B44948609FEDB48B4FF0000815E01C
:1047F00001207EF0B5FA4FF0FF320121002030F0A9
:104800005EFB064680F036F941EC100B38EE400BAB
:10481000B0EE408B08F1010000F0FF08B8F1080F7E
:10482000E6DB00234FF480621946012054F0A6FA1B
:10483000FA210A20FFF79CFA08B90020B6E79C4845
:10484000C06B9C494968884201D00020AEE74FF018
:10485000000815E001207EF083FA4FF0FF320121BD
:10486000002030F02CFB064680F004F941EC100BE0
:1048700030EE080BB0EE408B08F1010000F0FF08AD
:10488000B8F1080FE6DB8A49D1E90E01894A03C273
:104890008349B1F850100803C11700EBD161083A01
:1048A000526802EB6111834A516000234FF4806229
:1048B0001946012054F062FA0A210846FFF758FA17
:1048C00008B9002072E77A48C06B7A494968884283
:1048D00001D000206AE77648D0E90E10754AC2E997
:1048E00000106F49B1F850100803C11700EBD161F7
:1048F0005268A2EB61116F4A516000234FF480624D
:104900001946012054F03AFAFA210A20FFF730FA4A
:1049100008B900204AE76648C06B66494968884282
:1049200001D0002042E76249D1E90E01614A03C289
:10493000604840685A49B1F850104FF4805202FB69
:1049400011005C4948604FF0000815E001207EF03E
:1049500007FA4FF0FF320121002030F0B0FA06468E
:1049600080F088F841EC100B30EE080BB0EE408B75
:1049700008F1010000F0FF08B8F1080FE6DB0023A2
:104980004FF480621946012054F0F8F9FA210A2008
:10499000FFF7EEF908B9002008E74548C06B454924
:1049A0004968884201D0002000E74FF0000815E078
:1049B00001207EF0D5F94FF0FF320121002030F0C8
:1049C0007EFA064680F056F841EC100B38EE400BAC
:1049D000B0EE408B08F1010000F0FF08B8F1080FBD
:1049E000E6DB374890ED001B9FED362B81EE020B86
:1049F00020EE080BB0EE408B2E4830C000234FF461
:104A000080621946012054F0B9F90A210846FFF7DF
:104A1000AFF908B90020C9E62548C06B25494968A7
:104A2000884201D00020C1E69FED280BB4EEC08B78
:104A3000F1EE10FA10DB9FED270BB4EEC08BF1EE18
:104A400010FA09D8164880ED048B0021084612F0B0
:104A5000CEFA0120FFF7CBF90120A7E670B52DEDC6
:104A6000028B04460D4616461DB90120BDEC028B93
:104A700070BD33E048350024F89A042480060020F5
:104A8000C006002000070020A40B002024350024CD
:104A90004002002458010024D29A04244C0500202E
:104AA0003006052498010024000000A09999C93F10
:104AB00020070020E00800200000000000000000A7
:104AC0007801002400000000000030422D431CEB60
:104AD000E2361A3F00000000000059404EB1FF20AE
:104AE000FD4981F8FC002EF06AFE60B2FA4981F8B7
:104AF000FC00C4EBC400F94901EB0010D0E90E1032
:104B0000F74A02EBC402C2E90010F54800EBC4000A
:104B100040682844F24901EBC4014860F14800EBC9
:104B2000C40090ED008B20462FF0AEFFB7EEC00A18
:104B3000EC4800EBC40080ED000B0121A140C8B29D
:104B400000234FF48062194654F018F9E54800EB51
:104B5000C40080ED008B00BF0A207EF001F9E2481E
:104B600030F8140000F0010028B9E04800EB4400E0
:104B700040780428F0D00A207EF0F2F8D64890F968
:104B8000FC00A04208D1FF20D34981F8FC00204658
:104B90002EF08EFE2EF013FED44800EB4400407839
:104BA000042803D00020BDEC028B70BD0120FAE781
:104BB0002DE9F0412DED028B04460025C64890F802
:104BC000500000F0010000B10125C34890F84A00F0
:104BD00020F00100C04981F84A001FED490BB0EEFA
:104BE000408B4FF0FF320021084630F068F906464E
:104BF0007FF040FF41EC100B38EE400BB0EE408BE5
:104C000001207EF0ADF84FF0FF320021084630F071
:104C100056F906467FF02EFF41EC100B38EE400BA4
:104C2000B0EE408B2A4621460020FFF717FFAF4821
:104C30004078042804D00020BDEC028BBDE8F08150
:104C400064207EF08DF84FF0FF320021084630F0EE
:104C500036F906467FF00EFF41EC100B30EE080BE4
:104C6000B0EE408B01207EF07BF84FF0FF32002148
:104C7000084630F024F906467FF0FCFE41EC100BAC
:104C800030EE080BB0EE408B9FED990B88EE001BC9
:104C9000B0EE418B904890F84B0000F001000028E6
:104CA00079D08D4890F84A0000F00100002872D1B8
:104CB000B0EEC81B00EE104AB8EEC00BB0EE002BF1
:104CC00020EE020BB0EEC00BB4EEC01BF1EE10FAFA
:104CD00061D8B0EEC81B00EE104AB8EEC00BB6EEBD
:104CE000002B20EE020BB0EEC00BB4EEC01BF1EEB9
:104CF00010FA50DB8048007800F0010050BB00EE55
:104D0000104AB8EEC00B28EE000BB5EEC00BF1EE6A
:104D100010FA09D27348983890F8520280F00100D6
:104D20007049983981F852026B4890F85000042875
:104D300011D16C48983890ED8C0B9FED701BB4EE40
:104D4000C10BF1EE10FA06DD6B48007820F001008F
:104D50006949087027E0604890F8500000F0400072
:104D600090B16048983890EDA00B9FED641BB4EEB5
:104D7000C10BF1EE10FA07DD5F48007820F001006A
:104D80005D4908700FE006E05B48007840F00100E4
:104D90005949087007E0002C05DD5748007820F0DD
:104DA0000100554908705448007800F0010010B91E
:104DB00000202EF021FD01203EE770B52DED028B85
:104DC00086B00020049005904648983890F8E40199
:104DD000022813DB4B4890ED141B4B4890ED002B41
:104DE00021EE021B9FED492B21EE021BB0EE410B81
:104DF00051EC100B7FF0D4FFCDE904011FEDD20B75
:104E0000444880ED000B344890F84A103A48007846
:104E1000884300F00100E0B32F4890F8500000F004
:104E20003000B0B33C4890ED010AB8EEC00BB0EED4
:104E3000408B01207DF094FF374890ED010AB8EED9
:104E4000C00B30EE080BB0EE408B01207DF088FFE8
:104E5000314890ED010AB8EEC00B30EE080BB0EE11
:104E6000408B01207DF07CFF2B4890ED010AB8EECD
:104E7000C00B30EE080BB0EE408B1A48983890ED1E
:104E8000A00B20EE080BB1EE001B80EE012B214899
:104E900000E002E080ED002B00BF1248983890F847
:104EA000D001012849D11D48007800F0010090B9D7
:104EB0000A48D0E90E60DDE90415721A60EB0501BD
:104EC00010467FF0D7FD41EC100B154890ED001B0C
:104ED00020EE010B26E030E08803002020070020B0
:104EE000E0080020C8060524F00500200006002088
:104EF0000000000000000042B40500209A99999932
:104F00009999B93F300A0524580100240000000097
:104F10000000F04160020024D805002088420030E3
:104F2000780100241FED071B80EE012BFD4880ED6A
:104F3000002B06B0BDEC028B70BD9FEDFB0BF9485A
:104F400080ED000BFA48007800F0010010B132202B
:104F50007DF006FFF74804780020F6490870F44811
:104F6000007800F0010018B114B164207DF0F8FE63
:104F70009FEDED0BF04880ED000BF048006840F02D
:104F80000100EE49086000BF00BF00BFBFF34F8FB4
:104F9000BFF36F8F00BF00BF00BFE948D0E90E101C
:104FA000DDE90423891A60EB0300CDE90210E4482F
:104FB000D0E91020DDE9021351185841E04AC2E956
:104FC00010101046806D0399401A11468865DDE97E
:104FD0000401C2E90E0100BF00BF00BFBFF34F8F45
:104FE000BFF36F8F00BF00BF00BFD448006820F040
:104FF0000100D2490860D34890F8A70000F00100F2
:1050000000286FD0CF4890F89C0000286AD0CD4887
:1050100090F89800002865D1CA4A92F93820002AF1
:1050200014DBC84A92F93830C74A02EB831292ED7A
:10503000020AB7EEC00AC54A92ED001B20EE010B32
:10504000BDEEC00BBF4A82ED040A02E00022BD4B58
:105050001A61BC4A136A1569B94AD26BAA1A83FB52
:1050600002202CE0BA4A12880192BA4A1268111A38
:105070000A2905DDB74A12680A3AB64B1A6007E0FA
:1050800011F10A0F04DAB34A12680A32B14B1A60FE
:10509000002905DDAF4A1268521EAE4B1A6006E0C9
:1050A000002904DAAB4A1268521CAA4B1A6000E0CD
:1050B00000BFA74A1288BDF804309A42F8D0A54A2A
:1050C00012688242CED19F4A92F8A020002A08DDC1
:1050D0009C4A92F8A020062A03D00122994B83F81B
:1050E0003C2000BF9C4890F85000A8B30A207DF0F7
:1050F00037FE994890F8500000F03000B8B9974852
:1051000090F8520200F0010088B14FF0FF3100200A
:1051100030F027F80023424263EB0100DDE904315F
:10512000D21A60EB01008E49C1E9002010E04FF077
:10513000FF31002030F015F80A460023414263EBAE
:105140000200DDE9042389185841854AC2E90010AC
:10515000012100201BF048F97648047000BFE8E602
:105160002DE9F0417248007800F0010010B90020EC
:10517000BDE8F081784890F8500000F0030008B9CD
:105180000020F5E700250024002613E005207DF02F
:10519000E7FD0121704880F8F810D0F8D8000544E8
:1051A0006D48D0F8E800044400216B4880F8F810FE
:1051B000701CC6B2042EE9DB2846E91705EB917195
:1051C0008D102046E11704EB91718C106248B0F904
:1051D00030002D1A6048B0F93200241A5E49B1F946
:1051E000401001FB04F0C11700EB5151CC12291EF5
:1051F00001DB0A4600E04A42782A08DA201E01DB79
:10520000024600E04242782A01DA0020B0E7B5F514
:10521000004F02DB47F6FF7503E015F5004F00DC99
:10522000504DB4F5004F02DB47F6FF7403E014F570
:10523000004F00DC4B4C21B228B2FEF78AFD074636
:1052400007B90127384693E770B5474800884749B2
:105250000880FFF785FF04463548007800F001001C
:1052600028B99FED310B424880ED000B0FE03B4821
:1052700090ED8C1B00EE104AB8EEC00B21EE000B37
:105280009FED3C1B80EE012B394880ED002B3B4805
:10529000007808B9012070BD0020384908702E48F8
:1052A00090F8500000F0030008B90020F3E7002553
:1052B0002A4890F8280100F0010000B1012530488B
:1052C00020F815402848008820B901202D4921F8F0
:1052D000150005E02548008800B22A4921F815008C
:1052E00034B91E4890F85402022801D10020D2E7B8
:1052F0000120D0E72DE9F04781460025174890F8B6
:10530000280100F0010000B10125144890F8540272
:10531000022839D0114890F85402032834D00020D4
:10532000BDE8F087400200240000000000000000FB
:10533000B40500204C050020D8000024E00C00201B
:1053400020070020C4330024E85500305801002411
:10535000AE0B00202C060020880300203006052418
:10536000B80500200180FFFFA8020024800200246D
:1053700020020024000000000000F04084420030C1
:105380008802002498020024F948007810B1002017
:10539000BDE8F087F74890F8540202281AD1F64881
:1053A00030F81500A0B1F548007800F0010078B1A0
:1053B000F04890ED8C0B9FEDF21BB4EEC10BF1EEBB
:1053C00010FA05D3F04890F8500000F0030008B937
:1053D0000020DDE7E74890F85402032805D1EB48A8
:1053E00030F8150008B90020D2E7E94840780428D1
:1053F00002D04FF0FF30CBE70020FEF7F8FC10B9E9
:105400004FF0FF30C4E732207DF0AAFCFFF7A8FE82
:105410008046D84890F85402022860D1B8F1000FB5
:105420005DD0D54830F8150008B90020B0E7D24863
:1054300030F91500A8EB0004B4F5004F02DBA4F529
:10544000803404E014F5004F01DC04F58034C948D1
:1054500090F82801C74991F85212484000F0010025
:1054600000B16442C34890F8280100F0010000B97F
:10547000644214F57A5F01DA002089E7B4F57A5FB7
:1054800001DD002084E70120C249088094B3B948B7
:1054900090ED8C2B01EE104AB8EEC11B22EE011BE1
:1054A000BD4890ED002B21EE021B1FED4E2B21EE8F
:1054B000021BB0EE410B51EC100B7FF071FCB74AB0
:1054C000D2E90E32C61841EB02074B4601223046A4
:1054D0003946FEF7C9FC68B94FF0FF3058E7A548D8
:1054E00090F8540203282FD1A84830F8150010B9BD
:1054F00000204DE72AE0AA480088A44931F9151098
:10550000441AB4F5005F02DBA4F5804404E014F50E
:10551000005F01DC04F58044964890F8280100F013
:10552000010000B9644201209A49088074B19B4887
:10553000C06B071900264B46012230463946FEF75C
:1055400093FC18B9701E23E7002021E701201FE714
:1055500070B52DED028B82B00024924890ED040AC4
:10556000B8EEC00B20EE000BB0EE408B90ED050ABC
:10557000B8EEC01B90ED050AB8EEC02BB0EE480B9C
:1055800001EE020BB0EE408B8748007800F010006F
:1055900018B96120854908701AE07848007800F051
:1055A000010090B19FED820BB4EEC08BF1EE10FACA
:1055B0000BDB8148007818B162207C49087007E055
:1055C00063207A490870012402E06420774908705A
:1055D00074480169794801627248416977480163FA
:1055E0007048C168754801610021016400BF322024
:1055F0007DF0B6FB5F4890F8E401022803DB002150
:10560000009101913FE05B4890ED6A1B6C4890ED82
:10561000000AB1EE400AB7EEC00AB4EEC01BF1EECC
:1056200010FA15D290ED001AB7EEC11A5A4890ED53
:10563000002B21EE021B9FED632B21EE021BB0EE2F
:10564000410B51EC100B7FF0ABFBCDE900011AE0F0
:10565000484890ED6A2B5A4890ED001AB7EEC11AEF
:1056600032EE011B4C4890ED002B21EE021B9FED0A
:10567000552B21EE021BB0EE410B51EC100B7FF0CD
:105680008FFBCDE9000149480078612809D14F49D5
:10569000DDE90020D1E90031D2184841CDE90020F0
:1056A00033E042480078642809D13E4ADDE9001021
:1056B000D2E90032C9185041CDE9001025E04FF47D
:1056C0008062012100202FF0FAFBDDE90023801821
:1056D0005941CDE9000135480078632815D14FF0D4
:1056E000FF32012100202FF0EAFBDDE90032181A19
:1056F00062EB0102CDE90002284BDDE90020D3E98D
:105700000E1351185841CDE9001026488068002832
:1057100004DD244901988968401A01900020009016
:1057200001230022DDE900512846FEF79DFB20B948
:10573000002002B0BDEC028B70BD0120FEF757FBCC
:1057400008B90020F5E7201EA4F101014CB23FF793
:105750004EAF0120EDE72DE9F0412DED048B0C4813
:105760004078042834D00020BDEC048BBDE8F081E3
:10577000844200303006052488020024B40500204D
:105780007B14AE47E17A943F8803002098020024FE
:1057900000060020F005002058010024200700200A
:1057A000A8020024680C0020C80C00200000002083
:1057B0000000008030E663414C0500203869042475
:1057C000189B0424000000000000F041809B04248A
:1057D0000120FD4908809FEDFD0BFE4880ED000B88
:1057E0000020FD4908809FEDF90BFC4880ED000B7F
:1057F0000020FEF7FCFA20B90020BDEC048BBDE8C8
:10580000F081F749D1E90E01F64A03C20025F648B6
:1058100090F8D00180B1F44890F8D00103280BD063
:10582000F14890F8500200F0010028B1EF480078EC
:1058300000F0010000B90125EB4890F8D00130B12B
:10584000EB48007800F0010008B9002D7ED000E0A0
:1058500000BFE84890F900000028F9DA0020E54987
:1058600008702FF069F840B1E34890F84A0040F022
:105870000100E14981F84A0007E0DF4890F84A005A
:1058800020F00100DC4981F84A00FF20D949087066
:10589000D54890F8500200F00100002872D0D64898
:1058A00090F84A0000F0010000286BD1D24890F82F
:1058B0005000002866D0CC4890F8D00103287FD053
:1058C000CE48007840B10020CC490870C64991F814
:1058D000A81248007DF044FAC74890F8500000F044
:1058E000070038B1C04890ED8C0BB0EE001B20EEE5
:1058F000018B06E0BC4890EDA00BB3EE041B20EE3C
:10590000018B9FEDBF0BB4EEC08BF1EE10FA05D208
:10591000B0EE000B28EE000BB0EE408B9FEDB80B05
:10592000B4EEC08BF1EE10FA03D29FEDB50BB0EEE2
:10593000408BB54890ED000B20EE080BBDEEC00B80
:1059400010EE104A0120FEF7ADFD00E047E008B977
:10595000002052E700202DF0E9FE00202DF04CFF42
:105960002046FFF725F920B90020FEF79BFD002017
:1059700043E76042FFF71CF928B90020FEF792FDCB
:1059800000203AE71CE09A48007800F00100B0B12E
:10599000954890ED260BB0EE409BFEF7CCFE50B93B
:1059A000914880ED269B0020FEF77CFD072097495B
:1059B0000870002021E78C4880ED269B00BF0BE09B
:1059C0008A48007820F00100884908700020904A39
:1059D000106050602DF010FF0020FEF763FDFFF710
:1059E000B7FD08B9002008E78A48007880BB7E48E8
:1059F00090F85402022804D17C48007800F001009D
:105A000020B9794890F85402032822D10120FFF7E9
:105A100071FC002801DA0020EFE67448007800F0FD
:105A20000100A8B1704890F85402022811D17348BF
:105A3000007868B90020FFF75DFC002801DA00203B
:105A4000DBE60020FFF756FC002802DA0020D4E64F
:105A5000FFE7FFF7B2F9FEF771FDADB163480078DB
:105A600000F0010080B1604890F8D00101280BD10E
:105A7000811E00202FF075FB594AD2E90E32181A08
:105A800062EB0102624905C15848007800F001004C
:105A900058B16148007840F001005F4908705248F1
:105AA00090F8A4025549087008E05B48007820F09F
:105AB0000100594908700020504908700120FEF784
:105AC00096F908B9002098E6FFF7BEFB08B9002058
:105AD00093E6454890F8E401801E062872D2DFE87C
:105AE00000F003040607393A00BF012085E600BF35
:105AF0004A48007810B14A48007808B900207CE68E
:105B0000484890ED000B384880ED260B4648D0E918
:105B10000030464A06CA5E1840EB0201022200230A
:105B20003046FAF72CFE424A03C200234FF480624B
:105B30001946012053F022F90A210846FEF718F908
:105B400008B9002059E60120FEF751F908B90020F4
:105B500053E697E000BF3148007808B900204CE6D2
:105B6000304890ED000B204880ED260B2E49D1E9FE
:105B7000002110467EF07EFF41EC100B1A4890ED9C
:105B8000BA1AB7EEC11AB7EE082B31EE022B9FED11
:105B9000293B82EE031B1C4890ED002B21EE021BDB
:105BA0001FEDF82B01EE420BB0EE408B51EC180BC1
:105BB0007FF0F6F81E4A03C2FF234FF480620021F3
:105BC00001203BE05CE00000F00500200000000048
:105BD0000000000020020024800200244002002473
:105BE00020070020809B042430060524B4050020F3
:105BF00088420030A19B0424880300204C0500202B
:105C00009A9999999999A93F58010024A69B04242F
:105C1000B80500208442003070340024CE9A042459
:105C2000D29A0424809A0424D89A0424F89A04244A
:105C3000E00800200000000000408F4053F09EF874
:105C40000A210846FEF794F808B90020D5E5F9497D
:105C500003C9F94A03C200234FF4806219460120A8
:105C600053F08CF80A210846FEF782F808B90020A4
:105C7000C3E50120FEF7BBF808B90020BDE501E04F
:105C80000020BAE500BF0120B7E52DE9F04F2DED6A
:105C9000088B83B0044600200290E848007810B9D1
:105CA0001E20E6490870E64890F8500200F0010016
:105CB00028B9012003B0BDEC088BBDE8F08FE148A6
:105CC000007800F0010008B90020F3E7DC4890F804
:105CD0005402012801D00120ECE7DB4890F8500085
:105CE00000F0300008B10120E4E70120D749088026
:105CF000D34890ED040BD64890ED001B20EE010B2D
:105D0000BDEEC00B10EE105ACD4890ED9B0AB7EED9
:105D1000C08AD048007800F0010030B1C84890ED4A
:105D2000520AB7EEC00AB0EE408BC54890ED520A59
:105D3000B7EEC00AB4EEC80BF1EE10FA05D290ED42
:105D4000520AB7EEC00AB0EE408BBD4890ED320B60
:105D5000B4EEC80BF1EE10FA03D290ED320BB0EEB8
:105D6000408BBD48C06B0190DFF8F092002C1EDB29
:105D7000B34890F8ED0100F00200C0B9B84890EDCA
:105D8000000AB5EEC00AF1EE10FA10DD90ED000A3F
:105D9000B7EEC00AAE4890ED001B20EE010BBDEE41
:105DA000C00B10EE100AAC49C96B00EB0109A64804
:105DB00090F8480020F01000A34981F84800002C1A
:105DC0000ADBA84890ED001B21EE081BB0EE410B4A
:105DD00000200EF07CF90BE0A24890ED001BB1EE24
:105DE000482B21EE021BB0EE410B00200EF06FF9A4
:105DF00000BF0A207CF0B4FF9B48407804281BD1E8
:105E000095488069C0B18F48007800F0010098B1D2
:105E10008D4890F84A0000F0010068B9002C02DBC0
:105E20009248807840B9002C02DA9048007818B97E
:105E30008948C06B48450DDB8448008848F2010161
:105E4000084038B98448808C20B9022200210846D5
:105E500054F0DFFD4FF0FF32012100202FF02FF82A
:105E60000E4600BF00BF00BFBFF34F8FBFF36F8F61
:105E700000BF00BF00BF744890F8480000F0100059
:105E800000B90196704890F8480000F0100028B959
:105E90006E48008800F001000028AAD01FEDB50B65
:105EA00000200EF014F932210A20FDF761FF08B935
:105EB0000020FFE6644890F8480000F0100020B988
:105EC00014205E4908700020F4E65F4890F848000E
:105ED00020F010005C4981F848005F48806920B9D3
:105EE0000320564908700020E4E66148008800F06D
:105EF0000300012802D164207CF032FF5A48407828
:105F0000042803D000204D490870D3E64A4901987F
:105F10004860002008604A4890ED8C0BB7EEC0AB9B
:105F20009FED540AB4EEC0AAF1EE10FA04DD9FED25
:105F3000510AB0EE40AA0AE09FED4F0AB4EEC0AAA3
:105F4000F1EE10FA03D29FED4D0AB0EE40AA4C4894
:105F5000D0ED000AB0EE001A80EE810AB4EECA0A53
:105F6000F1EE10FA07D290ED000AF0EE000A80EE92
:105F7000201AB0EE41AA30484168354890ED000B38
:105F8000B7EECA1A20EE010BBDEEC00B10EE100AE0
:105F9000081A29494860002C25DD2F48C06B461996
:105FA0000846406828444860254880ED268B002339
:105FB0004FF480621946012052F0E0FE32210A209F
:105FC000FDF7D6FE08B9002074E62348806908B9B9
:105FD00000206FE624484078042801D0002069E6BC
:105FE0001548466050E0002C4EDA1B48C06B461B3B
:105FF00011484068401B10494860114880ED268BCD
:1060000000234FF480621946012052F0B7FE32217E
:106010000A20FDF7ADFE08B900204BE60E48806966
:1060200008B9002046E61048407804282AD000200D
:1060300040E60000D89A0424E0080020A69B04242F
:1060400030060524B405002088030020F005002058
:1060500058010024BA420030200700200000F47EDE
:10606000243500249801002400060020B8020024F2
:10607000500500200AD7A33C0AD7A33B6F12033B6D
:10608000189B0424FD484660FD4890F8500000F03D
:106090000400E8B1FB4890ED8C0B9FEDFB1B20EE5C
:1060A000019B9FEDFB0BB4EEC09BF1EE10FA03D207
:1060B0009FEDF70BB0EE409BB7EE000BB4EEC09B2C
:1060C000F1EE10FA0BDDB7EE000BB0EE409B06E0F0
:1060D000EC4890ED8C0B9FEDF01B20EE019BB4EE95
:1060E000C89BF1EE10FA01DDB0EE489BE54880ED6B
:1060F000269BEB48007840F00100E9490870002336
:106100004FF480621946012052F038FE1CE00A204C
:106110007CF026FEE3484078042807D1E048007868
:1061200000F0010010B1E048806968B9DF480088DC
:1061300048F20101084038B9DB48808C20B90222BE
:106140000021084654F065FCD848008800F00100A2
:106150000028DCD032210A20FDF70AFED2488069EF
:1061600008B90020A6E5D248008800F00300012805
:1061700002D164207CF0F4FDCA484078042801D0A4
:10618000002097E5C648007800F0010018B11520FE
:10619000C849087061E14FF48062012100202EF0AF
:1061A0008EFEB64A03C2002C1DDDB4484068284468
:1061B000B2494860B34890ED8C1BBF4890ED002B6E
:1061C00021EE021B9FEDBD2B21EE021BB0EE410B19
:1061D00051EC100B7EF0E4FDA84B0CCB801859411C
:1061E000A64A03C206E0002C04DAA4484068401B1B
:1061F000A2494860A24890F8500000F00400A0B105
:10620000A04890ED8C1BAC4890ED002B21EE021BBA
:106210009FEDAC2B21EE021BB0EE410B51EC100BAD
:106220007EF0BEFD074688464EE0A848D0F820B074
:10623000D0F830A09248B0F93000ABEB000B90489A
:10624000B0F93200AAEB000A8D49B1F9401001FB08
:106250000AF0C11700EB51514FEAE12ABBF5004F9C
:1062600002DB47F6FF7B04E01BF5004F01DCDFF8A3
:1062700060B2BAF5004F02DB47F6FF7A04E01AF588
:10628000004F01DCDFF848A20FFA8AF10FFA8BF019
:10629000FDF75FFD00EE100AB8EEC00B864890EDEA
:1062A000001B784890ED8C2B21EE021B20EE010B99
:1062B0009FED881B20EE010BB0EE40BB51EC1B0B99
:1062C0007EF06EFD074688466E4890F8520200F058
:1062D000010048B16948D0E90010C91940EB080035
:1062E000664AC2E9001008E06448D0E90010C91B02
:1062F00060EB0800614AC2E90010624890ED520A62
:10630000B7EEC00A80ED260B00234FF480621946D9
:10631000012052F033FD32210A20FDF729FD08B992
:106320000020C7E46048806908B90020C2E45D48E5
:106330004078042801D00020BCE4684890ED140B9C
:10634000B5EEC00BF1EE10FA38D04E4890ED520A7F
:10635000B7EEC00A80ED260B604890ED141B56483E
:1063600090ED002B21EE021B9FED542B21EE021B22
:10637000B0EE410B51EC100B7EF012FD4A4BD3E90D
:106380000E23801859413D4A03C200234FF4806216
:106390001946012052F0F2FC32210A20FDF7E8FCF8
:1063A00008B9002086E44048806908B9002081E4EB
:1063B0003C484078042801D000207BE4304890F825
:1063C000500000F0040058B12E4890ED8C0BB1EE57
:1063D000001B80EE012BB7EEC20B80EDB60A19E070
:1063E000284890ED8C0B9FED3E2B80EE021B90ED2C
:1063F000B60AB7EEC00AB4EEC01BF1EE10FA09D22D
:1064000090ED8C0B9FED361B80EE012BB7EEC20B8F
:1064100080EDB60A0520009000BF14207CF0A0FC9F
:106420002348008800F00300012802D164207CF09A
:1064300097FC0098411EC9B200910028EDDC2A4863
:10644000007800F0010038B10D4890F84A0000F0E3
:10645000010008B90120029000BF1148007820F027
:1064600001010F4801700120FDF7C1FC029820B125
:106470000D49D1E90E21104638E055E0E008002032
:106480008803002030060524000000000088B34087
:1064900000000040E17A943F00000000006AA8403C
:1064A0004B0500200006002020070020F0050020FA
:1064B00050050020A69B0424580100240000000081
:1064C0000000F041000000000000D04138690424C1
:1064D0000180FFFF000000000000F040300A0524AA
:1064E0000000000000004040B40500207EF0C2FA29
:1064F00041EC100BFE4890ED001B1FED102B81EEC0
:10650000023B20EE030BFB4880ED000B90ED000BEF
:10651000B1EE400BF84880ED000BF84800781E28DB
:1065200002D10020F5490870F54890ED000BF548C0
:1065300080ED260BF4484078042801D00020B8E410
:106540000298B6E470B52DED048BEF48407804282E
:1065500003D00020BDEC048B70BDEA4890F85002D7
:1065600000F0010020B91F20E44908700020F1E785
:10657000E44890F85402012804D02020DF49087034
:106580000020E7E7DF4890F8D001032804D121205C
:10659000DA4908700020DDE7DC4890F8500000F090
:1065A000060020B92220D54908700020D2E7D7483C
:1065B00090F84B0000F0010020B92320CF4908706B
:1065C0000020C7E7D14890F84A0000F0010020B150
:1065D0002420CA4908700020BCE70120CC4908806B
:1065E0009FEDCC0BCD4880ED000B0020CC490880FE
:1065F0009FEDC80BCB4880ED000B0020FDF7F7FBAB
:1066000008B90020A6E7C849D1E90E01C74A03C26C
:106610000024C7480078822802D0C648007808B114
:10662000012408E0C2480078832802D0C14880785D
:1066300008B14FF0FF34C0480078C04909780840DD
:1066400000F0010000287DD100E000BFBC4890F9B7
:1066500000000028F9DA0020B94908702EF06CF922
:1066600040B1AA4890F84A0040F00100A74981F8DB
:106670004A0007E0A54890F84A0020F00100A3492D
:1066800081F84A00FF20AE4908709E4890F85002F9
:1066900000F0010000287DD09C4890F84A0000F0EE
:1066A0000100002876D1994890F8500000287ED04B
:1066B000944890F8D001032879D0A248007840B1DE
:1066C0000020A04908708F4991F8A81248007CF07A
:1066D00047FB8E4890F8500000F0070038B1894819
:1066E00090ED8C0BB0EE001B20EE018B06E0854890
:1066F00090EDA00BB3EE041B20EE018B814890EDD2
:10670000040B9FED911B20EE011B90ED0C2B81EEF5
:10671000020BB4EEC80BF1EE10FA0BDD90ED040B9A
:106720009FED891B20EE010B90ED0C1B80EE012BE1
:10673000B0EE428B734890ED040B9FED851B20EE6D
:10674000019B00E054E0B4EEC98BF1EE10FA01D2E7
:10675000B0EE498B804890ED000B20EE080BBDEEAB
:10676000C00B10EE105A0120FDF79CFE08B9002066
:10677000F0E600202CF0DAFF00202DF03DF8002C90
:1067800009DB2846FEF714FA28B90020FDF78AFE37
:106790000020DFE60BE0002C08DC6842FEF708FA78
:1067A00020B90020FDF77EFE0020D3E60BE0624812
:1067B000007820F00100604908700020674A1060EE
:1067C00050602DF019F85C48007800F0010060B1CD
:1067D0004FF0FF3100202EF0C4FC534AD2E90E32B4
:1067E000181A62EB01025D4905C10020FDF75AFE4F
:1067F0005148007800F0010020B90B203F49087093
:106800000020A7E6FEF7D9FAFDF756FD2046FFF770
:106810003CFA06465248007820F0010050490870C2
:10682000FDF70FFE0EB9002094E6FEF7C6FAFDF75D
:1068300085FE4148007800F0010058B13F480078DB
:1068400040F001003D4908702E4890F8A4023D49EF
:10685000087008E03948007820F0010037490870D6
:106860000020384908700120FDF7C1FA08B900205E
:1068700070E6FEF7E9FC6DE670B52DED088B224859
:106880004078042803D00020BDEC088B70BD0120A7
:106890001F4908809FED1F0B204880ED000B002052
:1068A0001F4908809FED1B0B1E4880ED000B002048
:1068B000FDF79DFA08B90020E6E71B49D1E90E0172
:1068C0001A4A03C20F4890ED560AB7EEC0AAB7EEB7
:1068D000000BB4EEC0ABF1EE10FA03DDB7EE000B27
:1068E000B0EE40AB074880ED26AB1E483CE0000010
:1068F00078010024609B0424D8000024A69B042473
:10690000809A042430060524000600208803002015
:10691000F00500200000000000000000200200241C
:10692000800200244002002420070020809B0424D1
:10693000A29B0424B8020024B40500207034002473
:10694000A19B04244C050020FCA9F1D24D62603FBC
:106950007B14AE47E17A743F58010024B80500204B
:106960004B050020189B042490ED000AB7EEC00AE6
:10697000FE4890ED001B20EE010BBDEEC00B10EEAB
:10698000100AFB49C96B0844FA49486000234FF4D8
:1069900080621946012052F0F1F90A210846FDF7FC
:1069A000E7F908B900206FE70120FDF720FA08B9E0
:1069B000002069E70025F04890F8D00180B1EE484A
:1069C00090F8D00103280BD0EB4890F8500200F06B
:1069D000010028B1E948007800F0010000B9012564
:1069E000E54890F8D00130B1E548007800F00100AA
:1069F00008B9002D7CD000E000BFE24890F900000B
:106A00000028F9DA0020DF4908702DF095FF40B129
:106A1000DD4890F84A0040F00100DB4981F84A0067
:106A200007E0D94890F84A0020F00100D64981F8E3
:106A30004A00FF20D3490870CF4890F8500200F078
:106A40000100002872D0D04890F84A0000F0010000
:106A500000286BD1CC4890F850000028F2D0C648EE
:106A600090F8D001032861D0C848007840B10020D8
:106A7000C6490870C04991F8A81248007CF070F926
:106A8000C14890F8500000F0070038B1BA4890EDC6
:106A90008C0BB0EE001B20EE018B06E0B64890EDAB
:106AA000A00BB3EE041B20EE018BB34890ED040B5A
:106AB0001FED5B1B20EE011B90ED0C2B81EE020BFA
:106AC000B4EEC80BF1EE10FA0BDD90ED040B1FEDE8
:106AD000621B20EE010B90ED0C1B80EE012BB0EE43
:106AE000428BAB48007848B1A34890ED040B00E01E
:106AF00074E01FED691B20EE019B01E09FEDA59B5B
:106B0000B4EEC98BF1EE10FA01D2B0EE498B974882
:106B100090ED000B20EE080BBDEEC00B10EE104AFE
:106B20000120FDF7BFFC10B90020ADE634E00020E5
:106B30002CF0FCFD00202CF05FFE2046FEF738F81C
:106B400020B90020FDF7AEFC00209DE66042FEF774
:106B50002FF820B90020FDF7A5FC002094E6884816
:106B6000007800F00100B0B1834890ED260BB0EE44
:106B700040BBFDF7E0FD50B97F4880ED26BB00200B
:106B8000FDF790FC07208549087000207CE67A48D4
:106B900080ED26BB00BF0CE07848007820F00100B3
:106BA0007649087000217E4A1160516000202CF067
:106BB00023FE7248007800F0010060B14FF0FF3111
:106BC00000202EF0CEFA6A4AD2E90E32181A62EB91
:106BD0000102734905C10020FDF764FCFEF7B8FC13
:106BE00008B9002050E66F48007880BB624890F8F2
:106BF0005402022804D16148007800F0010020B955
:106C00005D4890F85402032822D10120FEF772FB60
:106C1000002801DA002037E65848007800F001002B
:106C2000A8B1554890F85402022811D1574800786D
:106C300068B90020FEF75EFB002801DA002023E699
:106C40000020FEF757FB002802DA00201CE6FFE7D1
:106C5000494890F85402012829D1474890F8500239
:106C600000F0010018B3484890F8500000F0070009
:106C7000E8B14248007800F0010020B90B204749F4
:106C80000870002000E6FEF798F8FDF715FB0020DD
:106C9000FEF7FBFF04464448007820F0010042491B
:106CA0000870FDF7CEFB0CB90020EDE500BFFEF744
:106CB00084F8FDF743FCADB13048007800F00100E6
:106CC00080B12D4890F8D00101280BD1811E002001
:106CD0002EF047FA264AD2E90E32181A62EB010268
:106CE0002F4905C12548007800F0010058B12F4810
:106CF000007840F001002D4908701F4890F8A40268
:106D00002249087008E02948007820F0010027494E
:106D1000087000201D4908700120FDF768F808B9C7
:106D20000020B1E5FEF790FAAEE570B52DED028BCF
:106D3000044615485030005D00F00100E0B301202A
:106D4000A0400E4909780840B0B30F4890F84A00B7
:106D50000121A140084078BB154800780121A140DD
:106D6000084048B3134890F9000026E05801002479
:106D700020070020E008002030060524B40500208C
:106D800088420030A19B0424880300204C05002089
:106D9000A29B04249A9999999999A93FA69B0424A6
:106DA000B8050020844200304B05002070340024D8
:106DB000A40B0020A09B042407E0A04205D1FE48BC
:106DC000005D10B9FD48005D18B10120BDEC028BDB
:106DD00070BDFA48603000EBC40090ED000BB0EEDF
:106DE000001B20EE018B1FED150BB4EEC08BF1EEF6
:106DF00010FA05D2B0EE000B28EE000BB0EE408B7F
:106E00001FED1C0BB4EEC08BF1EE10FA03D21FED98
:106E10001F0BB0EE408BEA4800EBC40090ED000B76
:106E200020EE080BBDEEC00B10EE105AE54830F80E
:106E30002400E5490880E34800EB8400408848804E
:106E4000E048103030F81400E0490880002600BF08
:106E50006D42012229462046FDF700FE08B1701C54
:106E600006B2DB4800EB44004078042801D0002043
:106E7000ACE7D44830F82400D3490880D14800EB6F
:106E8000840040884880CF48103030F81400CF4943
:106E90000880002DDCDB002E34DD0120C6490855BA
:106EA000C84931F92410C84A1288032313FB021081
:106EB000C11700EB917189100AB2C24921F8242050
:106EC00001EB8401B1F90210BF4A528813FB021092
:106ED000C11700EB917189100AB2BA4901EB840124
:106EE0004A80B849103131F91410B84A128803FBAE
:106EF0000210C11700EB917189100AB2B14910312B
:106F000021F81420012061E710B5B1484078042829
:106F100001D0002010BD0120AE490880AE4890EDA0
:106F2000620B90ED5E1AB7EEC11A80EE012BB0EE47
:106F3000000BB4EEC02BF1EE10FA06DD90ED5A0A0C
:106F4000B7EEC00A80ED260B06E0A34890ED5E0A7E
:106F5000B7EEC00A80ED260B9F4890ED260B90ED12
:106F6000321BB4EEC10BF1EE10FA03DD90ED320BE3
:106F700080ED260B984890ED621B984890ED000A32
:106F8000B7EEC00A31EE001B8D4890ED002B9448FF
:106F900090ED0F0AB8EEC00B01EE420BBDEEC00B38
:106FA000904880ED010A00234FF4806219460120C9
:106FB00051F0E4FE64210A20FCF7DAFE08B9002053
:106FC000A8E70120FDF76EFA28B10020FFF7ADFE1B
:106FD0000020FDF767FA0021834A116051607E4866
:106FE00090F8C80108BB7E48D0E90E107F4AC2E97C
:106FF00000107B48D0E90E107D4AC2E900107848A5
:10700000D0E90E107B4AC2E900107B48007800F0FE
:10701000010050B17648D0E90030784A06CA591AC2
:1070200060EB0200704AC2E900100120FCF7DFFEAD
:1070300001206FE700BF00207CF03EFF64484078ED
:1070400000F0080010B104206149487000206C492C
:1070500008706C4908706C4A1060506000216B4ADF
:10706000116051606A49087045245D48806908B91B
:1070700054249DE15648407800F0020008B14524B0
:1070800096E15348007800F0010000287ED0FCF71C
:10709000B1FF6048007800F0010050B14948303835
:1070A00090F8500000F0060018B1FFF74BFA0546C3
:1070B0000BE0494890F8E401012803DCFFF7DCFB12
:1070C000054602E0FEF747FB05460020FDF7EAF91A
:1070D0005148007820F001004F4908704F4800786F
:1070E00020F001004D4908704A48007820F0010066
:1070F00048490870FDF7ACF832243648008800F0A3
:10710000010080B901203649888404E0601EC4B2C1
:107110000A207BF025FE2F48008800F0010008B906
:10712000002CF3D1002595B33D48007800F0010014
:1071300068B33C4890ED000AB5EEC00AF1EE10FAD3
:107140002AD01F4890ED001B364890ED000AB7EE9C
:10715000C00A21EE000BBDEEC00B10EE100A204954
:10716000C96B08441F49486000234FF480621946E8
:10717000012051F003FE64210A20FCF7F9FD00B95B
:1071800000251748C06B1749496801E0CCE003E0CF
:10719000884271D000256FE065B12148007800F089
:1071A000100038B11F4890ED080AB5EEC00AF1EEA4
:1071B00010FA39E060E00000C69A042400080524B3
:1071C00058010024B8030020C09A0424C49A04245F
:1071D00000060020F005002030060524189B04243A
:1071E00020070020E0080020483500248006002009
:1071F000C006002000070020A40B0020A0060020ED
:10720000CE9A0424D29A0424D89A0424F89A042406
:10721000CA9A0424BA420030C80C00204B05002052
:1072200000430030C042003026D0784890ED001B6B
:10723000774890ED080AB7EEC00A21EE000BBDEECC
:10724000C00B10EE100A7349C96B084472494860BC
:1072500000234FF480621946012051F08FFD642114
:107260000A20FCF785FD00B900256A48C06B6A4911
:107270004968884200D000256848007820F0110055
:10728000664908708DB16648407804280DD165487C
:10729000007810B90120634908706348007840F015
:1072A000010061490870412418E05A48806918B902
:1072B00003205C4908700DE059484078022803D14A
:1072C00005205849087005E05648007810B902209A
:1072D000544908704524022051494870534890F899
:1072E000500000F0070028B15148007820F001005C
:1072F0004F49087044F0E2FD02207BF031FD4D481B
:10730000006810B10A207BF02BFD002053F036FC02
:1073100018B90021084646F005FC4748007810B12E
:107320000E204649888043E03D48007800F0020086
:10733000E0B3FCF75FFEFFF7E7FD0546FCF788FFCB
:107340005DB137484078042807D13748407840F08D
:10735000010035494870442419E032243848008837
:1073600000F0010078B901202A49888404E0601EF9
:10737000C4B20A207BF0F4FC3148008800F0010020
:1073800008B9002CF3D1452402202549487000207B
:1073900053F0F4FB18B90021084646F0C3FB264819
:1073A000807810B10E202549888001E0FFE7002495
:1073B00054B31848806920B9412C02D0442C00D025
:1073C00054240020FDF76EF81E48007850B911488B
:1073D000808C38B11A48008800F0010010B10020FC
:1073E0000C4988840020184908701848047000BFB0
:1073F00000BF00BFBFF34F8FBFF36F8F00BF00BF51
:1074000000BF01200649487015E60000580100241D
:10741000C042003020070020E00800200043003078
:1074200000060020A69B0424A40B00208803002053
:10743000B5050020C00D0020B8020024C8000024BB
:10744000F0050020AF0D002084420030AC9B0424E6
:107450002DE9F04104460D4627462E46002F00DC5C
:107460000127002E00DC012619E0F948C078042825
:1074700003D1F848D0F8880070B9F748408848F23E
:107480000101084040B9F348B0F8940020B9022245
:107490000121084653F0BDFA38467BF061FCEE4806
:1074A000408800F001000028DFD0EA48D0F88800CA
:1074B00028B90420E94948700020BDE8F081304631
:1074C0007BF04EFCE248C078042801D00020F4E7AD
:1074D0000120F2E770B5054632207BF041FCE04820
:1074E000007800F0020028B1DE48407810B9322060
:1074F0007BF036FCDA48007800F0020010B1D94881
:10750000407808B9012070BDD748408800F00100DC
:1075100008B90120F7E7052405B1142413E0CC488D
:10752000C078042801D00020EDE70021CF48416455
:10753000016432207BF014FCCC48006C08B90120B7
:10754000E1E7601EC4B2002CE9DC0120DBE72DE995
:10755000F0412DED0A8B04460D4616461F46C448E1
:1075600090ED280BB0EE409B90ED570AB7EEC00AA5
:10757000B0EE408B90ED530AB7EEC00AB0EE40CBB0
:1075800090ED340BB4EEC80BF1EE10FA03D290ED8F
:10759000340BB0EE408BB64890ED340BB4EECC0B10
:1075A000F1EE10FA03D290ED340BB0EE40CB66B1A1
:1075B000B7EE000BB4EEC08BF1EE10FA03DDB7EEC0
:1075C000000BB0EE408BB0EE48CBAA4890ED020B1A
:1075D00020EE080BB7EEC0ABB5EEC0AAF1EE10FA84
:1075E00003D19FEDA50AB0EE40AA9A49D1F8AC109C
:1075F000681A002801DB014600E0414200EE101A43
:10760000F8EEC0AA8AEE8ABAB0EE000AB4EEC0BAAA
:10761000F1EE10FA03DD964880ED28CB02E09448A5
:1076200080ED288BB7B39548C0E90245944890EDAA
:10763000010AF2EE040A80EE201AB7EEC11A8D4854
:1076400090ED022B8D4890ED030AB8EEC00B01EED1
:10765000420BBDEEC00B80ED030A00234FF48062A5
:107660001946022051F08AFB0A210846FFF7F0FE76
:1076700038B97F4880ED289B0020BDEC0A8BBDE81F
:10768000F0810020FFF726FF28B9794880ED289B7C
:107690000020F2E702E0764880ED288B7748C0E9C9
:1076A000024500234FF480621946022051F066FB28
:1076B0000A210846FFF7CCFE20B96D4880ED289BD3
:1076C0000020DAE70120FFF705FF20B9684880EDC8
:1076D000289B0020D1E7664880ED289B0120CCE75D
:1076E0001CB50020009001905E494978F1B35C49D7
:1076F000097801F00201C9B3624991F84A1001F01A
:10770000020199BB6049897801F0010171B35949BF
:1077100091ED020B9FED5D1B20EE010BB0EE002BF7
:1077200080EE021B5B49C868002801DB014600E0CF
:10773000414200EE101AB8EEC00BB4EEC01BF1EEE1
:1077400010FA18D2012108462DF00BFDCDE90001F9
:107750004048D0F8AC000199411A3E48D0F8B40036
:1077600001443C48C0F8B410703000E003E0DDE9AB
:107770000021C0E90E213E4890F8250148B93C4857
:1077800090F83501032804D04348007800F0020047
:1077900060B19FED420A3A4880ED010A344890F802
:1077A000250140F080003E49487007E09FED320A15
:1077B000334880ED010A0020394948702C4890ED8B
:1077C000280B384880ED020B294890F81103364900
:1077D00048702748B0F8120134494880244890F88E
:1077E000190133494870224890EDB30A314880EDC1
:1077F000010A1F4890F825012F4948701C4890F84D
:10780000ED042E4948700021194880F8251180F8B0
:10781000ED1480F811136421A0F81211002180F8F2
:10782000191190ED060BB2EE081BB4EEC10BF1EE90
:1078300010FA45DD90EDB30AF7EE000AB4EEE00A67
:10784000F1EE10FA3CD2B7EE000A80EDB30A45E043
:107850000006002020070020F0050020A69B04243D
:10786000B40500204C05002050050020D009002060
:107870003006052458010024CDCCCC3DE008002082
:10788000189B042488030020B4020024000000A0F8
:107890009999B93F58050020BA420030B4A29139F5
:1078A000A29B0424809A0424A09A0424A89A042465
:1078B000A49A0424B09A0424789A04247C9A042478
:1078C000FE4890EDB30A5FED140AB4EEE00AF1EE63
:1078D00010FA03D21FED180A80EDB30AF848408869
:1078E000642802DA0A207BF03BFAF648C0780828C0
:1078F00022D10421F348C1700198E8B1F2484078E0
:1079000000F0010070B140F2E241F048A0F896109A
:1079100002E001207BF024FAEC48B0F9960001283F
:10792000F7DC09E0E848407830B1E449B1F8B21238
:1079300001F10A007BF014FA0120E54948701CBDF2
:1079400010B5E348407800B910BD01200FF0BCF934
:10795000E0484178D94880F82511DF484178D74878
:1079600080F8ED14DD4890ED020BD44880ED280B33
:10797000DB484178D14880F81113D148408801B2E2
:10798000CE48A0F81211D7484178CC4880F8191198
:10799000D54890ED010AC94880EDB30AD34890F864
:1079A000480020F02000D14981F8480000BFCBE713
:1079B000C24890EDB70ACE4880ED010AC24840782F
:1079C000CC494870BD4890F8BD02CB494870BB48CF
:1079D00090F8C102C9494870B848B0F8B202C84925
:1079E0004880B648B0F8B2023F2803DA3F21B348D6
:1079F000A0F8B2124FF0FF30C2494860AF48D0F84B
:107A0000AC02B0F51C7F08D8AC48D0F8AC02486096
:107A100040F27120A949C1F8AC02B44890F8510075
:107A200000F0400058B1A54890EDA20BB1EE001B4C
:107A300020EE010BB7EEC00B80EDB70A10E0AB48AB
:107A400090F8510000F0040050B19C4890ED8E0B6E
:107A5000B0EE001B80EE012BB7EEC20B80EDB70A33
:107A6000964890EDB70ADFEDA80AB4EEE00AF1EE11
:107A700010FA03D29FEDA40A80EDB70A9C4890ED5E
:107A8000010AB2EE041AC0EE010A8C4890EDB70A62
:107A9000F4EEC00AF1EE10FA0ADD954890ED010A05
:107AA000F2EE040A80EE201A844880EDB71A17E03F
:107AB000824890EDB70A8E48D0ED010AB2EE041A62
:107AC00060EE810AB4EEE00AF1EE10FA08DD90ED06
:107AD000010AF2EE040A20EE200A784880EDB70A87
:107AE000764890F8BD02022803DA0221734880F834
:107AF000BD12724890F8C102022803DA02216F48D1
:107B000080F8C1126D4890F8A502022811DA6B487E
:107B100090F8BD02142803DD1421684880F8BD12D6
:107B2000664890F8C102142803DD1421634880F8E8
:107B3000C1120220644948707047724840680021B1
:107B4000494071EA000004D06E4840685B49C1F8C2
:107B5000AC024FF0FF306B49486069484188574894
:107B6000A0F8B212624890ED010A544880EDB70ABD
:107B70006048407854494870504890F8A50202285F
:107B80000CDA5C48407848705B4841784B4880F894
:107B9000BD125A484178494880F8C112704770B503
:107BA000054655B959480078012804D1FF205749A6
:107BB0000870012070BD0020FCE74FF4FA766324C2
:107BC00000BF4048C078042801D00020F2E7301EF2
:107BD000A6F101010EB204DC0A204D4948700020D4
:107BE000E8E74A4890F90000002803DA01204749F5
:107BF00008701BE0454890F90000A04213D04348AC
:107C000090F90040002C0CDB4248807DA04208DD4A
:107C10000120A04040490978084010B140F26B367D
:107C200001E04FF4FA7628207BF09AF83748007884
:107C30000128C6D100BFBDE770B5264840780028AE
:107C400000DD70BD21487030D0E90E451B4890F82A
:107C5000E50102282BDB314890ED020BB5EEC00B9D
:107C6000F1EE10FA08D82E48D0F8840000F48020F5
:107C700010B900242B4D1AE0284890ED021B2A4829
:107C800090ED022B21EE021B9FED282B21EE021B13
:107C9000B0EE410B51EC100B7DF082F8241A65EB2D
:107CA00001052448C0E902450120234948700348E2
:107CB00090F8C90100287DD1204841E03006052414
:107CC000A89A0424000600204C050020200700206C
:107CD000CA9A0424789A04247C9A0424809A04245E
:107CE000A09A0424A49A0424B09A042488030020AF
:107CF000289B0424389B04243C9B0424409B04249C
:107D0000449B04244C9B042417B7D138A09B042423
:107D1000A69B04244000002488420030800A0524E9
:107D20009034002400000C81580100240000000061
:107D30000000F041D89A0424CE9A04246006002062
:107D4000C0E90245FE48C0E90245FE48C0E90245D7
:107D5000FD4890F8EE0100F0020060B3FA4890F898
:107D6000D10101282FD0F84890F8E50102282ADA3D
:107D7000F648C068002826DDF548D0E90210F34A2D
:107D8000D2E90232C9185041F24AC2E90210104643
:107D9000D0E90210F04AC2E90210EE48D0E9021020
:107DA000EE4AC2E90210EB48D0E90210EC4AC2E9FF
:107DB000021001E045E006E0EA48407840F00200A9
:107DC000E84948703DE0E84890ED010AB5EEC00A88
:107DD000F1EE10FA35DD90ED011AB7EEC11AE34865
:107DE00090ED022B31EE021BE14890ED022B21EECB
:107DF000021B1FED322B21EE021BB0EE410B51ECAA
:107E0000100B7CF0CDFFD34AC2E902010120D94911
:107E100048701046D0E90210CF4AC2E90210CD489E
:107E2000D0E90210CD4AC2E90210CA48D0E90210D6
:107E3000CB4AC2E90210CB48407840F00200C94961
:107E4000487000BFFDE62DE9F0412DED028BCA48D8
:107E5000407850B10020C8494870BB4991F8A81239
:107E6000490001F164007AF07BFFC44890ED020BF9
:107E70009FEDC31B81EE002BB34880ED282BC24839
:107E8000D0E90E45C148C0E90245AF49B1F85210EA
:107E90000803C11700EBD1614A11BC49C9680A4403
:107EA000BA49CA6000234FF480621946022050F09C
:107EB00065FFFA210A20FFF7CBFA20B90020BDECBC
:107EC000028BBDE8F081B0487038D0F8AC10AF48F4
:107ED000C068814201D00020F1E7AB49D1E90E0131
:107EE000AA4AC2E902011046C1689748B0F8520098
:107EF0004FF4805202FB0011A448C1609FEDA48B97
:107F00004FF0000815E001207AF02AFF4FF0FF3211
:107F1000012108462CF0D3FF06467CF0ABFD41EC76
:107F2000100B38EE400BB0EE408B08F1010000F072
:107F3000FF08B8F1080FE6DB00234FF48062194612
:107F4000022050F01BFFFA210A20FFF781FA08B93E
:107F50000020B4E78C487038D0F8AC108B48C0686B
:107F6000814201D00020AAE74FF0000815E001206F
:107F70007AF0F6FE4FF0FF32012108462CF09FFF09
:107F800006467CF077FD41EC100B30EE080BB0EEAE
:107F9000408B08F1010000F0FF08B8F1080FE6DBA4
:107FA0007949D1E90E01794AC2E902016649B1F87D
:107FB00052100803C11700EBD1614A117349C96817
:107FC0000A447249CA6000234FF4806219460220B5
:107FD00050F0D4FE0A210846FFF73AFA08B900200B
:107FE0006DE769487038D0F8AC106848C0688142C5
:107FF00001D0002063E76448D0E90E10634AC2E96B
:1080000002105149B1F852100803C11700EBD161B9
:108010004A115E49C9688A1A5C49CA6000234FF454
:1080200080621946022050F0A9FEFA210A20FFF7CB
:108030000FFA08B9002042E753487038D0F8AC1066
:108040005248C068814201D0002038E74E48D0E94C
:108050000E104E4AC2E902101046C1683A48B0F804
:1080600052004FF4805202FB10114848C1604FF09B
:10807000000815E001207AF073FE4FF0FF32012175
:1080800008462CF01CFF06467CF0F4FC41EC100B7B
:1080900030EE080BB0EE408B08F1010000F0FF0855
:1080A000B8F1080FE6DB00234FF480621946022086
:1080B00050F064FEFA210A20FFF7CAF908B900203F
:1080C000FDE631487038D0F8AC103048C0688142C5
:1080D00001D00020F3E64FF0000815E001207AF00F
:1080E0003FFE4FF0FF32012108462CF0E8FE064625
:1080F0007CF0C0FC41EC100B38EE400BB0EE408B36
:1081000008F1010000F0FF08B8F1080FE6DB224893
:1081100090ED021B9FED212B81EE020B20EE080B50
:10812000B0EE408B1948C0E9024500234FF480624D
:108130001946022050F022FE0A21084632E00000D3
:10814000A0060020E0060020300605244835002463
:1081500060060020F89A042480060020C006002053
:1081600000070020A40B0020243500244002002436
:1081700058010024D29A04244C05002098010024C0
:10818000000000A09999C93F90070020E008002056
:108190000000000000000000780100240000000042
:1081A00000003042FFF754F908B9002087E6FE4886
:1081B000D0F8AC10FD48C068814201D000207EE6B6
:1081C0009FEDFB0BB4EEC08BF1EE10FA10DB9FEDD0
:1081D000FA0BB4EEC08BF1EE10FA09D8F84880ED36
:1081E000068B002101200EF002FF0120FFF772F93B
:1081F000012064E62DE9F0412DED028B04460025B7
:10820000F04890F8510000F0010000B10125ED4860
:1082100090F84A0020F00200EA4981F84A001FED78
:10822000240BB0EE408B4FF0FF32002101202CF0E8
:1082300046FE06467CF01EFC41EC100B38EE400B6F
:10824000B0EE408B01207AF08BFD4FF0FF32002121
:1082500001202CF034FE06467CF00CFC41EC100BA7
:1082600038EE400BB0EE408B2A4621460120FCF749
:10827000F5FBD548C078042804D00020BDEC028B63
:10828000BDE8F08164207AF06BFD4FF0FF320021F1
:1082900001202CF014FE06467CF0ECFB41EC100BA8
:1082A00030EE080BB0EE408B01207AF059FD4FF014
:1082B000FF32002101202CF002FE06467CF0DAFBA2
:1082C00041EC100B30EE080BB0EE408B9FEDBF0B76
:1082D00088EE001BB0EE418BBA4890F84B0000F0DE
:1082E0000200002875D0B74890F84A0000F002005C
:1082F00000286ED1B0EEC81B00EE104AB8EEC00BDD
:10830000B0EE002B20EE020BB0EEC00BB4EEC01BA3
:10831000F1EE10FA5DD8B0EEC81B00EE104AB8EED0
:10832000C00BB6EE002B20EE020BB0EEC00BB4EE8D
:10833000C01BF1EE10FA4CDBA648007800F00200FA
:1083400038BB00EE104AB8EEC00B28EE000BB5EEBD
:10835000C00BF1EE10FA07D2994890F8520280F063
:108360000200974981F85202964890F8510004287B
:1083700010D1934890ED8E0B9FED971BB4EEC10B7F
:10838000F1EE10FA06DD9348007820F002009149E2
:10839000087026E08B4890F8510000F0400080B152
:1083A000874890EDA20B9FED8C1BB4EEC10BF1EE54
:1083B00010FA06DD8748007820F002008549087031
:1083C0000FE08448007840F002008249087008E01D
:1083D000FFE7002C05DD7F48007820F002007D4992
:1083E00008707C48007800F0020010B901202BF0E2
:1083F00003FA012042E770B52DED028B86B0002014
:10840000049005906E4890F8E501022813DB74484B
:1084100090ED021B734890ED022B21EE021B9FEDA5
:10842000722B21EE021BB0EE410B51EC100B7CF0D5
:10843000B7FCCDE904011FEDAA0B6D4880ED020BDE
:10844000604890F84A1063480078884300F00200C2
:10845000E8B35C4890F8510000F03000B8B36548CC
:1084600090ED030AB8EEC00BB0EE408B01207AF01D
:1084700077FC604890ED030AB8EEC00B30EE080BB5
:10848000B0EE408B01207AF06BFC5A4890ED030A65
:10849000B8EEC00B30EE080BB0EE408B01207AF046
:1084A0005FFC544890ED030AB8EEC00B30EE080BA9
:1084B000B0EE408B424890EDA20B20EE080BB1EEDF
:1084C000001B80EE012B4A4880ED022B00BF3C4888
:1084D00090F8D101012822D14748007800F002002D
:1084E000E8B931487030D0E90E50DDE90461AA1BCB
:1084F00060EB010110467CF0BDFA41EC100B3F48E7
:1085000090ED021B20EE010B9FED371B80EE012B3F
:108510003B4880ED022B06B0BDEC028B70BD1FED19
:10852000E40B374880ED020B2A48007800F0020087
:1085300010B132207AF014FC3248447800203149DE
:1085400048702448007800F0020018B114B164208B
:108550007AF006FC1FEDF20B2B4880ED020B2B4846
:10856000006840F001002949086000BF00BF00BF5B
:10857000BFF34F8FBFF36F8F00BF00BF00BF0A482C
:108580007030D0E90E10DDE90423891A60EB030096
:10859000CDE9021004487030D0E91010DDE9023254
:1085A000C9185041004A33E020070020E0080020AD
:1085B0002D431CEBE2361A3F00000000000059403A
:1085C000300605248803002000060020000000007B
:1085D00000000042B40500209A9999999999B93FF1
:1085E000800A052458010024000000000000F0412A
:1085F00060020024D8050020884200307801002461
:10860000400200244C050020D8000024E00C00208B
:108610007032C2E91010A2F17000D0F8C8000399BE
:10862000411AA2F17000C0F8C810FE49DDE904202B
:10863000C1E90E2000BF00BF00BFBFF34F8FBFF3E3
:108640006F8F00BF00BF00BFF748006820F0010037
:10865000F5490860F54890F8A70000F002000028EE
:1086600071D0F24890F89D0000286CD0EF4890F847
:108670009900002867D1ED4A92F93920002A14DBCD
:10868000EA4A92F93930EA4A02EB831292ED060A7D
:10869000B7EEC00AE74A92ED021B20EE010BBDEED9
:1086A000C00BE24A82ED050A02E00023DF4A536173
:1086B000DE4A536A5569DB4A703AD2F8AC20AA1AEE
:1086C00083FB02202CE0DC4A12880192DB4A5268CC
:1086D000111A0A2905DDD94A52680A3AD74B5A605D
:1086E00007E011F10A0F04DAD44A52680A32D34B78
:1086F0005A60002905DDD14A5268521ECF4B5A609C
:1087000006E0002904DACD4A5268521CCB4B5A606D
:1087100000E000BFC84A1288BDF804309A42F8D081
:10872000C64A52688242CED1C04A92F8A120002A9D
:1087300008DDBE4A92F8A120062A03D00123BB4AD5
:1087400082F83D3000BFBE4890F85100A0B30A2027
:108750007AF006FBBA4890F8510000F03000B8B942
:10876000B84890F8520200F0020088B14FF0FF3193
:1087700001202CF0F6FC0022434262EB0100DDE90F
:108780000412591A60EB0200AF4AC2E902100FE06E
:108790004FF0FF3101202CF0E4FC0023424263EB58
:1087A0000100DDE90431D2184841A749C1E902209E
:1087B0000121084617F018FEA448447000BFAAE63D
:1087C0002DE9F041A248007800F0020010B9002025
:1087D000BDE8F0819A4890F8510000F0030008B914
:1087E0000020F5E700250024002613E005207AF09C
:1087F000B7FA0121924880F8F810D0F8DC0005445F
:108800008F48D0F8EC00044400218D4880F8F8101F
:10881000701CC6B2042EE9DB2846E91705EB9171FE
:108820008D102046E11704EB91718C108448B0F94B
:1088300034002D1A8248B0F93600241A8049B1F963
:10884000421001FB04F0C11700EB5151CC12291E5C
:1088500001DB0A4600E04A42782A08DA201E01DBE2
:10886000024600E04242782A01DA0020B0E7B5F57E
:10887000004F02DB47F6FF7503E015F5004F00DC03
:10888000744DB4F5004F02DB47F6FF7403E014F5B6
:10889000004F00DC6F4C21B228B2FBF75AFA0746B2
:1088A00007B90127384693E770B56B4840886B4994
:1088B0004880FFF785FF04466548007800F0020015
:1088C00028B99FED670B684880ED020B0FE05D480B
:1088D00090ED8E1B00EE104AB8EEC00B21EE000B9F
:1088E0009FED621B80EE012B5F4880ED022B6148FB
:1088F000407808B9012070BD00205E49487050489A
:1089000090F8510000F0030008B90020F3E70025BB
:108910004C4890F8280100F0020000B101255648AB
:1089200020F815404C48408820B90121534820F8D0
:10893000151005E04948408801B2504820F815104C
:1089400034B9404890F85502022801D10020D2E7FE
:108950000120D0E72DE9F04781460025394890F8FD
:10896000280100F0020000B10125364890F85502B8
:10897000022807D0334890F85502032802D000207F
:10898000BDE8F0873B48407808B10020F8E72D4863
:1089900090F8550202281AD1374830F81500A0B1D6
:1089A0002B48007800F0020078B1264890ED8E0B3D
:1089B0009FED331BB4EEC10BF1EE10FA05D3204846
:1089C00090F8510000F0030008B90020D8E71D48D6
:1089D00090F85502032805D1284830F8150008B949
:1089E0000020CDE72848C078042802D04FF0FF309F
:1089F000C6E70020FEF76EFD10B94FF0FF30BFE76D
:108A000032207AF0ADF9FFF7DBFE80460D4890F892
:108A1000550202287DD1B8F1000F7AD0164830F8FF
:108A2000150033E090070020E00C0020C433002440
:108A3000E855003058010024AE0B00202C06002021
:108A40008803002030060524B80500204C050020CE
:108A5000B40500200180FFFFA8020024800200244A
:108A600000000000000000002002002400000000C0
:108A70000000F040844200308C0200249C0200245C
:108A80007B14AE47E17A943F0006002008B900202D
:108A900076E7FC4830F91500A8EB0004B4F5004F68
:108AA00002DBA4F5803404E014F5004F01DC04F58A
:108AB0008034F54890F82801F34991F85212484063
:108AC00000F0020000B16442EF4890F8280100F085
:108AD000020000B9644214F57A5F01DA00204FE722
:108AE000B4F57A5F01DD00204AE70120E7494880BC
:108AF000002C62D0E44890ED8E2B01EE104AB8EEC7
:108B0000C11B22EE011BE24890ED022B21EE021B5D
:108B100000E019E01FED2B2B21EE021BB0EE410B04
:108B200051EC100B7CF03CF9DA4BD3E90E2386189C
:108B300041EB03074B46012230463946FEF707FD5D
:108B4000C0BB4FF0FF301BE7CF4890F85502032819
:108B500031D1D14830F8150008B9002010E7CF48CE
:108B60004188CD4830F915000C1AB4F5005F02DBDE
:108B7000A4F5804404E014F5005F01DC04F58044B2
:108B8000C14890F8280100F0020000B964420120B9
:108B9000BE49488074B1BF487038D0F8AC0007199E
:108BA00000264B46012230463946FEF7D0FC08B974
:108BB000701EE5E601E00020E2E60120E0E670B587
:108BC0002DED028B82B00024B54890ED0A0AB8EE74
:108BD000C00B20EE000BB0EE408B90ED0B0AB8EE10
:108BE000C01B90ED0B0AB8EEC02BB0EE480B01EEA7
:108BF000020BB0EE408BAB48007800F0200018B9B3
:108C00006120A94908701AE0A848007800F0020025
:108C100090B19FEDA70BB4EEC08BF1EE10FA0BDB19
:108C2000A548407818B162209F49087007E063208A
:108C30009D490870012402E064209B49087098480F
:108C4000816A9E4841629648C16A9C484163944843
:108C5000416A9A4841610021416400BF32207AF0A4
:108C60007FF8894890F8E501022803DB0020009096
:108C700001903FE0844890ED6C1B914890ED010A13
:108C8000B1EE400AB7EEC00AB4EEC01BF1EE10FA26
:108C900015D290ED011AB7EEC11A7D4890ED022B66
:108CA00021EE021B9FED872B21EE021BB0EE410B44
:108CB00051EC100B7CF074F8CDE900011AE0724819
:108CC00090ED6C2B7E4890ED011AB7EEC11A32EE92
:108CD000011B6F4890ED022B21EE021B9FED792BBB
:108CE00021EE021BB0EE410B51EC100B7CF058F85A
:108CF000CDE900016C480078612809D17349DDE9AC
:108D00000030D1E902219A184841CDE9002033E032
:108D100065480078642809D1614ADDE90010D2E98C
:108D20000632C9185041CDE9001025E04FF48062A9
:108D3000012108462CF0C3F8DDE9002380185941D1
:108D4000CDE9000158480078632815D14FF0FF3273
:108D5000012108462CF0B3F8DDE90032181A62EB65
:108D60000102CDE900024B49DDE90030D1E90E21D5
:108D70009A184841CDE900204948006A002804DDDE
:108D800047480199006A081A0190002000900123C9
:108D90000022DDE900512846FEF7D9FB20B900206A
:108DA00002B0BDEC028B70BD0120FEF793FB08B949
:108DB0000020F5E7201EA4F101014CB23FF74EAFB1
:108DC0000120EDE72DE9F0412DED048B4048C078FE
:108DD000042804D00020BDEC048BBDE8F081012004
:108DE0002A4948801FEDE20B3A4880ED020B002033
:108DF000394948801FEDE60B384880ED020B002012
:108E0000FEF768FB08B90020E5E72248D0E90E101C
:108E10002E4AC2E9021000251B4890F8D10180B10A
:108E2000194890F8D10103280BD0174890F8500248
:108E300000F0020028B11D48007800F0020000B9DF
:108E40000125114890F8D10130B12548007800F093
:108E5000020008B9002D7DD000E000BF214890F944
:108E600000000028F9DA01201E4908702BF064FD8B
:108E7000E0B31D4890F84A0040F002001A4981F81A
:108E80004A003CE08C02002430060524F005002056
:108E900058010024900700209C020024A80200240E
:108EA000680C0020C80C002001000020B405002040
:108EB0000000008030E663414C050020386904243E
:108EC000189B0424000000000000F041809B042453
:108ED000000600202002002480020024400200241A
:108EE00088420030A19B042488030020FFE7F64855
:108EF00090F84A0020F00200F34981F84A00FF2070
:108F0000F2490870F24890F8500200F00200002880
:108F100072D0ED4890F84A0000F0020000286BD1B2
:108F2000E94890F85100002866D0E94890F8D1014E
:108F300003287FD0E748407840B10020E5494870D9
:108F4000E34991F8A812480079F00AFFDE4890F84A
:108F5000510000E07EE000F0070038B1DC4890ED01
:108F60008E0BB0EE001B20EE018B06E0D84890ED92
:108F7000A20BB3EE041B20EE018B9FEDD70BB4EEDA
:108F8000C08BF1EE10FA05D2B0EE000B28EE000B0C
:108F9000B0EE408B9FEDD00BB4EEC08BF1EE10FA2B
:108FA00003D29FEDCD0BB0EE408BCD4890ED020B80
:108FB00020EE080BBDEEC00B10EE104A0120FEF7AC
:108FC000EEFD08B9002006E701202AF0AFFB0120E2
:108FD0002AF012FC2046FFF70DF920B90020FEF719
:108FE000DEFD0020F7E66042FFF704F928B9002013
:108FF000FEF7D5FD0020EEE61CE0BA48007800F050
:109000000200B0B1B24890ED280BB0EE409BFEF7E5
:109010001AFF50B9AE4880ED289B0020FEF7BFFD37
:109020000720B14948700020D5E6A94880ED289B6B
:1090300000BF0CE0AD48007820F00200AB4908709A
:109040000021AB4A9160D16001202AF0D5FB0020BD
:10905000FEF7A5FDFFF7B3FD08B90020BBE6A54864
:10906000407880BB9A4890F85502022804D19F4866
:10907000007800F0020020B9954890F855020328C6
:1090800022D10120FFF766FC002801DA0020A2E6C9
:109090009648007800F00200A8B18D4890F855027B
:1090A000022811D18B48407868B90020FFF752FCA4
:1090B000002801DA00208EE60020FFF74BFC002894
:1090C00002DA002087E6FFE7FFF795F9FEF7B4FD27
:1090D000ADB18648007800F0020080B17C4890F87D
:1090E000D10101280BD1811E2CF03BF8824AD2E934
:1090F0000E32181A62EB01027D49C1E902027B4877
:10910000007800F0020058B17C48007840F002007E
:109110007A4908706E4890F8A5026E49487008E0D8
:109120007648007820F002007449087000206949F0
:1091300048700120FEF7CEF908B900204BE6FFF792
:10914000B3FB08B9002046E6614890F8E501801EAF
:1091500006287DD2DFE800F0030406073B3C00BF91
:10916000012038E600BF6648407810B16548407875
:1091700008B900202FE6644890ED020B544880EDBA
:10918000280B6248D0E90230614AD2E902125E1827
:1091900040EB0201022200233046F7F7F0FA5D4A65
:1091A000C2E9020100234FF48062194602204FF009
:1091B000E5FD0A210846FEF74BF908B900200AE64A
:1091C0000120FEF787F908B9002004E65EE000BF41
:1091D0004B48407808B90020FDE54B4890ED020B64
:1091E0003B4880ED280B4948D0E9022110467BF02E
:1091F00041FC41EC100B364890EDBB1AB7EEC11A9A
:10920000B7EE082B31EE021B9FED433B81EE032BA3
:10921000334890ED021B22EE011B1FEDD62B01EE11
:10922000420BB0EE408B51EC180B7BF0B9FD394A84
:10923000C2E90201FF234FF48062002102204FF0B7
:109240009DFD0A210846FEF703F910B90020C2E58A
:109250001AE02E49D1E902012E4AC2E90201002397
:109260004FF48062194602204FF088FD0A2108461B
:10927000FEF7EEF808B90020ADE50120FEF72AF967
:1092800008B90020A7E501E00020A4E500BF012007
:10929000A1E52DE9F04F2DED088B83B004460020A9
:1092A00002901148407810B91E200F4948700848B4
:1092B00090F8500200F0020028B9012003B0BDEC84
:1092C000088BBDE8F08F2BE088030020A19B0424CD
:1092D000300605244C0500209A9999999999A93F3F
:1092E0005801002488420030A69B0424B4050020C5
:1092F000B80500208442003090070020703400241C
:10930000CE9A0424D29A0424809A0424D89A04245D
:10931000F89A0424E00800200000000000408F407C
:10932000F748007800F0020028B9002003B0BDEC37
:10933000088BBDE8F08FF34890F85502012801D062
:109340000120F3E7F04890F8510000F0300008B138
:109350000120EBE70120ED494880EA4890ED060B3B
:10936000EB4890ED021B20EE010BBDEEC00B10EEA2
:10937000105AE44890ED9C0AB7EEC08AE5480078A0
:1093800000F0020030B1DF4890ED530AB7EEC00A9A
:10939000B0EE408BDB4890ED530AB7EEC00AB4EE56
:1093A000C80BF1EE10FA05D290ED530AB7EEC00AE1
:1093B000B0EE408BD34890ED340BB4EEC80BF1EE19
:1093C00010FA03D290ED340BB0EE408BD248D0F8B7
:1093D000AC000190DFF84493002C1FDBC94890F8E3
:1093E000ED0100F00800C8B9CD4890ED010AB5EED6
:1093F000C00AF1EE10FA11DD90ED010AB7EEC00AD5
:10940000C34890ED021B20EE010BBDEEC00B10EE29
:10941000101AC148D0F8AC0001EB0009BA4890F826
:10942000480020F02000B84981F84800002C0ADBF1
:10943000BC4890ED021B21EE081BB0EE410B012051
:109440000AF045FE0BE0B74890ED021BB1EE482B49
:1094500021EE021BB0EE410B01200AF038FE00BFE6
:109460000A2079F07DFCB048C07804281DD1AA48B4
:10947000D0F88800C8B1A248007800F00200A0B17E
:10948000A14890F84A0000F0020070B9002C02DBFD
:10949000A648407948B9002C02DAA448C07820B91F
:1094A0009D48D0F8AC0048450EDB9848408848F20B
:1094B0000101084040B99848B0F8940020B9022250
:1094C0000121084651F0A5FA4FF0FF32012108466C
:1094D0002BF0F5FC0E4600BF00BF00BFBFF34F8F5F
:1094E000BFF36F8F00BF00BF00BF874890F84800F0
:1094F00000F0200000B90196834890F8480000F081
:10950000200028B98148408800F001000028A7D039
:109510009FED870B01200AF0DAFD32210A20FDF7CA
:1095200097FF08B9002001E7774890F8480000F05D
:10953000200020B91420804948700020F6E67248C7
:1095400090F8480020F020006F4981F848007248E8
:10955000D0F8880020B90320774948700020E5E65C
:109560007648408800F00300012802D1642079F099
:10957000F7FB6D48C078042803D000206E4948707E
:10958000D4E66F490198C860002088605D4890ED7E
:109590008E0BB7EEC0AB9FED6B0AB4EEC0AAF1EE36
:1095A00010FA04DD9FED670AB0EE40AA0AE09FEDD5
:1095B000660AB4EEC0AAF1EE10FA03D29FED630A78
:1095C000B0EE40AA6248D0ED010AB0EE001A80EE7B
:1095D000810AB4EECA0AF1EE10FA07D290ED010A40
:1095E000F0EE000A80EE201AB0EE41AA5448C1689D
:1095F000474890ED020BB7EECA1A20EE010BBDEE04
:10960000C00B10EE100A091A4D48C160002C28DD6D
:109610004148D0F8AC0046194948C068411948484B
:10962000C160384880ED288B00234FF480621946D2
:1096300002204FF0A3FB32210A20FDF709FF08B9F1
:10964000002073E63448D0F8880008B900206DE6A1
:109650003548C078042801D0002067E63848C66045
:1096600029E0002C27DA2C48D0F8AC00461B3448FF
:10967000C068411B3248C160224880ED288B00231E
:109680004FF48062194602204FF078FB32210A2005
:10969000FDF7DEFE08B9002048E61F48D0F8880034
:1096A00008B9002042E62048C078042801D00020F4
:1096B0003CE62348C660144890F8510000F00400CE
:1096C000E8B1104890ED8E0B9FED221B20EE019B20
:1096D0009FED220BB4EEC09BF1EE10FA03D29FED8A
:1096E0001F0BB0EE409BB7EE000BB4EEC09BF1EE4B
:1096F00010FA3EDDB7EE000BB0EE409B39E031E0F2
:10970000B40500203006052488030020F005002061
:1097100058010024BA420030200700200000F47EE7
:10972000243500249801002400060020B8020024FB
:109730000000000000000000A69B0424500500204B
:10974000E00800200AD7A33C0AD7A33B6F12033BD3
:10975000189B0424000000000088B3400000004073
:10976000E17A943FFE4890ED8E0B9FEDFE1B20EEBC
:10977000019BB4EEC89BF1EE10FA01DDB0EE489B00
:10978000F74880ED289BF948007840F00200F7493F
:10979000087000234FF48062194602204FF0EEFA61
:1097A0001EE00A2079F0DCFAF148C078042808D1DC
:1097B000EE48007800F0020018B1EE48D0F88800BA
:1097C00070B9ED48408848F20101084040B9E948C5
:1097D000B0F8940020B902220121084651F019F98D
:1097E000E548408800F001000028DAD032210A2044
:1097F000FDF72EFEDF48D0F8880008B9002095E577
:10980000DE48408800F00300012802D1642079F08E
:10981000A7FAD748C078042801D0002086E5D348AD
:10982000007800F0020018B11520D549487068E1B1
:109830004FF48062012108462BF041FBD14AC2E976
:109840000201002C1FDD1046C06841191046C1609E
:10985000C34890ED8E1BCC4890ED022B21EE021BED
:109860009FEDCA2B21EE021BB0EE410B51EC100B09
:109870007BF096FAC34BD3E9022380185941C14AC1
:10988000C2E9020106E0002C04DABE48C068411BB0
:10989000BC48C160BF4890F8510000F00400A0B17E
:1098A000AF4890ED8E1BB84890ED022B21EE021BC5
:1098B0009FEDB92B21EE021BB0EE410B51EC100BCA
:1098C0007BF06EFA074688464EE0B548D0F824B0E3
:1098D000D0F834A0AF48B0F93400ABEB000BAD4882
:1098E000B0F93600AAEB000AAA49B1F9421001FB0F
:1098F0000AF0C11700EB51514FEAE12ABBF5004FC6
:1099000002DB47F6FF7B04E01BF5004F01DCDFF8CC
:1099100094B2BAF5004F02DB47F6FF7A04E01AF57D
:10992000004F01DCDFF87CA20FFA8AF10FFA8BF00E
:10993000FAF70FFA00EE100AB8EEC00B924890ED5D
:10994000021B874890ED8E2B21EE021B20EE010BAF
:109950009FED951B20EE010BB0EE40BB51EC1B0BB5
:109960007BF01EFA074688467D4890F8520200F0C8
:10997000020048B18348D0E90210C91940EB080041
:10998000804AC2E9021008E07E48D0E90210C91BF3
:1099900060EB08007B4AC2E90210714890ED530A5F
:1099A000B7EEC00A80ED280B00234FF48062194601
:1099B00002204FF0E3F932210A20FDF749FD08B9F2
:1099C0000020B3E46B48D0F8880008B90020ADE46B
:1099D0006748C078042801D00020A7E4744890EDBF
:1099E000020BB5EEC00BF1EE10FA3BD05C4890EDE7
:1099F000530AB7EEC00A80ED280B6D4890ED021BAC
:109A0000614890ED022B21EE021B9FED602B21EEB1
:109A1000021BB0EE410B51EC100B7BF0C1F9554B22
:109A20007033D3E90E2380185941564AC2E9020126
:109A300000234FF48062194602204FF09FF9322133
:109A40000A20FDF705FD08B900206FE44948D0F869
:109A5000880008B9002069E44548C078042801D08E
:109A6000002063E44B4890F8510000F0040058B126
:109A70003B4890ED8E0BB1EE001B80EE012BB7EE54
:109A8000C20B80EDB70A19E0354890ED8E0B9FEDC3
:109A9000492B80EE021B90EDB70AB7EEC00AB4EE78
:109AA000C01BF1EE10FA09D290ED8E0B9FED411B19
:109AB00080EE012BB7EEC20B80EDB70A05200090B7
:109AC00000BF142079F04CF92C48408800F00300C6
:109AD000012802D1642079F043F90098411EC9B2EF
:109AE00000910028EDDC3548007800F0020038B124
:109AF000284890F84A0000F0020008B901200290BE
:109B000000BF1A48007820F00200184908700120B0
:109B1000FDF7E0FC029808B316487030D0E90E213A
:109B200010467AF0A7FF41EC100B254890ED022B70
:109B30009FED161B82EE013B20EE030B214880EDCA
:109B4000020B90ED020BB1EE400B1F4880ED020BB3
:109B50000B4840781E283BD1002037E038E0000059
:109B60003006052400000000006AA8404B050020D4
:109B70000006002020070020F005002050050020EE
:109B8000A69B0424E00800205801002400000000E7
:109B90000000F04188030020000000000000D041D8
:109BA000386904240180FFFF000000000000F0403D
:109BB000800A05240000000000004040B405002099
:109BC00078010024609B0424D8000024FE494870DA
:109BD000FE4890ED020BFE4880ED280BFD48C07852
:109BE000042801D000209EE402989CE470B52DED7D
:109BF000048BF848C078042803D00020BDEC048B07
:109C000070BDF34890F8500200F0020020B91F2008
:109C1000ED4948700020F1E7ED4890F85502012821
:109C200004D02020E84948700020E7E7E84890F891
:109C3000D101032804D12120E34948700020DDE749
:109C4000E54890F8510000F0060020B92220DE49D6
:109C500048700020D2E7E04890F84B0000F0020086
:109C600020B92320D84948700020C7E7DA4890F887
:109C70004A0000F0020020B12420D349487000209F
:109C8000BCE70120D54948809FEDD50BD64880ED33
:109C9000020B0020D54948809FEDD10BD44880EDC0
:109CA000020B0020FDF716FC08B90020A6E7D149F9
:109CB000D1E90E01D04AC2E902010024CF48407820
:109CC000822802D0CE48C07808B1012408E0CB48F1
:109CD0004078832802D0CA48407908B14FF0FF3459
:109CE000C8480078C8490978084000F002000028F8
:109CF0007DD100E000BFC54890F900000028F9DAE6
:109D00000120C24908702AF017FE40B1B24890F80D
:109D10004A0040F00200B04981F84A0007E0AE482E
:109D200090F84A0020F00200AB4981F84A00FF2079
:109D3000B6490870A64890F8500200F002000028CA
:109D40007DD0A54890F84A0000F00200002876D1A6
:109D5000A14890F8510000287ED09D4890F8D1018C
:109D6000032879D0AA48407840B10020A84948701B
:109D7000974991F8A812480078F0F2FF964890F8B9
:109D8000510000F0070038B1914890ED8E0BB0EE15
:109D9000001B20EE018B06E08D4890EDA20BB3EE88
:109DA000041B20EE018B8A4890ED060B9FED991B5A
:109DB00020EE011B90ED0E2B81EE020BB4EEC80BD2
:109DC000F1EE10FA0BDD90ED060B9FED921B20EEED
:109DD000010B90ED0E1B80EE012BB0EE428B7C4808
:109DE00090ED060B9FED8D1B20EE019B00E056E0F1
:109DF000B4EEC98BF1EE10FA01D2B0EE498B89486E
:109E000090ED020B20EE080BBDEEC00B10EE105AC9
:109E10000120FDF7C4FE08B90020EFE6012029F07B
:109E200085FC012029F0E8FC002C09DB2846FEF720
:109E3000E1F928B90020FDF7B2FE0020DEE60BE0D4
:109E4000002C08DC6842FEF7D5F920B90020FDF7A8
:109E5000A6FE0020D2E60CE06A48007820F002005E
:109E6000684908700021704A9160D160012029F092
:109E7000C3FC6448007800F0020068B14FF0FF3185
:109E800001202BF06EF95B4AD2E90E32181A62EB10
:109E900001026549C1E902020020FDF780FE594830
:109EA000007800F0020020B90B20474948700020DC
:109EB000A4E6FEF7A0FAFDF77BFD2046FFF7E9F9DF
:109EC00006465A48007820F0020058490870FDF70D
:109ED00034FE0EB9002091E6FEF78DFAFDF7ACFED8
:109EE0004848007800F0020058B14748007840F038
:109EF000020045490870364890F8A5024449487068
:109F000008E04148007820F002003F490870002036
:109F10003F4948700120FDF7DDFA08B900206DE6E1
:109F2000FEF7C2FC6AE670B52DED088B2948C078B3
:109F3000042803D00020BDEC088B70BD0120274908
:109F400048809FED270B284880ED020B0020274911
:109F500048809FED230B264880ED020B0020FDF783
:109F6000B9FA08B90020E6E72248D0E90E10224AE3
:109F7000C2E90210164890ED570AB7EEC0AAB7EE34
:109F8000000BB4EEC0ABF1EE10FA03DDB7EE000B40
:109F9000B0EE40AB0E4880ED28AB254890ED010AAD
:109FA000B7EEC00A1F4890ED021B20EE010BBDEE7C
:109FB000C00B10EE101A0F487038D0F8AC000144F6
:109FC0001C48C160002337E0A69B0424809A042427
:109FD000300605240006002088030020F00500203C
:109FE0000000000000000000200200248002002485
:109FF0004002002490070020809B0424A29B04249C
:10A00000B8020024B405002070340024A19B04246D
:10A010004C050020FCA9F1D24D62603F7B14AE4795
:10A02000E17A743F58010024B80500204B05002058
:10A03000189B0424E00800204FF480621946022097
:10A040004EF09CFE0A210846FDF702FA08B90020EE
:10A0500071E70120FDF73EFA08B900206BE7002503
:10A06000FE4890F8D10180B1FC4890F8D101032856
:10A070000BD0FA4890F8500200F0020028B1F848DE
:10A08000007800F0020000B90125F44890F8D101F1
:10A0900030B1F448007800F0020008B9002D7CD0FF
:10A0A00000E000BFF04890F900000028F9DA012034
:10A0B000ED4908702AF040FC40B1EC4890F84A00A5
:10A0C00040F00200E94981F84A0007E0E74890F8CB
:10A0D0004A0020F00200E54981F84A00FF20E249E9
:10A0E0000870DE4890F8500200F00200002872D09C
:10A0F000DE4890F84A0000F0020000286BD1DB48EF
:10A1000090F851000028F2D0D44890F8D1010328EB
:10A1100061D0D748407840B10020D5494870CF4938
:10A1200091F8A812480078F01BFED04890F8510032
:10A1300000F0070038B1C94890ED8E0BB0EE001B5F
:10A1400020EE018B06E0C54890EDA20BB3EE041B98
:10A1500020EE018BC14890ED060B1FED521B20EE47
:10A16000011B90ED0E2B81EE020BB4EEC80BF1EE4D
:10A1700010FA0BDD90ED060B1FED5A1B20EE010BC4
:10A1800090ED0E1B80EE012BB0EE428BB94840786B
:10A1900048B1B24890ED060B00E075E01FED611B81
:10A1A00020EE019B01E09FEDB49BB4EEC98BF1EE74
:10A1B00010FA01D2B0EE498BB14890ED020B20EEBF
:10A1C000080BBDEEC00B10EE104A0120FDF7E7FCB6
:10A1D00010B90020AFE634E0012029F0A7FA0120F1
:10A1E00029F00AFB2046FEF705F820B90020FDF70C
:10A1F000D6FC00209FE66042FDF7FCFF20B900205E
:10A20000FDF7CDFC002096E69648007800F00200AD
:10A21000B0B1924890ED280BB0EE40BBFDF713FEB5
:10A2200050B98E4880ED28BB0020FDF7B8FC072010
:10A230009449487000207EE6884880ED28BB00BF26
:10A240000CE08748007820F0020085490870002063
:10A250008D4A9060D060012029F0CEFA80480078C5
:10A2600000F0020068B14FF0FF3101202AF079FFC1
:10A27000864AD2E90E32181A62EB01028249C1E91C
:10A2800002020020FDF78BFCFEF799FC08B90020C4
:10A2900051E67F48407880BB704890F8550202280C
:10A2A00004D16F48007800F0020020B96B4890F8A4
:10A2B0005502032822D10120FEF74CFB002801DAC9
:10A2C000002038E66648007800F00200A8B1634834
:10A2D00090F85502022811D16548407868B90020ED
:10A2E000FEF738FB002801DA002024E60020FEF704
:10A2F00031FB002802DA00201DE6FFE7574890F8FE
:10A300005502012829D1554890F8500200F002006A
:10A3100018B3564890F8510000F00700E8B15048D3
:10A32000007800F0020020B90B2056494870002048
:10A3300001E6FEF760F8FDF73BFB0020FEF7A9FF02
:10A3400004465448007820F0020052490870FDF796
:10A35000F4FB0CB90020EEE500BFFEF74CF8FDF76A
:10A360006BFCADB13E48007800F0020080B13B4884
:10A3700090F8D10101280BD1811E2AF0F2FE434A48
:10A38000D2E90E32181A62EB01023F49C1E902021A
:10A390003348007800F0020058B13F48007840F0A0
:10A3A00002003D4908702D4890F8A50230494870D8
:10A3B00008E03948007820F0020037490870002092
:10A3C0002B4948700120FDF785F808B90020B2E557
:10A3D000FEF76AFAAFE510B53048C078042801D01E
:10A3E000002010BD01202E4948801C4890ED640BD0
:10A3F00090ED5F1AB7EEC11A80EE012BB0EE000BA4
:10A40000B4EEC02BF1EE10FA06DD90ED5B0AB7EE6C
:10A41000C00A80ED280B06E0104890ED5F0AB7EE09
:10A42000C00A80ED280B0D4890ED280B90ED341BF1
:10A43000B4EEC10BF1EE10FA03DD90ED340B80EDBC
:10A44000280B064890ED641B164890ED010AB7EE04
:10A45000C00A31EE001B0A4826E000003006052441
:10A46000B405002088420030A19B0424880300200A
:10A470004C050020A29B04249A9999999999A93F87
:10A4800058010024A69B0424B80500209007002052
:10A49000844200304B050020703400240006002068
:10A4A000F0050020189B042490ED022BFE4890ED4F
:10A4B0002B0AB8EEC00B01EE420BBDEEC00BFB4801
:10A4C00080ED030A00234FF48062194602204EF00B
:10A4D00055FC64210A20FCF7BBFF08B9002080E787
:10A4E0000120FDF75CFB28B10120FCF71EFC0020D9
:10A4F000FDF755FB0021EE4A9160D160ED4890F8E0
:10A50000C90128BBE8497031D1E90E01EA4AC2E924
:10A510000201E5497031D1E90E01E84AC2E90201C0
:10A52000E1487030D0E90E10E54AC2E90210E54872
:10A53000007800F0020058B1E048D0E90220E2497A
:10A54000D1E90231D21A60EB0100D949C1E90220F8
:10A550000120FCF7BFFF012043E700BF002079F096
:10A56000ABFCDA48C07800F0080010B10421D748ED
:10A57000C1700020D6494870D6494870D64A9060CC
:10A58000D060D64A9060D060D54948704524C6480E
:10A59000D0F8880008B9542468E1CC48C07800F0AD
:10A5A000020008B1452461E1C848807800F001004C
:10A5B00000287CD0FDF794F8CA48007800F002002B
:10A5C00048B1C94890F8510000F0060018B1FFF7F3
:10A5D0000DFB05460BE0B74890F8E501012803DCC8
:10A5E000FFF7A1FC054602E0FEF7ECFB0546002064
:10A5F000FDF7D5FABD48007820F00200BB4908708D
:10A60000BB48007820F00200B9490870B5480078CE
:10A6100020F00200B3490870FDF792F93224B548E2
:10A62000408800F0010088B901219F48A0F89410EB
:10A6300004E0601EC4B20A2078F092FBAD48408866
:10A6400000F0010008B9002CF3D1002585B3AA4819
:10A65000007800F0020058B3A84890ED000AB5EE6B
:10A66000C00AF1EE10FA2CD0A54890ED021BA348C9
:10A6700090ED000AB7EEC00A21EE000BBDEEC00B54
:10A6800010EE101A8848D0F8AC0001448748C16029
:10A6900000234FF48062194602204EF06FFB6421C4
:10A6A0000A20FCF7D5FE00B900257F4801E098E0BC
:10A6B00007E0D0F8AC107D48C068814238D0002552
:10A6C00036E0ADB38C48007800F0200080B38B48B2
:10A6D00090ED080AB5EEC00AF1EE10FA28D08848CD
:10A6E00090ED021B854890ED080AB7EEC00A21EEF6
:10A6F000000BBDEEC00B10EE101A6B48D0F8AC008A
:10A7000001446A48C16000234FF480621946022068
:10A710004EF034FB64210A20FCF79AFE00B90025B4
:10A720006148D0F8AC106148C068814200D0002573
:10A730007148007820F022006F4908708DB163489D
:10A74000C07804280DD16F48407810B901206D49B8
:10A7500048705C48007840F002005A490870412473
:10A7600019E05148D0F8880018B9032065494870AD
:10A770000DE05648C078022803D105206149487091
:10A7800005E06048407810B902205E4948704524D1
:10A7900002214E48C170544890F8510000F0070063
:10A7A00028B15948007820F002005749087041F05C
:10A7B00085FB022078F0D4FA5448406810B10A2092
:10A7C00078F0CEFA012050F0D9F918B90021012013
:10A7D00043F0A8F94E48C07810B10E204D4988804A
:10A7E00044E03A48807800F00200E8B3FCF778FFD4
:10A7F000FFF7F1FD0546FDF7A3F85DB13348C078DA
:10A80000042807D12F48407840F002002D494870B5
:10A8100044241AE032243748408800F0010080B90F
:10A8200001212148A0F8941004E0601EC4B20A205F
:10A8300078F096FA2F48408800F0010008B9002C03
:10A84000F3D1452402212148C170012050F096F92E
:10A8500018B90021012043F065F92D48407910B165
:10A860000E202C49888001E0FFE70024D4B10E4877
:10A87000D0F8880020B9412C02D0442C00D05424B8
:10A880000020FDF78CF92448007860B90648B0F83C
:10A89000940040B11748408800F0010018B1002131
:10A8A00001483BE04EE03BE020070020E0080020AC
:10A8B000483500243006052480060020C00600200C
:10A8C00000070020A40B0020A006002000060020A6
:10A8D000CE9A0424D29A0424D89A0424F89A042400
:10A8E000CA9A0424BA42003088030020C80C002011
:10A8F0004B050020F005002000430030C04200302E
:10A9000058010024A69B0424B5050020C00D00209A
:10A91000B8020024C8000024AF0D0020A0F8941055
:10A920000020094948700948447000BF00BF00BFBB
:10A93000BFF34F8FBFF36F8F00BF00BF00BF012178
:10A940000348C1700AE6000084420030AC9B042436
:10A95000000600202DE9F04104460D4627462E460C
:10A96000002F00DC0127002E00DC012619E0F94849
:10A970004079042803D1F848D0F8F80070B9F748B6
:10A98000808848F20101084040B9F348B0F804015A
:10A9900020B902221146104650F03BF8384678F0B4
:10A9A000DFF9EE48808800F001000028DFD0EA4897
:10A9B000D0F8F80028B90420E94988700020BDE8E3
:10A9C000F081304678F0CCF9E2484079042801D093
:10A9D0000020F4E70120F2E770B50546322078F058
:10A9E000BFF9E048007800F0040028B1DE48807824
:10A9F00010B9322078F0B4F9DA48007800F0040099
:10AA000010B1D948807808B9012070BDD748808836
:10AA100000F0010008B90120F7E7052405B114246E
:10AA200013E0CC484079042801D00020EDE7002154
:10AA3000CF4881664166322078F092F9CC48406E6A
:10AA400008B90120E1E7601EC4B2002CE9DC012056
:10AA5000DBE72DE9F0412DED0A8B04460D46164645
:10AA60001F46C44890ED2A0BB0EE409B90ED580A6B
:10AA7000B7EEC00AB0EE408B90ED540AB7EEC00AB4
:10AA8000B0EE40CB90ED360BB4EEC80BF1EE10FA01
:10AA900003D290ED360BB0EE408BB64890ED360BFE
:10AAA000B4EECC0BF1EE10FA03D290ED360BB0EE13
:10AAB00040CB66B1B7EE000BB4EEC08BF1EE10FAEE
:10AAC00003DDB7EE000BB0EE408BB0EE48CBAA48EA
:10AAD00090ED040B20EE080BB7EEC0ABB5EEC0AAAC
:10AAE000F1EE10FA03D19FEDA50AB0EE40AA9A4903
:10AAF000D1F81C11681A002801DB014600E0414230
:10AB000000EE101AF8EEC0AA8AEE8ABAB0EE000A79
:10AB1000B4EEC0BAF1EE10FA03DD964880ED2ACB10
:10AB200002E0944880ED2A8BB7B39548C0E904450C
:10AB3000944890ED020AF2EE040A80EE201AB7EE75
:10AB4000C11A8D4890ED042B8D4890ED050AB8EEA2
:10AB5000C00B01EE420BBDEEC00B80ED050A0023D9
:10AB60004FF48062194604204EF008F90A21084685
:10AB7000FFF7F0FE38B97F4880ED2A9B0020BDEC3E
:10AB80000A8BBDE8F0810020FFF726FF28B979483D
:10AB900080ED2A9B0020F2E702E0764880ED2A8BC8
:10ABA0007748C0E9044500234FF480621946042029
:10ABB0004EF0E4F80A210846FFF7CCFE20B96D48B4
:10ABC00080ED2A9B0020DAE70120FFF705FF20B97E
:10ABD000684880ED2A9B0020D1E7664880ED2A9BDB
:10ABE0000120CCE71CB50020009001905E498978D7
:10ABF000F1B35C49097801F00401C9B3624991F8E5
:10AC00004A1001F0040199BB6049897801F0010103
:10AC100071B3594991ED040B9FED5D1B20EE010BC3
:10AC2000B0EE002B80EE021B5B494869002801DB77
:10AC3000014600E0414200EE101AB8EEC00BB4EE3F
:10AC4000C01BF1EE10FA18D2012102202AF089FA75
:10AC5000CDE900014048D0F81C010199411A3E4855
:10AC6000D0F8240101443C48C0F82411E03000E051
:10AC700003E0DDE90021C0E90E213E4890F82601FD
:10AC800048B93C4890F83601032804D0434800787E
:10AC900000F0040060B19FED420A3A4880ED020ADC
:10ACA000344890F8260140F080003E49887007E063
:10ACB0009FED320A334880ED020A0020394988703E
:10ACC0002C4890ED2A0B384880ED040B294890F869
:10ACD0001203364988702748B0F814013449888037
:10ACE000244890F81A0133498870224890EDB40A3C
:10ACF000314880ED020A1F4890F826012F498870DC
:10AD00001C4890F8EE042E4988700021194880F8FC
:10AD1000261180F8EE1480F812136421A0F81411A3
:10AD2000002180F81A1190ED080BB2EE081BB4EE6A
:10AD3000C10BF1EE10FA45DD90EDB40AF7EE000A12
:10AD4000B4EEE00AF1EE10FA3CD2B7EE000A80ED64
:10AD5000B40A45E00006002020070020F00500208E
:10AD6000A69B0424B40500204C05002050050020BB
:10AD7000D00900203006052458010024CDCCCC3D5C
:10AD8000E0080020189B042488030020B40200245B
:10AD9000000000A09999B93F58050020BA42003040
:10ADA000B4A29139A29B0424809A0424A09A04247A
:10ADB000A89A0424A49A0424B09A0424789A042417
:10ADC0007C9A0424FE4890EDB40A5FED140AB4EEB8
:10ADD000E00AF1EE10FA03D21FED180A80EDB40A72
:10ADE000F8488088642802DA0A2077F0B9FFF6482C
:10ADF0004079082822D10421F34841710198E8B133
:10AE0000F248807800F0010070B140F2E241F04871
:10AE1000A0F8061102E0012077F0A2FFEC48B0F99B
:10AE200006010128F7DC09E0E848807830B1E44900
:10AE3000B1F8B41201F10A0077F092FF0120E54960
:10AE400088701CBD10B5E348807800B910BD0220A1
:10AE50000BF03AFFE0488178D94880F82611DF48A6
:10AE60008178D74880F8EE14DD4890ED040BD44883
:10AE700080ED2A0BDB488178D14880F81213D14845
:10AE8000808801B2CE48A0F81411D7488178CC4808
:10AE900080F81A11D54890ED020AC94880EDB40A2D
:10AEA000D34890F8480020F04000D14981F848008C
:10AEB00000BFCBE7C24890EDB80ACE4880ED020A49
:10AEC000C2488078CC498870BD4890F8BE02CB4912
:10AED0008870BB4890F8C202C9498870B848B0F879
:10AEE000B402C8498880B648B0F8B4023F2803DAF3
:10AEF0003F21B348A0F8B4124FF0FF30C249886038
:10AF0000AF48D0F8AC02B0F51C7F08D8AC48D0F8F8
:10AF1000AC02886040F27120A949C1F8AC02B44883
:10AF200090F8520000F0400058B1A54890EDA40BF5
:10AF3000B1EE001B20EE010BB7EEC00B80EDB80A9E
:10AF400010E0AB4890F8520000F0040050B19C486B
:10AF500090ED900BB0EE001B80EE012BB7EEC20B14
:10AF600080EDB80A964890EDB80ADFEDA80AB4EE75
:10AF7000E00AF1EE10FA03D29FEDA40A80EDB80AC0
:10AF80009C4890ED020AB2EE041AC0EE010A8C4809
:10AF900090EDB80AF4EEC00AF1EE10FA0ADD954819
:10AFA00090ED020AF2EE040A80EE201A844880ED49
:10AFB000B81A17E0824890EDB80A8E48D0ED020A20
:10AFC000B2EE041A60EE810AB4EEE00AF1EE10FA75
:10AFD00008DD90ED020AF2EE040A20EE200A78481D
:10AFE00080EDB80A764890F8BE02022803DA022102
:10AFF000734880F8BE12724890F8C202022803DA41
:10B0000002216F4880F8C2126D4890F8A60202280B
:10B0100011DA6B4890F8BE02142803DD1421684849
:10B0200080F8BE12664890F8C202142803DD14218D
:10B03000634880F8C21202206449887070477248E1
:10B0400080680021494071EA000004D06E488068A1
:10B050005B49C1F8AC024FF0FF306B49886069482A
:10B0600081885748A0F8B412624890ED020A54480B
:10B0700080EDB80A6048807854498870504890F84C
:10B08000A60202280CDA5C48807888705B488178D8
:10B090004B4880F8BE125A488178494880F8C2125D
:10B0A000704770B5054655B959480078022804D153
:10B0B000FF2057490870012070BD0020FCE74FF4C5
:10B0C000FA76632400BF40484079042801D000206C
:10B0D000F2E7301EA6F101010EB204DC0A204D4950
:10B0E00088700020E8E74A4890F90000002803DA59
:10B0F0000220474908701BE0454890F90000A04233
:10B1000013D0434890F90040002C0CDB4248807D6E
:10B11000A04208DD0120A04040490978084010B154
:10B1200040F26B3601E04FF4FA76282077F018FEF3
:10B13000374800780228C6D10120BDE770B52648FF
:10B140008078002800DD70BD2148E030D0E90E4550
:10B150001B4890F8E60102282BDB314890ED040BE8
:10B16000B5EEC00BF1EE10FA08D82E48D0F88800E2
:10B1700000F4802010B900242B4D1AE0284890EDEF
:10B18000041B2A4890ED042B21EE021B9FED282B77
:10B1900021EE021BB0EE410B51EC100B79F000FEDA
:10B1A000241A65EB01052448C0E904450120234920
:10B1B0008870034890F8CA0100287DD1204841E0FA
:10B1C00030060524A89A0424000600204C0500201F
:10B1D00020070020CA9A0424789A04247C9A042424
:10B1E000809A0424A09A0424A49A0424B09A0424E3
:10B1F00088030020289B0424389B04243C9B0424BF
:10B20000409B0424449B04244C9B042417B7D1384E
:10B21000A09B0424A69B0424400000248842003004
:10B22000800A05249034002400000C815801002479
:10B23000000000000000F041D89A0424CE9A0424B3
:10B2400060060020C0E90445FE48C0E90445FE4808
:10B25000C0E90445FD4890F8EE0100F0040060B339
:10B26000FA4890F8D20101282FD0F84890F8E6016A
:10B2700002282ADAF6484069002826DDF548D0E998
:10B280000410F34AD2E90432C9185041F24AC2E923
:10B2900004101046D0E90410F04AC2E90410EE4848
:10B2A000D0E90410EE4AC2E90410EB48D0E90410DA
:10B2B000EC4AC2E9041001E045E006E0EA484078C3
:10B2C00040F00400E84948703DE0E84890ED020A8B
:10B2D000B5EEC00AF1EE10FA35DD90ED021AB7EEC8
:10B2E000C11AE34890ED042B31EE021BE14890EDCA
:10B2F000042B21EE021B1FED322B21EE021BB0EEC0
:10B30000410B51EC100B79F04BFDD34AC2E904011B
:10B310000120D94988701046D0E90410CF4AC2E90B
:10B320000410CD48D0E90410CD4AC2E90410CA483F
:10B33000D0E90410CB4AC2E90410CB48407840F071
:10B340000400C949487000BFFDE62DE9F0412DED2C
:10B35000028BCA48807850B10020C8498870BB4928
:10B3600091F8A812490001F1640077F0F9FCC44893
:10B3700090ED040B9FEDC31B81EE002BB34880EDD5
:10B380002A2BC248D0E90E45C148C0E90445AF495F
:10B39000B1F854100803C11700EBD1614A11BC4940
:10B3A00049690A44BA494A6100234FF48062194648
:10B3B00004204DF0E3FCFA210A20FFF7CBFA20B974
:10B3C0000020BDEC028BBDE8F081B048E038D0F839
:10B3D0001C11AF484069814201D00020F1E7AB4920
:10B3E000D1E90E01AA4AC2E9040110464169974811
:10B3F000B0F854004FF4805202FB0011A4484161A0
:10B400009FEDA48B4FF0000815E0012077F0A8FC19
:10B410004FF0FF320121022029F051FD064679F05C
:10B4200029FB41EC100B38EE400BB0EE408B08F1DD
:10B43000010000F0FF08B8F1080FE6DB00234FF42D
:10B440008062194604204DF099FCFA210A20FFF78A
:10B4500081FA08B90020B4E78C48E038D0F81C1114
:10B460008B484069814201D00020AAE74FF00008D4
:10B4700015E0012077F074FC4FF0FF32012102202B
:10B4800029F01DFD064679F0F5FA41EC100B30EE7F
:10B49000080BB0EE408B08F1010000F0FF08B8F196
:10B4A000080FE6DB7949D1E90E01794AC2E90401C6
:10B4B0006649B1F854100803C11700EBD1614A1175
:10B4C000734949690A4472494A6100234FF4806212
:10B4D000194604204DF052FC0A210846FFF73AFABB
:10B4E00008B900206DE76948E038D0F81C116848B9
:10B4F0004069814201D0002063E76448D0E90E1022
:10B50000634AC2E904105149B1F854100803C11745
:10B5100000EBD1614A115E4949698A1A5C494A6166
:10B5200000234FF48062194604204DF027FCFA21D5
:10B530000A20FFF70FFA08B9002042E75348E03825
:10B54000D0F81C1152484069814201D0002038E7F0
:10B550004E48D0E90E104E4AC2E904101046416927
:10B560003A48B0F854004FF4805202FB101148489A
:10B5700041614FF0000815E0012077F0F1FB4FF03A
:10B58000FF320121022029F09AFC064679F072FA76
:10B5900041EC100B30EE080BB0EE408B08F10100CF
:10B5A00000F0FF08B8F1080FE6DB00234FF48062DB
:10B5B000194604204DF0E2FBFA210A20FFF7CAF9F0
:10B5C00008B90020FDE63148E038D0F81C113048B9
:10B5D0004069814201D00020F3E64FF0000815E0F9
:10B5E000012077F0BDFB4FF0FF320121022029F04E
:10B5F00066FC064679F03EFA41EC100B38EE400B43
:10B60000B0EE408B08F1010000F0FF08B8F1080F20
:10B61000E6DB224890ED041B9FED212B81EE020B0F
:10B6200020EE080BB0EE408B1948C0E9044500231A
:10B630004FF48062194604204DF0A0FB0A21084611
:10B6400032E00000A0060020E006002030060524BD
:10B650004835002460060020F89A04248006002063
:10B66000C006002000070020A40B00202435002481
:10B670004002002458010024D29A04244C050020E2
:10B6800098010024000000A09999C93F00080020FB
:10B69000E008002000000000000000007801002405
:10B6A0000000000000003042FFF754F908B9002004
:10B6B00087E6FE48D0F81C11FD484069814201D060
:10B6C00000207EE69FEDFB0BB4EEC08BF1EE10FA8E
:10B6D00010DB9FEDFA0BB4EEC08BF1EE10FA09D837
:10B6E000F84880ED088B002102200BF080FC01203F
:10B6F000FFF772F9012064E62DE9F0412DED028B90
:10B7000004460025F04890F8520000F0010000B116
:10B710000125ED4890F84A0020F00400EA4981F83C
:10B720004A001FED240BB0EE408B4FF0FF3200219A
:10B73000022029F0C4FB064679F09CF941EC100B7D
:10B7400038EE400BB0EE408B012077F009FB4FF054
:10B75000FF320021022029F0B2FB064679F08AF977
:10B7600041EC100B38EE400BB0EE408B2A462146E0
:10B770000220F9F773F9D5484079042804D0002055
:10B78000BDEC028BBDE8F081642077F0E9FA4FF060
:10B79000FF320021022029F092FB064679F06AF977
:10B7A00041EC100B30EE080BB0EE408B012077F02F
:10B7B000D7FA4FF0FF320021022029F080FB064625
:10B7C00079F058F941EC100B30EE080BB0EE408BDD
:10B7D0009FEDBF0B88EE001BB0EE418BBA4890F88E
:10B7E0004B0000F00400002875D0B74890F84A00DC
:10B7F00000F0040000286ED1B0EEC81B00EE104A25
:10B80000B8EEC00BB0EE002B20EE020BB0EEC00B7A
:10B81000B4EEC01BF1EE10FA5DD8B0EEC81B00EE1E
:10B82000104AB8EEC00BB6EE002B20EE020BB0EEC5
:10B83000C00BB4EEC01BF1EE10FA4CDBA64800784A
:10B8400000F0040038BB00EE104AB8EEC00B28EE42
:10B85000000BB5EEC00BF1EE10FA07D2994890F844
:10B86000520280F00400974981F85202964890F8FD
:10B870005200042810D1934890ED900B9FED971B38
:10B88000B4EEC10BF1EE10FA06DD9348007820F01B
:10B8900004009149087026E08B4890F8520000F0AF
:10B8A000400080B1874890EDA40B9FED8C1BB4EE57
:10B8B000C10BF1EE10FA06DD8748007820F0040095
:10B8C000854908700FE08448007840F00400824900
:10B8D000087008E0FFE7002C05DD7F48007820F0C5
:10B8E00004007D4908707C48007800F0040010B91D
:10B8F000022027F081FF012042E770B52DED028B79
:10B9000086B00020049005906E4890F8E601022869
:10B9100013DB744890ED041B734890ED042B21EE6B
:10B92000021B9FED722B21EE021BB0EE410B51EC7E
:10B93000100B79F035FACDE904011FEDAA0B6D4823
:10B9400080ED040B604890F84A1063480078884303
:10B9500000F00400E8B35C4890F8520000F03000BA
:10B96000B8B3654890ED050AB8EEC00BB0EE408B59
:10B97000012077F0F5F9604890ED050AB8EEC00BAC
:10B9800030EE080BB0EE408B012077F0E9F95A4811
:10B9900090ED050AB8EEC00B30EE080BB0EE408B10
:10B9A000012077F0DDF9544890ED050AB8EEC00BA0
:10B9B00030EE080BB0EE408B424890EDA40B20EE29
:10B9C000080BB1EE001B80EE012B4A4880ED042BE2
:10B9D00000BF3C4890F8D201012822D147480078A6
:10B9E00000F00400E8B93148E030D0E90E50DDE95C
:10B9F0000461AA1B60EB0101104679F03BF841ECB1
:10BA0000100B3F4890ED041B20EE010B9FED371B00
:10BA100080EE012B3B4880ED042B06B0BDEC028B81
:10BA200070BD1FEDE40B374880ED040B2A48007809
:10BA300000F0040010B1322077F092F93248847897
:10BA40000020314988702448007800F0040018B1C3
:10BA500014B1642077F084F91FEDF20B2B4880EDD0
:10BA6000040B2B48006840F001002949086000BF22
:10BA700000BF00BFBFF34F8FBFF36F8F00BF00BF8A
:10BA800000BF0A48E030D0E90E10DDE90423891A2E
:10BA900060EB0300CDE902100448E030D0E910105B
:10BAA000DDE90232C9185041004A33E02007002086
:10BAB000E00800202D431CEBE2361A3F0000000096
:10BAC00000005940300605248803002000060020AD
:10BAD0000000000000000042B40500209A999999E6
:10BAE0009999B93F800A05245801002400000000FC
:10BAF0000000F04160020024D80500208842003098
:10BB000078010024400200244C050020D8000024C5
:10BB1000E00C0020E032C2E91010A2F1E000D0F801
:10BB200038010399411AA2F1E000C0F83811FE492A
:10BB3000DDE90420C1E90E2000BF00BF00BFBFF354
:10BB40004F8FBFF36F8F00BF00BF00BFF748006883
:10BB500020F00100F5490860F54890F8A70000F0D2
:10BB60000400002871D0F24890F89E0000286CD0A4
:10BB7000EF4890F89A00002867D1ED4A92F93A20F0
:10BB8000002A14DBEA4A92F93A30EA4A02EB8312BD
:10BB900092ED0A0AB7EEC00AE74A92ED041B20EEC6
:10BBA000010BBDEEC00BE24A82ED060A02E0002363
:10BBB000DF4A9361DE4A936A9569DB4AE03AD2F83C
:10BBC0001C21AA1A83FB02202CE0DC4A1288019275
:10BBD000DB4A9268111A0A2905DDD94A92680A3AA5
:10BBE000D74B9A6007E011F10A0F04DAD44A926841
:10BBF0000A32D34B9A60002905DDD14A9268521E61
:10BC0000CF4B9A6006E0002904DACD4A9268521CB4
:10BC1000CB4B9A6000E000BFC84A1288BDF80430E0
:10BC20009A42F8D0C64A92688242CED1C04A92F86F
:10BC3000A220002A08DDBE4A92F8A220062A03D0DC
:10BC40000123BB4A82F83E3000BFBE4890F8520044
:10BC5000A0B30A2077F084F8BA4890F8520000F0B8
:10BC60003000B8B9B84890F8520200F0040088B12A
:10BC70004FF0FF31022029F074FA0022434262EBB8
:10BC80000100DDE90412591A60EB0200AF4AC2E973
:10BC900004100FE04FF0FF31022029F062FA002378
:10BCA000424263EB0100DDE90431D2184841A74963
:10BCB000C1E904200121022014F096FBA4488470FD
:10BCC00000BFAAE62DE9F041A248007800F0040088
:10BCD00010B90020BDE8F0819A4890F8520000F0B9
:10BCE000030008B90020F5E700250024002613E032
:10BCF000052077F035F80121924880F8F810D0F847
:10BD0000E00005448F48D0F8F000044400218D483D
:10BD100080F8F810701CC6B2042EE9DB2846E9173B
:10BD200005EB91718D102046E11704EB91718C1099
:10BD30008448B0F938002D1A8248B0F93A00241A24
:10BD40008049B1F9441001FB04F0C11700EB5151D7
:10BD5000CC12291E01DB0A4600E04A42782A08DAA2
:10BD6000201E01DB024600E04242782A01DA002070
:10BD7000B0E7B5F5004F02DB47F6FF7503E015F5B8
:10BD8000004F00DC744DB4F5004F02DB47F6FF7442
:10BD900003E014F5004F00DC6F4C21B228B2F7F736
:10BDA000D8FF074607B90127384693E770B56B48B7
:10BDB00080886B498880FFF785FF044665480078D6
:10BDC00000F0040028B99FED670B684880ED040B74
:10BDD0000FE05D4890ED901B00EE104AB8EEC00BEE
:10BDE00021EE000B9FED621B80EE012B5F4880ED82
:10BDF000042B6148807808B9012070BD00205E499D
:10BE00008870504890F8520000F0030008B90020F4
:10BE1000F3E700254C4890F8280100F0040000B139
:10BE20000125564820F815404C48808820B901214A
:10BE3000534820F8151005E04948808801B2504861
:10BE400020F8151034B9404890F85602022801D164
:10BE50000020D2E70120D0E72DE9F04781460025F8
:10BE6000394890F8280100F0040000B10125364857
:10BE700090F85602022807D0334890F8560203285B
:10BE800002D00020BDE8F0873B48807808B1002050
:10BE9000F8E72D4890F8560202281AD1374830F8B2
:10BEA0001500A0B12B48007800F0040078B12648B6
:10BEB00090ED900B9FED331BB4EEC10BF1EE10FA39
:10BEC00005D3204890F8520000F0030008B9002084
:10BED000D8E71D4890F85602032805D1284830F8C5
:10BEE000150008B90020CDE728484079042802D081
:10BEF0004FF0FF30C6E70020FEF76EFD10B94FF09F
:10BF0000FF30BFE7322076F02BFFFFF7DBFE8046E5
:10BF10000D4890F8560202287DD1B8F1000F7AD072
:10BF2000164830F8150033E000080020E00C00202F
:10BF3000C4330024E855003058010024AE0B002023
:10BF40002C0600208803002030060524B8050020B8
:10BF50004C050020B40500200180FFFFA80200244A
:10BF600080020024000000000000000020020024E5
:10BF7000000000000000F0408442003090020024E5
:10BF8000A00200247B14AE47E17A943F0006002013
:10BF900008B9002076E7FC4830F91500A8EB00044A
:10BFA000B4F5004F02DBA4F5803404E014F5004F33
:10BFB00001DC04F58034F54890F82801F34991F844
:10BFC0005212484000F0040000B16442EF4890F87B
:10BFD000280100F0040000B9644214F57A5F01DA28
:10BFE00000204FE7B4F57A5F01DD00204AE7012029
:10BFF000E7498880002C62D0E44890ED902B01EE58
:10C00000104AB8EEC11B22EE011BE24890ED042B52
:10C0100021EE021B00E019E01FED2B2B21EE021B8D
:10C02000B0EE410B51EC100B78F0BAFEDA4BD3E9CD
:10C030000E23861841EB03074B4601223046394652
:10C04000FEF707FDC0BB4FF0FF301BE7CF4890F86D
:10C050005602032831D1D14830F8150008B9002024
:10C0600010E7CF488188CD4830F915000C1AB4F597
:10C07000005F02DBA4F5804404E014F5005F01DCFE
:10C0800004F58044C14890F8280100F0040000B98C
:10C0900064420120BE49888074B1BF48E038D0F8BE
:10C0A0001C01071900264B46012230463946FEF78F
:10C0B000D0FC08B9701EE5E601E00020E2E60120B0
:10C0C000E0E670B52DED028B82B00024B54890ED0E
:10C0D000100AB8EEC00B20EE000BB0EE408B90EDD6
:10C0E000110AB8EEC01B90ED110AB8EEC02BB0EEED
:10C0F000480B01EE020BB0EE408BAB48007800F02D
:10C10000400018B96120A94908701AE0A8480078D1
:10C1100000F0040090B19FEDA70BB4EEC08BF1EEE0
:10C1200010FA0BDBA548807818B162209F4908708F
:10C1300007E063209D490870012402E064209B49C8
:10C1400008709848016C9E4881629648416C9C48F2
:10C1500081639448C16B9A4881610021816400BF6A
:10C16000322076F0FDFD894890F8E601022803DBD5
:10C170000020009001903FE0844890ED6E1B9148B4
:10C1800090ED020AB1EE400AB7EEC00AB4EEC01B51
:10C19000F1EE10FA15D290ED021AB7EEC11A7D48F1
:10C1A00090ED042B21EE021B9FED872B21EE021B4D
:10C1B000B0EE410B51EC100B78F0F2FDCDE900012F
:10C1C0001AE0724890ED6E2B7E4890ED021AB7EEA1
:10C1D000C11A32EE011B6F4890ED042B21EE021BB9
:10C1E0009FED792B21EE021BB0EE410B51EC100BB1
:10C1F00078F0D6FDCDE900016C480078612809D1BE
:10C200007349DDE90030D1E904219A184841CDE9AC
:10C21000002033E065480078642809D1614ADDE9EF
:10C220000010D2E90C32C9185041CDE9001025E0C8
:10C230004FF480620121022028F041FEDDE9002355
:10C2400080185941CDE9000158480078632815D17C
:10C250004FF0FF320121022028F031FEDDE90032EB
:10C26000181A62EB0102CDE900024B49DDE900300A
:10C27000D1E90E219A184841CDE900204948806B48
:10C28000002804DD47480199806B081A01900020BE
:10C29000009001230022DDE900512846FEF7D9FB7A
:10C2A00020B9002002B0BDEC028B70BD0120FEF76A
:10C2B00093FB08B90020F5E7201EA4F101014CB260
:10C2C0003FF74EAF0120EDE72DE9F0412DED048B56
:10C2D00040484079042804D00020BDEC048BBDE820
:10C2E000F08101202A4988801FEDE20B3A4880ED59
:10C2F000040B0020394988801FEDE60B384880ED9B
:10C30000040B0020FEF768FB08B90020E5E722488F
:10C31000D0E90E102E4AC2E9041000251B4890F8FF
:10C32000D20180B1194890F8D20103280BD01748E8
:10C3300090F8500200F0040028B11D48007800F089
:10C34000040000B90125114890F8D20130B1254808
:10C35000007800F0040008B9002D7DD000E000BF97
:10C36000214890F900000028F9DA02201E490870DF
:10C3700028F0E2FAE0B31D4890F84A0040F00400CB
:10C380001A4981F84A003CE0900200243006052456
:10C39000F00500205801002400080020A00200241D
:10C3A000A8020024680C0020C80C00200200002015
:10C3B000B40500200000008030E663414C050020F9
:10C3C00038690424189B0424000000000000F04198
:10C3D000809B042400060020200200248002002408
:10C3E0004002002488420030A19B042488030020DE
:10C3F000FFE7F64890F84A0020F00400F34981F87E
:10C400004A00FF20F2490870F24890F8500200F00C
:10C410000400002872D0ED4890F84A0000F00400B3
:10C4200000286BD1E94890F85200002866D0E9480E
:10C4300090F8D20103287FD0E748807840B10020EF
:10C44000E5498870E34991F8A812480076F088FC25
:10C45000DE4890F8520000E07EE000F0070038B1BE
:10C46000DC4890ED900BB0EE001B20EE018B06E057
:10C47000D84890EDA40BB3EE041B20EE018B9FED8A
:10C48000D70BB4EEC08BF1EE10FA05D2B0EE000B74
:10C4900028EE000BB0EE408B9FEDD00BB4EEC08BBE
:10C4A000F1EE10FA03D29FEDCD0BB0EE408BCD48EC
:10C4B00090ED040B20EE080BBDEEC00B10EE104A01
:10C4C0000120FEF7EEFD08B9002006E7022027F064
:10C4D0002DF9022027F090F92046FFF70DF920B939
:10C4E0000020FEF7DEFD0020F7E66042FFF704F9CA
:10C4F00028B90020FEF7D5FD0020EEE61CE0BA4882
:10C50000007800F00400B0B1B24890ED2A0BB0EE14
:10C51000409BFEF71AFF50B9AE4880ED2A9B0020E1
:10C52000FEF7BFFD0720B14988700020D5E6A94875
:10C5300080ED2A9B00BF0CE0AD48007820F004009D
:10C54000AB4908700021AB4A11615161022027F00C
:10C5500053F90020FEF7A5FDFFF7B3FD08B9002051
:10C56000BBE6A548807880BB9A4890F8560202281E
:10C5700004D19F48007800F0040020B9954890F855
:10C580005602032822D10120FFF766FC002801DAB9
:10C590000020A2E69648007800F00400A8B18D487B
:10C5A00090F85602022811D18B48807868B9002093
:10C5B000FFF752FC002801DA00208EE60020FFF78A
:10C5C0004BFC002802DA002087E6FFE7FFF795F929
:10C5D000FEF7B4FDB5B18648007800F0040088B1DC
:10C5E0007C4890F8D20101280CD1811E022028F04D
:10C5F000B8FD824AD2E90E32181A62EB01027D4977
:10C60000C1E904027A48007800F0040058B17C487F
:10C61000007840F004007A4908706E4890F8A6024D
:10C620006D49887008E07648007820F0040074496D
:10C6300008700020684988700120FEF7CDF908B91C
:10C6400000204AE6FFF7B2FB08B9002045E6614842
:10C6500090F8E601801E06287DD2DFE800F0030492
:10C6600006073B3C00BF012037E600BF65488078E5
:10C6700010B16548807808B900202EE6634890ED37
:10C68000040B544880ED2A0B6148D0E90430614A1C
:10C69000D2E904125E1840EB020102220023304668
:10C6A000F4F76DF85C4AC2E9040100234FF480629C
:10C6B000194604204CF062FB0A210846FEF74AF9AD
:10C6C00008B9002009E60120FEF786F908B9002024
:10C6D00003E65EE000BF4B48807808B90020FCE527
:10C6E0004A4890ED040B3B4880ED2A0B4848D0E9BE
:10C6F0000421104678F0BEF941EC100B354890ED5E
:10C70000BC1AB7EEC11AB7EE082B31EE021B9FED33
:10C71000433B81EE032B334890ED041B22EE011BBB
:10C720001FEDD72B01EE420BB0EE408B51EC180BF6
:10C7300078F036FB384AC2E90401FF234FF48062E7
:10C74000002104204CF01AFB0A210846FEF702F9EA
:10C7500010B90020C1E51AE02D49D1E904012E4AA3
:10C76000C2E9040100234FF48062194604204CF012
:10C7700005FB0A210846FEF7EDF808B90020ACE5F4
:10C780000120FEF729F908B90020A6E501E0002004
:10C79000A3E500BF0120A0E52DE9F04F2DED088BAA
:10C7A00083B00446002002901048807810B91E2003
:10C7B0000E498870074890F8500200F0040088BBCA
:10C7C000012003B0BDEC088BBDE8F08F880300208A
:10C7D000A19B0424300605244C0500209A999999C0
:10C7E0009999A93F5801002488420030A69B04244F
:10C7F000B4050020B8050020844200300008002065
:10C8000070340024CE9A0424D29A0424809A0424FA
:10C81000D89A0424F89A0424E008002000000000BC
:10C8200000408F40FFE7F848007800F0040028B986
:10C83000002003B0BDEC088BBDE8F08FF34890F802
:10C840005602012801D00120F3E7F14890F8520088
:10C8500000F0300008B10120EBE70120ED498880AD
:10C86000EA4890ED080BEC4890ED041B20EE010B1C
:10C87000BDEEC00B10EE105AE44890ED9D0AB7EEE5
:10C88000C08AE648007800F0040030B1DF4890ED3F
:10C89000540AB7EEC00AB0EE408BDC4890ED540A63
:10C8A000B7EEC00AB4EEC80BF1EE10FA05D290ED67
:10C8B000540AB7EEC00AB0EE408BD44890ED360B68
:10C8C000B4EEC80BF1EE10FA03D290ED360BB0EED9
:10C8D000408BD348D0F81C010190DFF84893002C1E
:10C8E0001FDBCA4890F8ED0100F02000C8B9CE481F
:10C8F00090ED020AB5EEC00AF1EE10FA11DD90EDEE
:10C90000020AB7EEC00AC44890ED041B20EE010BEA
:10C91000BDEEC00B10EE101AC148D0F81C0101EB9F
:10C920000009BB4890F8480020F04000B84981F861
:10C930004800002C0ADBBD4890ED041B21EE081BCB
:10C94000B0EE410B022007F0C2FB0BE0B74890EDC0
:10C95000041BB1EE482B21EE021BB0EE410B02206E
:10C9600007F0B5FB00BF0A2076F0FAF9B04840792D
:10C9700004281DD1AA48D0F8F800C8B1A248007810
:10C9800000F00400A0B1A24890F84A0000F00400B2
:10C9900070B9002C02DBA748007A48B9002C02DAF3
:10C9A000A448807920B99E48D0F81C0148450EDB88
:10C9B0009848808848F20101084040B99848B0F88A
:10C9C000040120B90222114610464EF022F84FF021
:10C9D000FF320121022028F072FA0E4600BF00BF8C
:10C9E00000BFBFF34F8FBFF36F8F00BF00BF00BF0B
:10C9F000874890F8480000F0400000B9019684484C
:10CA000090F8480000F0400028B98248808800F083
:10CA100001000028A7D09FED880B022007F057FBEC
:10CA200032210A20FDF796FF08B9002001E7784877
:10CA300090F8480000F0400020B914208049887028
:10CA40000020F6E6724890F8480020F04000704957
:10CA500081F848007248D0F8F80020B903207849DE
:10CA600088700020E5E67748808800F00300012800
:10CA700002D1642076F074F96D484079042803D01F
:10CA800000206F498870D4E66F4901984861002002
:10CA900008615E4890ED900BB7EEC0AB9FED6B0A5E
:10CAA000B4EEC0AAF1EE10FA04DD9FED680AB0EE14
:10CAB00040AA0AE09FED660AB4EEC0AAF1EE10FAB1
:10CAC00003D29FED640AB0EE40AA6348D0ED020A9B
:10CAD000B0EE001A80EE810AB4EECA0AF1EE10FA46
:10CAE00007D290ED020AF0EE000A80EE201AB0EEB6
:10CAF00041AA55484169484890ED040BB7EECA1A5F
:10CB000020EE010BBDEEC00B10EE100A091A4E48C4
:10CB10004161002C28DD4248D0F81C0146194A48E2
:10CB20004069411948484161384880ED2A8B00230B
:10CB30004FF48062194604204CF020F932210A207B
:10CB4000FDF708FF08B9002073E63548D0F8F80073
:10CB500008B900206DE636484079042801D000204D
:10CB600067E63948466129E0002C27DA2C48D0F8DE
:10CB70001C01461B34484069411B3348416123482E
:10CB800080ED2A8B00234FF48062194604204CF07C
:10CB9000F5F832210A20FDF7DDFE08B9002048E64D
:10CBA0001F48D0F8F80008B9002042E62048407934
:10CBB000042801D000203CE623484661144890F840
:10CBC000520000F00400E8B1104890ED900B9FED8A
:10CBD000231B20EE019B9FED230BB4EEC09BF1EED7
:10CBE00010FA03D29FED1F0BB0EE409BB7EE000B87
:10CBF000B4EEC09BF1EE10FA3FDDB7EE000BB0EEE5
:10CC0000409B3AE032E00000B405002030060524E5
:10CC100088030020F005002058010024BA420030AB
:10CC2000200700200000F47E243500249801002411
:10CC300000060020B80200240000000000000000F0
:10CC4000A69B042450050020E00800200AD7A33C3E
:10CC50000AD7A33B6F12033B189B0424000000007B
:10CC60000088B34000000040E17A943FFE4890ED18
:10CC7000900B9FEDFE1B20EE019BB4EEC89BF1EEE6
:10CC800010FA01DDB0EE489BF74880ED2A9BF94889
:10CC9000007840F00400F749087000234FF48062E8
:10CCA000194604204CF06AF81EE00A2076F058F885
:10CCB000F1484079042808D1EE48007800F00400DB
:10CCC00018B1EE48D0F8F80070B9ED48808848F205
:10CCD0000101084040B9E948B0F8040120B9022236
:10CCE000114610464DF095FEE548808800F00100A1
:10CCF0000028DAD032210A20FDF72CFEDF48D0F8D8
:10CD0000F80008B9002094E5DE48808800F00300B0
:10CD1000012802D1642076F023F8D748407904280E
:10CD200001D0002085E5D348007800F0040018B158
:10CD30001520D549887068E14FF4806201210220F6
:10CD400028F0BDF8D14AC2E90401002C1FDD1046CD
:10CD50004069411910464161C34890ED901BCC4891
:10CD600090ED042B21EE021B9FEDCA2B21EE021B3E
:10CD7000B0EE410B51EC100B78F012F8C34BD3E935
:10CD8000042380185941C14AC2E9040106E0002C7D
:10CD900004DABE484069411BBC484161BF4890F875
:10CDA000520000F00400A0B1AF4890ED901BB848CD
:10CDB00090ED042B21EE021B9FEDB92B21EE021BFF
:10CDC000B0EE410B51EC100B77F0EAFF07468846B6
:10CDD0004EE0B548D0F828B0D0F838A0AF48B0F948
:10CDE0003800ABEB000BAD48B0F93A00AAEB000AF3
:10CDF000AA49B1F9441001FB0AF0C11700EB5151E7
:10CE00004FEAE12ABBF5004F02DB47F6FF7B04E067
:10CE10001BF5004F01DCDFF894B2BAF5004F02DBDE
:10CE200047F6FF7A04E01AF5004F01DCDFF87CA238
:10CE30000FFA8AF10FFA8BF0F6F78BFF00EE100A6B
:10CE4000B8EEC00B924890ED041B874890ED902BF4
:10CE500021EE021B20EE010B9FED951B20EE010B36
:10CE6000B0EE40BB51EC1B0B77F09AFF07468846AB
:10CE70007D4890F8520200F0040048B18348D0E9A0
:10CE80000410C91940EB0800804AC2E9041008E008
:10CE90007E48D0E90410C91B60EB08007B4AC2E958
:10CEA0000410714890ED540AB7EEC00A80ED2A0BC9
:10CEB00000234FF48062194604204BF05FFF3221BB
:10CEC0000A20FDF747FD08B90020B2E46B48D0F80E
:10CED000F80008B90020ACE467484079042801D084
:10CEE0000020A6E4744890ED040BB5EEC00BF1EE03
:10CEF00010FA3BD05C4890ED540AB7EEC00A80EDC2
:10CF00002A0B6D4890ED041B614890ED042B21EE37
:10CF1000021B9FED602B21EE021BB0EE410B51EC8A
:10CF2000100B77F03DFF554BE033D3E90E2380180B
:10CF30005941564AC2E9040100234FF48062194660
:10CF400004204BF01BFF32210A20FDF703FD08B936
:10CF500000206EE44948D0F8F80008B9002068E4E1
:10CF600045484079042801D0002062E44B4890F8FD
:10CF7000520000F0040058B13B4890ED900BB1EE28
:10CF8000001B80EE012BB7EEC20B80EDB80A19E052
:10CF9000354890ED900B9FED492B80EE021B90EDF4
:10CFA000B80AB7EEC00AB4EEC01BF1EE10FA09D20F
:10CFB00090ED900B9FED411B80EE012BB7EEC20B65
:10CFC00080EDB80A0520009000BF142075F0C8FE5F
:10CFD0002C48808800F00300012802D1642075F0FD
:10CFE000BFFE0098411EC9B200910028EDDC354813
:10CFF000007800F0040038B1284890F84A0000F0AA
:10D00000040008B90120029000BF1A48007820F0FF
:10D010000400184908700120FDF7DEFC029808B3EF
:10D020001648E030D0E90E21104677F023FD41ECA0
:10D03000100B254890ED042B9FED161B82EE013B53
:10D0400020EE030B214880ED040B90ED040BB1EEB4
:10D05000400B1F4880ED040B0B4880781E283BD105
:10D06000002037E038E00000300605240000000012
:10D07000006AA8404B050020000600202007002081
:10D08000F005002050050020A69B0424E0080020A5
:10D0900058010024000000000000F0418803002037
:10D0A000000000000000D041386904240180FFFF27
:10D0B000000000000000F040800A0524000000008D
:10D0C00000004040B405002078010024609B042447
:10D0D000D8000024FE498870FE4890ED040BFE48FD
:10D0E00080ED2A0BFD484079042801D000209DE402
:10D0F00002989BE470B52DED048BF8484079042824
:10D1000003D00020BDEC048B70BDF34890F85002B2
:10D1100000F0040020B91F20ED4988700020F1E7DD
:10D12000ED4890F85602012804D02020E849887084
:10D130000020E7E7E84890F8D201032804D1212035
:10D14000E34988700020DDE7E54890F8520000F0E0
:10D15000060020B92220DE4988700020D2E7E0488E
:10D1600090F84B0000F0040020B92320D8498870C3
:10D170000020C7E7DA4890F84A0000F0040020B128
:10D180002420D34988700020BCE70120D54988803D
:10D190009FEDD50BD64880ED040B0020D549888043
:10D1A0009FEDD10BD44880ED040B0020FDF714FC5B
:10D1B00008B90020A6E7D149D1E90E01D04AC2E959
:10D1C00004010024CF488078822802D0CE4880799C
:10D1D00008B1012408E0CB488078832802D0CA48EF
:10D1E000007A08B14FF0FF34C8480078C849097880
:10D1F000084000F0040000287DD100E000BFC548D1
:10D2000090F900000028F9DA0220C249087027F0DE
:10D2100093FB40B1B24890F84A0040F00400B04996
:10D2200081F84A0007E0AE4890F84A0020F0040078
:10D23000AB4981F84A00FF20B6490870A64890F82B
:10D24000500200F0040000287DD0A54890F84A0064
:10D2500000F00400002876D1A14890F85200002880
:10D260007ED09D4890F8D201032879D0AA488078D2
:10D2700040B10020A8498870974991F8A812480049
:10D2800075F06EFD964890F8520000F0070038B136
:10D29000914890ED900BB0EE001B20EE018B06E064
:10D2A0008D4890EDA40BB3EE041B20EE018B8A4851
:10D2B00090ED080B9FED991B20EE011B90ED102BBC
:10D2C00081EE020BB4EEC80BF1EE10FA0BDD90ED1F
:10D2D000080B9FED921B20EE010B90ED101B80EED2
:10D2E000012BB0EE428B7C4890ED080B9FED8D1B1F
:10D2F00020EE019B00E056E0B4EEC98BF1EE10FA8F
:10D3000001D2B0EE498B894890ED040B20EE080B5A
:10D31000BDEEC00B10EE105A0120FDF7C2FE08B999
:10D320000020EFE6022026F001FA022026F064FA3F
:10D33000002C09DB2846FEF7DFF928B90020FDF7AD
:10D34000B0FE0020DEE60BE0002C08DC6842FEF7B1
:10D35000D3F920B90020FDF7A4FE0020D2E60CE0AE
:10D360006A48007820F00400684908700021704A7B
:10D3700011615161022026F03FFA6448007800F004
:10D38000040068B14FF0FF31022027F0EAFE5B4A4B
:10D39000D2E90E32181A62EB01026549C1E90402B2
:10D3A0000020FDF77EFE5948007800F0040020B907
:10D3B0000B20474988700020A4E6FEF79EFAFDF78F
:10D3C00079FD2046FFF7E8F906465A48007820F034
:10D3D000040058490870FDF732FE0EB9002091E6AE
:10D3E000FEF78BFAFDF7AAFE4848007800F004002B
:10D3F00058B14748007840F0040045490870364865
:10D4000090F8A6024449887008E04148007820F06E
:10D4100004003F49087000203F4988700120FDF753
:10D42000DBFA08B900206DE6FEF7C0FC6AE670B5CD
:10D430002DED088B29484079042803D00020BDEC4D
:10D44000088B70BD0120274988809FED270B284855
:10D4500080ED040B0020274988809FED230B264890
:10D4600080ED040B0020FDF7B7FA08B90020E6E7CD
:10D470002248D0E90E10224AC2E90410164890ED65
:10D48000580AB7EEC0AAB7EE000BB4EEC0ABF1EE8F
:10D4900010FA03DDB7EE000BB0EE40AB0E4880EDA6
:10D4A0002AAB254890ED020AB7EEC00A1F4890ED5E
:10D4B000041B20EE010BBDEEC00B10EE101A0F483E
:10D4C000E038D0F81C0101441C484161002337E0DA
:10D4D000A69B0424809A042430060524000600201C
:10D4E00088030020F005002000000000000000007C
:10D4F00020020024800200244002002400080020B2
:10D50000809B0424A29B0424B8020024B4050020BC
:10D5100070340024A19B04244C050020FCA9F1D206
:10D520004D62603F7B14AE47E17A743F580100249E
:10D53000B80500204B050020189B0424E0080020BB
:10D540004FF48062194604204BF018FC0A2108466B
:10D55000FDF700FA08B9002071E70120FDF73CFA59
:10D5600008B900206BE70025FE4890F8D20180B191
:10D57000FC4890F8D20103280BD0FA4890F85002EA
:10D5800000F0040028B1F848007800F0040000B969
:10D590000125F44890F8D20130B1F448007800F049
:10D5A000040008B9002D7CD000E000BFF04890F9DD
:10D5B00000000028F9DA0220ED49087027F0BCF9D4
:10D5C00040B1EC4890F84A0040F00400E94981F885
:10D5D0004A0007E0E74890F84A0020F00400E549D7
:10D5E00081F84A00FF20E2490870DE4890F85002B6
:10D5F00000F00400002872D0DE4890F84A0000F0E5
:10D60000040000286BD1DB4890F852000028F2D0CB
:10D61000D44890F8D201032861D0D748807840B12F
:10D620000020D5498870CF4991F8A812480075F0BC
:10D6300097FBD04890F8520000F0070038B1C94875
:10D6400090ED900BB0EE001B20EE018B06E0C5487C
:10D6500090EDA40BB3EE041B20EE018BC14890EDBE
:10D66000080B1FED521B20EE011B90ED102B81EEDD
:10D67000020BB4EEC80BF1EE10FA0BDD90ED080BC7
:10D680001FED5A1B20EE010B90ED101B80EE012BBD
:10D69000B0EE428BB948807848B1B24890ED080BA3
:10D6A00000E075E01FED611B20EE019B01E09FEDA6
:10D6B000B49BB4EEC98BF1EE10FA01D2B0EE498BF7
:10D6C000B14890ED040B20EE080BBDEEC00B10EE40
:10D6D000104A0120FDF7E5FC10B90020AFE634E068
:10D6E000022026F023F8022026F086F82046FEF7D6
:10D6F00003F820B90020FDF7D4FC00209FE660422B
:10D70000FDF7FAFF20B90020FDF7CBFC002096E6DC
:10D710009648007800F00400B0B1924890ED2A0BD2
:10D72000B0EE40BBFDF711FE50B98E4880ED2ABB2C
:10D730000020FDF7B6FC07209449887000207EE6A3
:10D74000884880ED2ABB00BF0CE08748007820F0B5
:10D7500004008549087000208D4A10615061022044
:10D7600026F04AF88048007800F0040068B14FF0D5
:10D77000FF31022027F0F5FC864AD2E90E32181A52
:10D7800062EB01028249C1E904020020FDF789FC35
:10D79000FEF797FC08B9002051E67F48807880BBEF
:10D7A000704890F85602022804D16F48007800F0C3
:10D7B000040020B96B4890F85602032822D10120BA
:10D7C000FEF74AFB002801DA002038E666480078B8
:10D7D00000F00400A8B1634890F85602022811D165
:10D7E0006548807868B90020FEF736FB002801DA2A
:10D7F000002024E60020FEF72FFB002802DA00209C
:10D800001DE6FFE7574890F85602012829D15548F0
:10D8100090F8500200F0040018B3564890F85200F7
:10D8200000F00700E8B15048007800F0040020B98B
:10D830000B2056498870002001E6FEF75EF8FDF7E0
:10D8400039FB0020FEF7A8FF04465448007820F07A
:10D85000040052490870FDF7F2FB0CB90020EEE518
:10D8600000BFFEF74AF8FDF769FCB5B13E48007805
:10D8700000F0040088B13B4890F8D20101280CD197
:10D88000811E022027F06DFC424AD2E90E32181A9E
:10D8900062EB01023E49C1E904023348007800F01E
:10D8A000040058B13E48007840F004003C4908703C
:10D8B0002C4890F8A6023049887008E03848007873
:10D8C00020F004003649087000202B4988700120A0
:10D8D000FDF782F808B90020B1E5FEF767FAAEE57A
:10D8E00010B530484079042801D0002010BD012037
:10D8F0002D4988801B4890ED660B90ED601AB7EEBD
:10D90000C11A80EE012BB0EE000BB4EEC02BF1EE8D
:10D9100010FA06DD90ED5C0AB7EEC00A80ED2A0B26
:10D9200006E0104890ED600AB7EEC00A80ED2A0BC1
:10D930000C4890ED2A0B90ED361BB4EEC10BF1EEC6
:10D9400010FA03DD90ED360B80ED2A0B054890EDC3
:10D95000661B164890ED020AB7EEC00A31EE001BB6
:10D96000094825E030060524B4050020884200302F
:10D97000A19B0424880300204C050020A29B0424C2
:10D980009A9999999999A93F58010024A69B042432
:10D99000B805002000080020844200304B0500201C
:10D9A0007034002400060020F0050020189B042499
:10D9B00090ED042BFE4890ED470AB8EEC00B01EE47
:10D9C000420BBDEEC00BFB4880ED050A00234FF46F
:10D9D0008062194604204BF0D1F964210A20FCF73B
:10D9E000B9FF08B9002081E70120FDF75AFB28B1F3
:10D9F0000220F9F79AF90020FDF753FB0021EE4AC7
:10DA000011615161ED4890F8CA0128BBE849E03145
:10DA1000D1E90E01EA4AC2E90401E549E031D1E960
:10DA20000E01E84AC2E90401E148E030D0E90E10F5
:10DA3000E54AC2E90410E548007800F0040058B156
:10DA4000E048D0E90420E249D1E90431D21A60EB80
:10DA50000100D949C1E904200120FCF7BDFF0120E4
:10DA600044E700BF002076F027FADA48407900F05A
:10DA7000080010B10421D74841710020D6498870B0
:10DA8000D6498870D64A10615061D64A10615061FB
:10DA9000D54988704524C648D0F8F80008B9542400
:10DAA00068E1CC48407900F0020008B1452461E10A
:10DAB000C848007900F0010000287CD0FDF792F8FA
:10DAC000CA48007800F0040048B1C94890F85200F4
:10DAD00000F0060018B1FFF70DFB05460BE0B74854
:10DAE00090F8E601012803DCFFF7A1FC054602E0FF
:10DAF000FEF7EAFB05460020FDF7D3FABD480078A3
:10DB000020F00400BB490870BB48007820F00400F6
:10DB1000B9490870B548007820F00400B34908708E
:10DB2000FDF790F93224B548808800F0010088B9EB
:10DB300001219F48A0F8041104E0601EC4B20A202D
:10DB400075F00EF9AD48808800F0010008B9002C8E
:10DB5000F3D1002585B3AA48007800F0040058B33B
:10DB6000A84890ED000AB5EEC00AF1EE10FA2CD0EC
:10DB7000A54890ED041BA34890ED000AB7EEC00A3B
:10DB800021EE000BBDEEC00B10EE101A8848D0F845
:10DB90001C0101448748416100234FF4806219460B
:10DBA00004204BF0EBF864210A20FCF7D3FE00B907
:10DBB00000257F4801E098E007E0D0F81C117D487F
:10DBC0004069814238D0002536E0ADB38C480078FA
:10DBD00000F0400080B38B4890ED080AB5EEC00A13
:10DBE000F1EE10FA28D0884890ED041B854890ED9E
:10DBF000080AB7EEC00A21EE000BBDEEC00B10EE16
:10DC0000101A6B48D0F81C0101446A484161002396
:10DC10004FF48062194604204BF0B0F864210A20CA
:10DC2000FCF798FE00B900256148D0F81C11614846
:10DC30004069814200D000257148007820F04400FE
:10DC40006F4908708DB16348407904280DD16F4841
:10DC5000807810B901206D4988705C48007840F0E8
:10DC600004005A490870412419E05148D0F8F800DE
:10DC700018B90320654988700DE05648407902289C
:10DC800003D105206149887005E06048807810B9AB
:10DC900002205E498870452402214E484171544853
:10DCA00090F8520000F0070028B15948007820F0A1
:10DCB0000400574908703EF001F9022075F050F851
:10DCC0005448806810B10A2075F04AF802204CF0E0
:10DCD00055FF18B9002102203FF024FF4E488079FB
:10DCE00010B10E204D49888044E03A48007900F098
:10DCF0000200E8B3FCF776FFFFF7F2FD0546FDF7FB
:10DD0000A1F85DB133484079042807D12F48407805
:10DD100040F004002D49487044241AE0322437486A
:10DD2000808800F0010080B901212148A0F8041189
:10DD300004E0601EC4B20A2075F012F82F488088F3
:10DD400000F0010008B9002CF3D14524022121483C
:10DD5000417102204CF012FF18B9002102203FF05F
:10DD6000E1FE2D48007A10B10E202C49888001E098
:10DD7000FFE70024D4B10E48D0F8F80020B9412CB8
:10DD800002D0442C00D054240020FDF78AF9244806
:10DD9000007860B90648B0F8040140B1174880889F
:10DDA00000F0010018B1002101483BE04EE03BE0EB
:10DDB00020070020E0080020483500243006052414
:10DDC00080060020C006002000070020A40B0020D1
:10DDD000A006002000060020CE9A0424D29A042433
:10DDE000D89A0424F89A0424CA9A0424BA42003027
:10DDF00088030020C80C00204B050020F0050020FF
:10DE000000430030C042003058010024A69B042487
:10DE1000B5050020C00D0020B8020024C800002471
:10DE2000AF0D0020A0F804110020094988700948AE
:10DE3000847000BF00BF00BFBFF34F8FBFF36F8F71
:10DE400000BF00BF00BF0121034841710AE6000086
:10DE500084420030AC9B04240006002008B576F014
:10DE6000F9FB009000BFFE4890F8A802012803DAF1
:10DE70000120FB4981F8A802F94890F8A8126846E9
:10DE800075F0E2FEF748807D032802DAF548807DD0
:10DE900000E00320441EF1E30120A040C7B20020AF
:10DEA000F1490855F1480078384010B9012008556B
:10DEB00046E0EF48005D18B90220EB4908553FE005
:10DEC000EC488078384018B91020E749085537E009
:10DED000E848C07818B12020E349085530E0E6480A
:10DEE0000057002803DC4020DF49085528E0E348BC
:10DEF00090F84A00384018B10120DB4908551FE06E
:10DF0000C4EBC400DE4901EB0010008C18B980207E
:10DF1000D549085514E0DB48007848B1DA4830F8B4
:10DF2000140000F0010018B10820CF49085507E09F
:10DF3000D648007800F0200010B10120CA490855E9
:10DF4000D348006800F0020010B10420C64908550B
:10DF5000C548005D88B30021CE4A02EBC4021160BF
:10DF600051600020CC4921F81400CC4921F814005C
:10DF7000C1480057002806DC002004EBC401C84A51
:10DF800002EB8101C861B848005D00F08800A8B1CB
:10DF9000E0B2C44926F016FEC34A03C2C248D0E923
:10DFA0000032C048D0E90010C91A60EB0200BF4A35
:10DFB00002EBC402C2E90010F3E306E00021BB4A11
:10DFC00002EBC40211605160F6E7B94800EBC400EF
:10DFD00090ED000BB74880ED000B4FF40075E0B2F8
:10DFE000B04926F0EFFDB04A03C2AF4806C8AD48BD
:10DFF000D0E90030591A60EB0200AC4A02EBC402CF
:10E00000C2E90010A94800EBC400D0F80480B8F1C0
:10E01000000001DB014600E041420E46A24903C96F
:10E02000A54A03C294490831095D002917DDC4EBF4
:10E03000C401934A02EB0111C86AC11700EB917148
:10E040008910B1420BDC0020064680460021974A29
:10E0500002EBC4021160516045F0040530E09748BE
:10E0600000EB840090ED000AB7EEC00A914890EDF5
:10E07000001B20EE010BBDEEC00B10EE100AB042EB
:10E0800001DB45F002057D4890F84A00384010B1A8
:10E0900045F0800514E08948103800EB840090EDCD
:10E0A000000AB7EEC00A834890ED001B20EE010B7A
:10E0B000BDEEC00B10EE100AB04201DB45F00405C6
:10E0C0006D480830005D20B16B480830005D0428C1
:10E0D00018D104EB44007A49085C30B145F01005D2
:10E0E000B8F1000F01DA45F0400504EB4400744933
:10E0F0000844807830B145F02005B8F1000F01DD0B
:10E1000045F04005C4EBC4005D4901EB0010D0E9C7
:10E110001210002359405840014301D045F4807546
:10E12000C4EBC400564901EB0010B0F926000028EA
:10E1300075DD644800783840002870D005F0C000D4
:10E1400000286CD1594901EBC40206CA564B06C3DC
:10E1500055494968B1F5002F03DB5B49524A5160CC
:10E1600008E05149496811F5002F03DC564949423E
:10E170004D4A516005F4807181B14B49D1E900C32A
:10E180004E491C39095D0022ACFB01AB03FB01B118
:10E190000CFB0211444AC2E900A10FE04249D1E957
:10E1A000003C46491839095D0022A3FB01AB0CFB7A
:10E1B00001B103FB02113C4AC2E900A13A4A06CA76
:10E1C000090F41EA0210354931F8141001F001013C
:10E1D00031B900213D4A42F824103D4941F824005C
:10E1E0003C4901EB4401497801F0C80109B945F007
:10E1F0000105374951F82410A1EB000805F481719D
:10E2000002290DD1324A52F82420111801EBD172A3
:10E210005210D317DFF890C0CCE9002303E034E1BB
:10E22000C117214A03C2002804DD294951F82410EE
:10E23000002906DC002877DA254951F82410002946
:10E2400072DA05F4807119B1014600EBD1725010F9
:10E25000154AD2E900C11CEB000341EBE0713BE041
:10E26000300605244000002498050020B405002055
:10E270004C050020B40200244C070524880300202C
:10E2800020070020AF0D0020F0050020C80000246A
:10E29000E00C0020780500209C050020500500209F
:10E2A000D009002020000024280000245805002068
:10E2B00058010024380000243000002408090524F7
:10E2C000B8020024B0020024FFFF07000C00002465
:10E2D0000000002400060020C2E90031FD4951F889
:10E2E00024100144FB4A42F82410FB4B53F824103D
:10E2F000021E01DB134600E05342002901DB8C467D
:10E3000001E0C1F1000C634508DBF449D1E90031BB
:10E310001B1841EBE071F14AC2E900314FEA4801B4
:10E32000021E02DB134601E019E05342002901DB23
:10E330008C4601E0C1F1000C63451ADDE749D1E9E3
:10E3400000311B1841EBE071E44AC2E90031E149B8
:10E3500051F824100144DF4A42F8241009E0DE4A53
:10E3600052F8241001EBD172A0EB6202D94B43F8B2
:10E37000242000280EDDD74951F8241000EB40027C
:10E380005200914206DD00EB40014900D14A42F8BB
:10E3900024100FE000280DDACE4951F8241000EBCC
:10E3A00040025200914205DA00EB40014900C94A9F
:10E3B00042F8241005F4807149B1C64A52F824107D
:10E3C000CA1701EB92729210C24B43F82420C34942
:10E3D000D1E900C2BF4951F82410CB171CEB010151
:10E3E0005A41BE4B06C3BC4941F82400BB49D1E9A0
:10E3F0000021C90241EA5251D202083BC3E900217F
:10E40000B749095D04291ED1B64A02EBC40292ED58
:10E41000000BB54A92ED001B20EE010BBDEEC00BC8
:10E4200010EE101ACA1701EB9272B6EBA20F2BDA9C
:10E4300000221A605A60A74951F824108910A54A91
:10E4400042F8241020E0A649095D01F04001D9B14D
:10E45000A449503101EBC40191ED000BA24991EDAB
:10E46000001B20EE010BBDEEC00B10EE101AB142E6
:10E470000ADD0022994B1A605A60964951F824101F
:10E480008910944A42F8241000BF9848808B00F409
:10E490000070002873D0022C71D195488088B0F5A7
:10E4A000807F1ED193488078D8B1934890ED080BB7
:10E4B0008D4890ED001B20EE010BB0EE081B80EEA6
:10E4C000012BBDEEC20B10EE100AB04209DA8B49E7
:10E4D00003C98B4AC2E904018A48C06D401C8949BE
:10E4E00088668348808801286ED17D48503890F82E
:10E4F0004A1085480078884300F00400F0B37D4856
:10E500008078D8B381488088C0BB774890ED000BF5
:10E510009FED7F1B20EE010BBDEEC00B10EE100A2D
:10E52000B04251DA7448B0F8140118B901217248A8
:10E53000A0F814117048B0F914017749B1F900102E
:10E54000884204DD6C48B0F8140173490880012149
:10E550006948A0F814117148A0F80011704880793A
:10E5600048B16648D0E900316C48D0F81C01C217A8
:10E57000181A91410FDB6A48007A01E024E033E089
:10E5800080B16648D0F81C01C1175C4AD2E900325C
:10E59000C01A914106DA6148E030D0E90E10574ABE
:10E5A000C2E900105548D0E900105C4AE032C2E9E7
:10E5B0000E1000225948E030026442640021594A9A
:10E5C0001161516100260FE04B48B0F91401012898
:10E5D0000ADC5148B0F90000012805DD4E48B0F9C9
:10E5E00000104548A0F814114FF40069C4EBC400B2
:10E5F0004A4901EB0010B0F92000642801DA4FF419
:10E60000806905F0300010B14FF04009C0E005F01E
:10E61000040090BB33489430005D062858D2DFE8F0
:10E6200000F00304070C1032B1E04FF04009AEE0F7
:10E6300000202A4A10605060A9E000202D490855AA
:10E64000A5E02A48007E40F0040028490876012011
:10E650003549087060B235490870E0B2002126F0F3
:10E66000B1FA334A03C2334800EBC40040680028C3
:10E6700005DAFF203049087004E089E04EE101200E
:10E680002D49087083E000201A490870487088708E
:10E69000C8702A48807800F00F00C0B12848008870
:10E6A000B8B926488078A0B10120A040244908804C
:10E6B0000B48503890F84A000121A140084040B171
:10E6C0000748503890F84A001D4909883AE05CE054
:10E6D0005CE03BE00C000024000000242800002443
:10E6E000D8030020600805243800002440000024DE
:10E6F000F00500204C0500203006052430000024E1
:10E70000E0080020D0090020B40500200006002009
:10E710007B14AE47E17A743F1800002420070020E4
:10E72000B802002478050020AF0D002090EC0424EE
:10E7300088EC04245805002091EC0424B402002441
:10E74000D80B002041EA0010F8490880F84880788A
:10E7500000F0070018B14FF46040F649088060B23D
:10E76000F5490870E0B2002126F02CFAF34A03C202
:10E77000F34800EBC4004068002803DAFF20F149A9
:10E78000087002E00120EF49087000E000BF00BF00
:10E7900005F0010008B3EC494868002802DB014697
:10E7A00001E0B9E0414249450EDDE74840680028F4
:10E7B00003DBE548C0F8049003E0C9F10000E2493A
:10E7C00048600020E0490860DF48D0E90010DF4AD7
:10E7D00002EBC402C2E900100FE0DC4901EBC40106
:10E7E0004868C11700EB91718910D84A02EBC40246
:10E7F00051600020D54941F83400D54830F8140064
:10E8000000F4E060F0B305F00200D8BB04EBC400F4
:10E81000D04901EB8000006A04EBC401CD4A02EB51
:10E8200081014969884238D904EBC400114601EBE3
:10E830008000016AC84830F81400084404EBC401A1
:10E8400002EB8101C861C4EBC400C44901EB0010B4
:10E85000B0F92010C24830F9140081423ADDC4EB0F
:10E86000C400BE4901EB0010B0F92000322831DDB0
:10E87000BB48103850F8240060BBC4EBC40001EB67
:10E88000001000E009E0008C401E00B2C4EBC4019F
:10E89000B24A02EB011108841CE0C4EBC400AF498A
:10E8A00001EB0010B0F92600012813DDC4EBC40011
:10E8B00001EB0010B0F92600B0F51C7F0ADC05F46E
:10E8C000817038B940F27120C4EBC401A34A02EB55
:10E8D0000111C884C4EBC400A04901EB0010B0F9D9
:10E8E0002600002814DD9F4830F9140000280FDDB1
:10E8F00005F4817002280BD09B4850F824000028B2
:10E9000006DD954830F8140000B2964921F814004D
:10E91000964921F8145000BF601E04B2002CBFF6C7
:10E92000BBAAFFF7A0BA2DE9F0412DED028BB0EEA6
:10E93000408A04460F461646BDEEC80A10EE105A2D
:10E94000C4EBC400854901EB0010D0F83C8025B928
:10E950000120BDEC028BBDE8F08104EB440084494A
:10E960000844807828B1002D03DD022E01D000205C
:10E97000EFE704EB44007E49085C28B1002D03DA80
:10E98000012E01D00020E4E74FB1FF20794981F842
:10E99000FC0024F014FF60B2764981F8FC0008EB1B
:10E9A0000500754901EBC40148600121A140C8B2CE
:10E9B00000234FF4806219464AF0E0F902E00A2091
:10E9C00074F0CEF9624830F8140000F0010000281D
:10E9D000F5D0684890F9FC00A04208D1FF206549B5
:10E9E00081F8FC00204624F063FF24F0E8FE04EBED
:10E9F00044005F490844807828B1002D03DD022ED1
:10EA000001D00020A5E704EB44005949085C28B177
:10EA1000002D03DA012E01D000209AE7012098E7AB
:10EA20002DE9F05F2DED048B04460120A040C7B214
:10EA30005248807D032802DA5048807D00E00320A0
:10EA4000A04203DCBDEC048BBDE8F09F4C4890F87D
:10EA50005002384000B9F5E74148C030005D042855
:10EA600000D1EFE73E48C030005D052800D1E9E75E
:10EA700000E000BF434890F900000028F9DA60B2D6
:10EA800040490870204625F057FF38B1394890F8C2
:10EA90004A003843374981F84A0006E0354890F883
:10EAA0004A00B843334981F84A00FF2035490870CD
:10EAB000304890F84A00384000B1C3E72D48503044
:10EAC000005D00F0300078BB4FF0FF31204626F0AB
:10EAD00048FB024608460023514263EB00002A4AE5
:10EAE00002EBC402C2E900101D48C030005D0328DB
:10EAF00019D1204890F84A003840A0B9204890F831
:10EB00005002384078B1002020490855204800784C
:10EB1000B8431F4908701F48007838431D490870E2
:10EB20000F201D4908708DE738E00000D80B002049
:10EB3000B40200241A1C025890EC042488EC04242B
:10EB40005805002091EC04242800002478050020BA
:10EB5000F0050020D0090020E0080524200700204F
:10EB6000400705249C050020A40500205005002036
:10EB7000B802002488030020E008002040000024A0
:10EB800030060524A19B0424B80500204C05002074
:10EB900070340024B40500206CA70024FE480078DF
:10EBA000384038B9FC4800783843FB4908700120E8
:10EBB00074F0D6F8F948005D00F00700E8B3F848B3
:10EBC00000EBC40090ED010AB8EEC00BF54880EDF3
:10EBD000000B012074F0C4F8F14800EBC40090ED84
:10EBE000010AB8EEC00BEF4890ED001B30EE010BB0
:10EBF00080ED000B4FF0FF31204626F0B2FA0022E4
:10EC0000434262EB0100E849C1E90030E44800EB0F
:10EC1000C40090ED010AB8EEC00BE24890ED001B75
:10EC200030EE010B80ED000B012074F099F8DC4808
:10EC300000EBC40090ED010A00E00EE0B8EEC00B5E
:10EC4000D84890ED001B30EE010B80ED000BD24850
:10EC50000078B843D049087040E0D14800EBC400C8
:10EC600090ED010AB8EEC00BCE4880ED000B0120FC
:10EC700074F076F8CA4800EBC40090ED010AB8EED3
:10EC8000C00BC84890ED001B30EE010B80ED000B6F
:10EC9000012074F065F8C24800EBC40090ED010A51
:10ECA000B8EEC00BBF4890ED001B30EE010B80EDBD
:10ECB000000B012074F054F8B94800EBC40090ED4B
:10ECC000010AB8EEC00BB74890ED001B30EE010B07
:10ECD00080ED000B0021B44A11605160B14890ED05
:10ECE000000BB1EE001B80EE012B80ED002B4FF0EE
:10ECF000000BD9469FEDAD8BAE48005DC0EBC00167
:10ED0000AC481A3000EB01105030005D48B3A94800
:10ED1000005D00EB400101EBC001A74800EB811052
:10ED2000E03004EB440100EB4118B8F800004FEA72
:10ED3000004BA048005D00EB400101EBC0019E4884
:10ED400000EB811000F5187004EB440100EBC10AE0
:10ED5000BAF8049009F0010018B19AED020BB0EE78
:10ED6000408B9648005D01282FD19548006800F03F
:10ED7000004050BB0021934A116051608748005DFC
:10ED800000F00700002879D18C48B03000EBC400B7
:10ED900090ED001B834890ED002BB1EE422B21EE4D
:10EDA000021B894800EBC40090ED002B21EE021BF2
:10EDB0009FED862B21EE021BB0EE410B51EC100BA8
:10EDC00075F0EEFF784A03C258E07C48B03000EBA3
:10EDD000C40090ED002B734890ED003BB0EE481B53
:10EDE00013EE021B784800EBC40090ED002B21EEDF
:10EDF000021B9FED762B21EE021BB0EE410B51EC76
:10EE0000100B75F0CDFF6F4A03C26448005D00F03F
:10EE10000700C8B96C4800EBC40090ED001B21EE60
:10EE2000081B9FED6A2B21EE021BB0EE410B51EC4B
:10EE3000100B75F0B5FF5C4AD2E90032181A62EB8C
:10EE40000102594905C109E05748D0E900105D4B5E
:10EE50000CCB89185841544AC2E900105D4890F81B
:10EE600052020121A140084040B1564806C8002086
:10EE7000494260EB0200534AC2E900105048006862
:10EE800040F001004E49086000BF00BF00BFBFF363
:10EE90004F8FBFF36F8F00BF00BF00BF4248D0E964
:10EEA00000104D4A02EBC402C2E90010C4EBC400DA
:10EEB0004A4901EB0010D0E91012C4EBC400474BE3
:10EEC00003EB0010D0E90E503E4BD3E9006CAB1BB6
:10EED00060EB0C000D461146EA184141C4EBC4003A
:10EEE0003E4B03EB0010C0E910213648D0E900107A
:10EEF000C4EBC40203EB0212C2E90E1000BF00BF54
:10EF000000BFBFF34F8FBFF36F8F00BF00BF00BFC5
:10EF10002B48006820F0010029490860274808387C
:10EF2000005D00287ED10BF4801000287AD009F013
:10EF30000100002876D098ED050AB5EEC00AF1EE82
:10EF400010FA6FDD1D48005D03286BD01B48005D83
:10EF500001287ED11948B03000EBC40090ED001BB1
:10EF6000104890ED002BB0EE480B12EE010BB0EE06
:10EF7000409B154800EBC40090ED001BB1EE492BFF
:10EF800021EE021B9FED112B21EE021BB0EE410B77
:10EF900051EC100B24E00000B5050020D803002040
:10EFA000D80500200800002010000020000000000C
:10EFB000000000000E430030E84400300008052443
:10EFC000E00C002018000020580100240000000080
:10EFD0000000F04130060524B8050020200700207D
:10EFE00075F0DEFE05460E46FD4800EBC40060C02D
:10EFF000FC4800EBC40060C0FB4800EBC40260C2E8
:10F0000098ED051AB7EEC11A31EE491BF74800EB2F
:10F01000C40090ED002B21EE021B1FED142B21EEFE
:10F02000021B01E053E014E0B0EE410B51EC100B79
:10F0300075F0B6FE05460E46ED4800EBC40060C014
:10F04000EC4800EBC40060C0EB4800EBC40260C2B7
:10F0500033E098ED051AB7EEC11AE44800EBC4009E
:10F0600090ED002B21EE021B1FED282B21EE021B41
:10F07000B0EE410B51EC100B75F092FE05460E46BA
:10F080000021D74A02EBC402116051600020D54A2A
:10F0900002EBC40210605060D54A02EBC40260C2A9
:10F0A000D44A02EBC40260C2CF4A02EBC402116030
:10F0B0005160D14A02EBC40260C2D04800783843A4
:10F0C000CE490870084640783843487000BFCC48A5
:10F0D000005D032819D1CB4890F84A003840A0B908
:10F0E000C94890F85002384078B10020C749085507
:10F0F000C7480078B843C6490870C6480078384306
:10F10000C44908700F20C449087000BF9AE42DE973
:10F11000F04F2DED0C8B83B00446032C04DD03B0BF
:10F12000BDEC0C8BBDE8F08F0120A040C5B2B94802
:10F130000078A843B7490870B848807D032802DAF0
:10F14000B648807D00E00320A04200DCE7E7AE483F
:10F1500090F850020121A140084000B9DFE7A9481A
:10F160005030005D00B9DAE7A548005D042800D101
:10F17000D5E7A348005D052800D1D0E7A048005D91
:10F18000032805D09E48B4380057002800DCC6E7A5
:10F190009B48005D032809D098480178A048007872
:10F1A00088430121A140084000B1B8E700E000BF5A
:10F1B0009C4890F900000028F9DA60B2994908707B
:10F1C000204625F0B9FB38B18E4890F84A00284314
:10F1D0008C4981F84A0006E08A4890F84A00A84322
:10F1E000884981F84A00FF208E490870854890F8C8
:10F1F0004A00284000B192E78148005D03282CD1E5
:10F20000804890F84B00284030B37E485030005D75
:10F2100000F0010000BB0021834A02EBC402116030
:10F22000516000207949085579480078A843784909
:10F230000870784800782843764908704FF0FF310D
:10F24000204625F08EFF0022434262EB0100764902
:10F2500001EBC401C1E9003061E76948C03830F80A
:10F260001400724921F814006548B838005D7049EF
:10F2700008556348AC38005D6E4908556E48005D1E
:10F280006E49085500215E48AC3801556A48015561
:10F290006421A0F5777020F8141000210830015582
:10F2A000624830F81400642802DA0A2073F058FD2E
:10F2B000204624F03BFA0020029052485030005D76
:10F2C00000F0010008B10120029000204F490855CC
:10F2D0004D48983000EBC40090ED000BB0EE40CBF1
:10F2E000204625F0D1FBB7EEC00A4748983000EB26
:10F2F000C40080ED000B04EB44005149085C30B1C0
:10F3000004EB44000844807808B901260CE004EBC3
:10F3100044004B490844807828B104EB4400085C61
:10F3200008B9022600E0002636485030005D00F0A3
:10F330003000E8B340489C3800EBC40090ED000B6F
:10F34000B5EEC00BF1EE10FA32D03E4800EB84006F
:10F3500090ED000AB5EEC00AF1EE10FA7EDD012153
:10F36000204625F0FEFE074675F084FB41EC100BAD
:10F37000354800EBC40090ED001B20EE010B1FEDA3
:10F38000ED1B80EE01AB204890F8ED0162000121F9
:10F390009140084058B928489C3800EBC40090EDD3
:10F3A000000BB4EECA0BF1EE10FA00DB012600E010
:10F3B00015E0154890F8ED016200022191400840E7
:10F3C00068B91D489C3800EBC40090ED001B1D4837
:10F3D00000EB840090ED000AB7EEC00A36E03DE095
:10F3E00060060020A0060020E0060020580100244E
:10F3F00080060020C006002000070020A40B00208B
:10F400000008052488030020300605244C05002050
:10F4100070340024B40500206CA7002440000024B0
:10F42000BC0D0020A19B0424B8050020A89A042448
:10F43000A49A0424789A04241C0B05247C9A04249E
:10F44000B8020024243500247801002431EE000B9A
:10F45000B4EECA0BF1EE10FA00D80226F94890F883
:10F460002C0100F0020020B10420F74901EB440117
:10F4700048700298002878D1F448005D00F0070039
:10F4800038B1F34800EBC40090ED000BB0EE408BB8
:10F4900009E0EF48503000EBC40090ED000BB2EEF5
:10F4A000041B20EE018B9FEDEB0BB4EEC08BF1EE55
:10F4B00010FA03D29FEDE70BB0EE408BE348005DFE
:10F4C00000F0070010B14FF002090FE0E0485030A3
:10F4D00000EBC40090ED000BB0EE001B20EE010B22
:10F4E00088EE001BBDEEC10B10EE109AD54810300F
:10F4F00000EBC40090ED000B9FEDD81B20EE011B2C
:10F50000D048303000EBC40090ED002B81EE020BB0
:10F51000B4EEC80BF1EE10FA13DDCA48103000EB60
:10F52000C40090ED000B9FEDCD1B20EE010BC548F4
:10F53000303000EBC40090ED001B80EE012BB0EEEC
:10F54000428BC84800EBC40090ED000BB7EE041BE3
:10F5500020EE010B20EE080BB0EE408B022E05D101
:10F56000B1EE480BB0EE408B0DE0D0E0012E0AD09A
:10F57000B44890F851020121A140084018B1B1EE01
:10F58000480BB0EE408B4FF00008002700BFAF489B
:10F59000683050F824A09FEDB40BB0EE409B4FF0C4
:10F5A000FF320021204625F08AFCCDE9000175F0EC
:10F5B00061FA41EC100B39EE400BB0EE409B01209C
:10F5C00073F0CEFB4FF0FF320021204625F077FC90
:10F5D000CDE9000175F04EFA41EC100B39EE400B0D
:10F5E000B0EE409B324600212046B7EEC80BFFF735
:10F5F0009AF91E2073F0B4FB4FF0FF320021204631
:10F6000025F05DFCCDE9000175F034FA41EC100BFA
:10F6100030EE090BB0EE409B012073F0A1FB4FF0E0
:10F62000FF320021204625F04AFCCDE9000175F0AB
:10F6300021FA41EC100B30EE090BB0EE409B8348F1
:10F64000683050F82400AAEB000ABAF1000001DB90
:10F65000014600E04142494512DB29EE080BB5EEB8
:10F66000C00BF1EE10FA02DD781C07B208E029EEBB
:10F67000080BB5EEC00BF1EE10FA01D2781E07B2FE
:10F68000B1EE480BB0EE408B08F101000FFA80F8A4
:10F69000B8F1060F0CDA381E01DB014600E04142EA
:10F6A0000329FFF674AF08F0010100297FF46FAF62
:10F6B00017F1020F07DA634890F852026840614977
:10F6C00081F852020AE0022F08DA6048503890F8B8
:10F6D0004A0028435D49503981F84A00381E01DB51
:10F6E000014600E04142022910DB5849503991F8A7
:10F6F0004A10294051B95549503991F84B102940C9
:10F7000021B15B480078284359490870FCE1504812
:10F7100000EBC40090ED001B9FED560BB0EE002BEC
:10F72000B0EE408B02EE018B9FED4A0BB4EEC08B26
:10F73000F1EE10FA05D2B0EE000B28EE000BB0EEA1
:10F74000408B9FED440BB4EEC08BF1EE10FA03D268
:10F750009FED400BB0EE408B424800EBC40090EDB3
:10F76000000B20EE080BB0EE408B022E04D1B1EE60
:10F77000480BB0EE408B0CE0012E0AD0314890F8D7
:10F7800051020121A140084018B1B1EE480BB0EE82
:10F79000408BC4EBC400394901EB0010D0E90E786E
:10F7A0004FF0020B00BF2948503890F84A00A84398
:10F7B0002649503981F84A00FF2081F8FC00204694
:10F7C00024F01AF89FED280BB0EE409B4FF0FF326B
:10F7D0000021204625F073FBCDE9000175F04AF9C0
:10F7E00041EC100B39EE400BB0EE409B012073F062
:10F7F000B7FA4FF0FF320021204625F060FBCDE93B
:10F80000000175F037F941EC100B39EE400BB0EE0A
:10F81000409B32462046B7EEC80B0299FFF783F8AB
:10F8200010B14FF0000B42E0154800EBC400C0E9F6
:10F83000007800234FF480621946284649F09EFA6A
:10F8400023E000003006052400060020D803002035
:10F85000600805249A9999999999A93FFCA9F1D230
:10F860004D62603F580100240000000000000000CD
:10F87000B40500207B14AE47E17A843F20070020C6
:10F88000E00800200A2073F06BFAFE4830F81400FC
:10F8900000F001000028F5D0B1EE480BB0EE408B2F
:10F8A000ABF1010000F0FF0B0EB186F003066420FF
:10F8B00073F056FA4FF0FF320021204625F0FFFA90
:10F8C000CDE9000175F0D6F841EC100B30EE090BD4
:10F8D000B0EE409B012073F043FA4FF0FF3200215D
:10F8E000204625F0ECFACDE9000175F0C3F841ECB3
:10F8F000100B30EE090BB0EE409BBBF1000F7FF414
:10F9000052AFE14800EBC40090ED000B20EE090B74
:10F910009FEDDE1B80EE012BB0EE42ABDD4890F890
:10F920004B002840F0B3DB4890F84A002840C8BBA1
:10F93000B0EECA0BD44800EBC40090ED001B21EEE2
:10F94000081BB0EE002B21EE021BB0EEC11BB4EE83
:10F95000C10BF1EE10FA28D8B0EECA0BCA4800EB82
:10F96000C40090ED001B21EE081BB6EE002B21EE2B
:10F97000021BB0EEC11BB4EEC10BF1EE10FA14DBAA
:10F9800029EE080BB5EEC00BF1EE10FA06D2C24814
:10F9900090F852026840C04981F85202BF4800788E
:10F9A000284300E001E0BD490870B1EE480BB0EE1D
:10F9B000408B1FED530BB0EE409B4FF0FF32002108
:10F9C000204625F07CFACDE9000175F053F841ECB2
:10F9D000100B39EE400BB0EE409B012073F0C0F9E4
:10F9E0004FF0FF320021204625F069FACDE90001F1
:10F9F00075F040F841EC100B39EE400BB0EE409B37
:10FA000032462046B7EEC80B0299FEF78CFF642001
:10FA100073F0A6F94FF0FF320021204625F04FFA8F
:10FA2000CDE9000175F026F841EC100B30EE090B22
:10FA3000B0EE409B012073F093F94FF0FF320021AC
:10FA4000204625F03CFACDE9000175F013F841ECB1
:10FA5000100B30EE090BB0EE409B8B4800EBC4005E
:10FA600090ED000B20EE090B9FED881B80EE01ABA3
:10FA7000884890F84B002840E8B3864890F84A0040
:10FA80002840C0BBB0EECA0B7F4800EBC40090ED2D
:10FA9000001B21EE081BB0EE002B21EE021BB0EE86
:10FAA000C11BB4EEC10BF1EE10FA2CD8B0EECA0BAC
:10FAB000754800EBC40090ED001B21EE081BB6EE6C
:10FAC000002B21EE021BB0EEC11BB4EEC10BF1EE18
:10FAD00010FA18DB71480078284060B929EE080B4D
:10FAE000B5EEC00BF1EE10FA08D26B4890F8520256
:10FAF0006840694900E006E081F8520267480078F2
:10FB000028436649087000BF6348983000EBC40082
:10FB100080ED00CBC82073F023F91FEDAD0B6048DA
:10FB200000EBC40080ED000B5A485030005D00F03F
:10FB30003000E0BB5B48006840F0010059490860B4
:10FB400000BF00BF00BFBFF34F8FBFF36F8F00BF79
:10FB500000BF00BFC4EBC401534800EB0110D0E963
:10FB60001030C4EBC401504A02EB0112D2E90E126C
:10FB700059185041C4EBC4024B4B03EB0212C2E9CB
:10FB80001010C4EBC400194601EB0010816DC4EBEA
:10FB9000C4001A4602EB0010C06B081AC4EBC40183
:10FBA00002EB011188650021C4EBC40200E003E010
:10FBB00003EB02129163D163384800782840002893
:10FBC0005FD034485030005D00F03000A0B33548BD
:10FBD000006820F00100334908602E485030005D75
:10FBE00000F0030020B301212A4880F8F81000F14A
:10FBF000E80252F82410103A52F82400F4F7A9F859
:10FC000000EE100AB8EEC00B284800EBC40090EDDF
:10FC1000001B20EE010B9FED261B80EE012B2648DA
:10FC200000EBC40080ED002B00211A4880F8F8108A
:10FC30002046FEF7F5FE9CE0FFE70121154880F81D
:10FC4000F810D83030F824000FFA80FB1148E83063
:10FC500030F8240000B201908A1E1146204625F09B
:10FC60002EF9074674F006FF41EC1B0B0D480068A7
:10FC700020F001000B49086058460199F4F769F833
:10FC80001CE097E0F005002078010024000000004F
:10FC9000000000428803002030060524B40500203F
:10FCA000D8000024E00C0020200700206008052474
:10FCB000000000000000F0402002002400EE100AC6
:10FCC000B8EEC00B5F4800EBC40090ED001B20EEC7
:10FCD000010B1FED091B80EE012B5B4800EBC400FC
:10FCE00080ED002B012073F03BF84FF0FF321146FE
:10FCF000204625F0E4F8074674F0BCFE41EC100BFA
:10FD000030EE0B0BB0EE40BB012073F029F84FF042
:10FD1000FF321146204625F0D2F8074674F0AAFEBD
:10FD200041EC100B30EE0B0BB0EE40BB012073F03A
:10FD300017F84FF0FF321146204625F0C0F807466D
:10FD400074F098FE41EC100B30EE0B0BB0EE40BBA4
:10FD5000B1EE4B0BB1EE001B80EE012BB0EE42DB9F
:10FD600051EC1D0B75F01CF8384A02EBC40203C2BB
:10FD700000BF34487430005D012815D10220344999
:10FD800008553048803030F8140080001921B0FB4D
:10FD9000F1F087B2962F03DD384672F0E1FF02E002
:10FDA000962072F0DDFF00BF26487430005D2849C0
:10FDB00008550FE09FED270B234800EBC40080EDB2
:10FDC000000B0021214A02EBC402116051600020A7
:10FDD0001F4908552148006820F001001F490860AC
:10FDE0001F48007828401F49097808431D490870BA
:10FDF000204606F069FF1C48015D1C4801551C485F
:10FE0000015D1C4801551C4830F8140001B2174828
:10FE1000143820F814101948015D14480C380155A5
:10FE2000402017490855174890F82C0100F00200AF
:10FE300020B10020144901EB4401487000BFFFF7D6
:10FE40006EB900006008052420020024B8050020D7
:10FE50004C0500200000000000000000E00C002025
:10FE6000B405002070340024789A04245407052433
:10FE70007C9A04241C0B0524A89A0424A49A042424
:10FE8000AC9B04243006052400060020002018E066
:10FE9000F74991F83B1101228240114059B1F449D0
:10FEA000B1F83C11F24AB2F83E2141EA0242F1496E
:10FEB00041F8202003E00022EE4941F82020411CB7
:10FEC000C8B20428E4DB704730B50021E84890F858
:10FED000EA21E94B9B7D581E2BE0E54B93F8ED3171
:10FEE00045000224AC4023403BB9E44B1B5C022B91
:10FEF00003DB012383401343DAB2E04B1B5C022B8C
:10FF00000FDB012383400B43D9B2DC4B1B5C03F0B6
:10FF1000010363B1031D012404FA03F30B43D9B2B7
:10FF200005E0002300EB4004D54D2C446370431ED4
:10FF300018B20028D1DAD3480270D348017030BD1E
:10FF4000D2480078D2490870D248007820B1032006
:10FF5000D14908701B207047D048C07820B10320D9
:10FF6000CD4908701D20F6E7CC48807820B90320E1
:10FF7000C94908701D20EEE70020ECE77CB5054676
:10FF80000C46012D11D11CB9C5A0F0F729FC08E0E1
:10FF9000207818B1C3A0F0F723FC02E0C0A0F0F76E
:10FFA0001FFCC148F0F747FF21E0F5B9BF49C04A3F
:10FFB000128888186B4601AABEA1F0F7DFFD06B2D1
:10FFC000012E01D006207CBD0CB90020FBE7BDF856
:10FFD000040010B90020207009E0BDF804000128D9
:10FFE00001D1207003E00520EDE70720EBE70020BA
:10FFF000E9E72DE9F04F87B081460E4614469A4650
:020000040801F1
:100000004FF0000B032E03DD012007B0BDE8F08F99
:1000100004AA0DF11A0006A9CDE901020091A34935
:10002000A34A128888180DF1160305AAA3A1F0F7B8
:10003000A5FD07B2B9F1010F46D1002F01DD062061
:10004000E3E7002E09DBA05D18B196A0F0F7C8FB2E
:1000500036E093A0F0F7C4FB32E0207818B19CA002
:10006000F0F7BEFB02E09BA0F0F7BAFB8248807D70
:10007000012808DD607818B197A0F0F7B1FB02E025
:1000800096A0F0F7ADFB7C48807D022808DDA078C3
:1000900018B191A0F0F7A4FB02E090A0F0F7A0FB4C
:1000A0007548807D032808DDE07818B18AA0F0F754
:1000B00097FB02E089A0F0F793FB89A0F0F790FB93
:1000C0007948F0F7B8FE53E0B9F1000F4ED1002E99
:1000D0002CDA002F01DD042F01DD062095E7002535
:1000E00021E005A830F8150010B94FF000080AE02B
:1000F00005A830F81500012801D1804603E04FF033
:10010000050B14F80580605D40450AD0594850F849
:10011000250000EA0A0010B14FF0480B01E004F896
:100120000580681CC5B2BD42DBDB21E0012F01D098
:1001300006206AE7BDF8140010B94FF0000807E088
:10014000BDF81400012801D1804601E005205CE7DC
:10015000A05D40450CD0474850F8260000EA0A0050
:1001600008B1482051E704F8068001E007204CE779
:1001700058464AE72DE9FC4104460D4616461F46FF
:100180004A494B4A128888186B4601AA49A1F0F7E0
:10019000F5FC0FFA80F8012C0DD1B8F1000F02DD4B
:1001A0000620BDE8FC8129784EA0F0F719FB3E48F7
:1001B000F0F741FE15E094B9B8F1010F01D0062027
:1001C000EFE7BDF90400B04203DBBDF90400B8421B
:1001D00001DD0520E5E7BDF80400287001E00720F7
:1001E000DFE70020DDE72DE9FE438046894615461E
:1001F000B9F1000F02DB0120BDE8FE8301A82B4905
:100200002B4A0090128888180DF10A0302AA37A120
:10021000F0F7B4FC06B2B8F1010F6DD1012E01DD8B
:100220000620E9E7002E15DC00240DE028780121E6
:10023000A140084018B131206DF01AF902E03020D9
:100240006DF016F9601CC4B2072CEFDD0D206DF0C7
:100250000FF9BEE0012E01D00620CDE7BDF9080060
:10026000002803DBBDF90800072846DD0520C3E7A9
:10027000300605241035002440000024140805240D
:10028000B8020024BC0D0020C8020024BB000024DA
:10029000BE000024AF0D0020A90B0020B4020024F2
:1002A000300D0000310D000000AF002018000030BC
:1002B000B80000242568642025686400256875203E
:1002C00025687520256875202568752025687500C6
:1002D000310000003000000020310000203000001C
:1002E0000D0000002568750D0000000025686420E1
:1002F000256864202568640012E0BDF80800C4B2D7
:1003000028780121A140084018B131206DF0B0F8E3
:1003100002E030206DF0ACF80D206DF0A9F858E047
:10032000B8F1000F53D1022E20D1BDF908000028EA
:1003300003DBBDF90800072801DD05205CE7BDF8F7
:100340000800C4B2BDF80A0028B928780121A140EC
:10035000884328703DE0BDF80A00012804D12978BF
:10036000A0400143297034E0052045E7012E2CD13F
:10037000F749F84A12888818F7A1F0F79BFD07465D
:100380003846F0F7DDFD082801D9052034E70024C0
:1003900015E0385D302805D129780120A04081433F
:1003A00029700AE0385D312805D129780120A04064
:1003B0000143297001E005201EE7601CC4B23846E5
:1003C000F0F7BEFDA042E4D803E0062014E70720C2
:1003D00012E7002010E72DE9FE43804689461546C6
:1003E000B9F1000F02DB0120BDE8FE8301A8D84966
:1003F000D84A0090128888180DF10A0302AAAFF2B9
:100400001411F0F7BBFB06B2B8F1010F3CD1012E7D
:1004100001DD0620E8E7002E15DC00240DE0288829
:100420000121A140084018B131206DF021F802E00F
:1004300030206DF01DF8601CC4B20F2CEFDD0D20D4
:100440006DF016F879E0012E01D00620CCE7BDF959
:100450000800002803DBBDF908000F2801DD052096
:10046000C2E7BDF80800C4B228880121A1400840B5
:1004700018B131206CF0FCFF02E030206CF0F8FF86
:100480000D206CF0F5FF58E0B8F1000F53D1022EAB
:1004900020D1BDF90800002803DBBDF908000F28B2
:1004A00001DD0520A0E7BDF80800C4B2BDF80A00D0
:1004B00028B928880121A140884328803DE0BDF863
:1004C0000A00012804D12988A0400143298034E092
:1004D000052089E7012E2CD19D499E4A1288881853
:1004E0009DA1F0F7E7FC07463846F0F729FD1028F4
:1004F00001D9052078E7002415E0385D302805D1C2
:1005000029880120A040814329800AE0385D3128F4
:1005100005D129880120A0400143298001E0052060
:1005200062E7601CC4B23846F0F70AFDA042E4D886
:1005300003E0062058E7072056E7002054E72DE99E
:10054000FC4104460D4616461F468149814A1288E1
:1005500088186B4601AAAFF2A421F0F70FFB0FFA3F
:1005600080F8012C0ED1B8F1000F02DD0620BDE8A5
:10057000FC81B5F9001079A0F0F732F97948F0F76D
:100580005AFC15E094B9B8F1010F01D00620EEE74E
:10059000BDF90400B04203DBBDF90400B84201DD3F
:1005A0000520E4E7BDF90400288001E00720DEE72C
:1005B0000020DCE770B505460C460DB9072070BD7C
:1005C0001CB131206CF054FF02E030206CF050FF81
:1005D0000D206CF04DFF0020F1E72DE9FC410646AF
:1005E0000F4614461D46002F02DB0120BDE8FC81AA
:1005F0000DB90220FAE70CB90220F7E7012E0DD160
:100600002078284018B131206CF032FF02E0302011
:100610006CF02EFF0D206CF02BFF24E00EBB4C493C
:100620004C4A128888186B4601AAAFF27831F0F76D
:10063000A5FA0FFA80F8B8F1010F01D00620D5E72E
:10064000BDF8040018B92078A84320700BE0BDF86D
:100650000400012803D120782843207003E00520FE
:10066000C4E70720C2E70020C0E72DE9FC410646A9
:100670000F4614461D46002F02DB0120BDE8FC8119
:100680000DB90220FAE70CB90220F7E7012E0DD1CF
:100690002068284018B131206CF0EAFE02E03020DA
:1006A0006CF0E6FE0D206CF0E3FE24E00EBB284962
:1006B000284A128888186B4601AAAFF20841F0F761
:1006C0005DFA0FFA80F8B8F1010F01D00620D5E7E6
:1006D000BDF8040018B92068A84320600BE0BDF8FD
:1006E0000400012803D120682843206003E005208E
:1006F000C4E70720C2E70020C0E72DE9F04F87B02C
:1007000081460E4690469A464FF0000B98F80040FE
:10071000032E03DD012007B0BDE8F08F04AA0DF120
:100720001A0006A9CDE9010200910949094A128877
:1007300088180DF1160305AA0BA1F0F71FFA07B2EE
:10074000B9F1010F71D1002F18DD0620E3E7000099
:1007500018000030B8000024200D0A002568640D40
:100760000000000000AF0020256864202568642098
:10077000256864202568642025686400002E0FDB4E
:1007800098F800000121B140084020B1AFF2EC40E0
:10079000F0F726F844E0AFF2F840F0F721F83FE038
:1007A00004F0010020B1AFF2D840F0F719F803E0EF
:1007B000AFF2E040F0F714F8FD48807D01280BDD32
:1007C00004F0020020B1AFF2F040F0F709F803E0C6
:1007D000AFF2F840F0F704F8F548807D02280BDD11
:1007E00004F0040020B1AFF21050EFF7F9FF03E07E
:1007F000AFF21850EFF7F4FFED48807D03280BDDD2
:1008000004F0080020B1AFF23050EFF7E9FF03E049
:10081000AFF23850EFF7E4FFAFF23C50EFF7E0FFF4
:10082000E448F0F708FB63E0FFE7B9F1000F5DD1A2
:10083000002E32DA002F01DD042F02DD4FF0060B0F
:1008400051E0002526E005A810F8150044FA05F14E
:10085000484000F00100D8B1D74850F8250000EA20
:100860000A0010B14FF0480B12E005A830F815004F
:1008700018B90120A84084430AE005A830F8150003
:10088000012803D1A8402043C4B201E04FF0050B7A
:10089000681CC5B2BD42D6DB25E0012F01D0062081
:1008A00039E7BDF8140044FA06F1484000F00100B1
:1008B000C8B1C14850F8260000EA0A0010B14FF054
:1008C000480B10E0BDF8140018B90120B040844373
:1008D00009E0BDF81400012803D1B0402043C4B2A0
:1008E00001E04FF0050B88F8004001E04FF0070BE6
:1008F000584610E72DE9F84306460C4615461F46B4
:10090000012E22D1287830B1012808D002280AD03F
:10091000032810D10BE0A9A0EFF762FF10E0A8A018
:10092000EFF75EFF0CE0A7A0EFF75AFF08E0A6A0E4
:10093000EFF756FF04E0AFF29860EFF751FF00BF0A
:1009400000BF9C48F0F777FA38E09EBB9F49A04A69
:10095000128888186A46AFF2E011F0F70FF90FFA23
:1009600080F897B1B8F1010F0FD1BDF8000018B1B0
:10097000BDF90000401C40B9002C02DB0120BDE89D
:10098000F883FF2028700020F9E7B8F1000F01DD9F
:100990000620F4E7002C01DB032C01DD0120EEE74B
:1009A0002878A04207D02C708148807DA04202DCCC
:1009B0000120E4E700E001E00720E0E70020DEE7B7
:1009C0002DE9F04F87B080460E4614469946DDE982
:1009D00010AB00200390032E03DD012007B0BDE81B
:1009E000F08F04AA0DF11A0006A9CDE901020091C9
:1009F0007649774A128888180DF1160305AAAFF2D6
:100A00009821F0F7BBF807B2B8F1010F30D1002FF1
:100A100001DD0620E2E7002E05DBA15DAFF23C70B0
:100A2000EFF7DEFE20E02178AFF26070EFF7D8FE3E
:100A30005F48807D012803DD617866A0EFF7D0FE76
:100A40005B48807D022803DDA17862A0EFF7C8FE35
:100A50005748807D032803DDE1785EA0EFF7C0FEF4
:100A6000AFF28470EFF7BCFE5248F0F7E4F953E0C0
:100A7000B8F1000F4ED1002E2DDA002F01DD042F2A
:100A800002DD0620039047E0002521E005A830F9AB
:100A90001500484504DB05A830F91500504502DD76
:100AA0000520039012E0605D05A931F91510884218
:100AB00008D0414850F8250000EA0B0010B148204A
:100AC000039003E005A810F815006055681CC5B236
:100AD000BD42DBDB20E0012F01D006207EE7BDF91F
:100AE0001400484503DBBDF91400504501DD052025
:100AF00074E7A05DBDF91410884207D02E4850F865
:100B0000260000EA0B0008B1482067E7BDF8140092
:100B1000A05501E00720039003985FE7F0B52DEDA5
:100B2000028B83B004460D46B0EE408B1646274933
:100B3000274A1288881801AB02AA28A1F0F71EF8EC
:100B400007B2012C1FD1002F04DD062003B0BDEC3D
:100B5000028BF0BD092E03DD39202249887003E0A5
:100B600006F130001F49887095ED001AB7EEC11AE2
:100B7000B0EE410B53EC102B1A48EFF725FE0D4851
:100B8000F0F759F938E07CBB012F01D00620DDE7F2
:100B90009DED020AB4EEC80AF1EE10FA06D39DEDFF
:100BA000020AB4EEE80AF1EE10FA1EDD0520CDE7E8
:100BB0004000002400AF002010350024780D000014
:100BC000790D00007A0D0000610D00001800003062
:100BD000B800002420256875000000002566202547
:100BE000686400002000002004E09DED020A85ED0D
:100BF000000A01E00720A9E70020A7E72DE9F04758
:100C00002DED028B88B080460E461446B0EE408B28
:100C100099464FF0000A032E05DD012008B0BDEC17
:100C2000028BBDE8F08703AA07A806A9CDE9010257
:100C30000091FD49FD4A1288881805AB04AAFCA161
:100C4000EFF79CFF07B2B8F1010F60D1002F01DD73
:100C50000620E3E7B9F1090F03DD3920F849C87030
:100C600003E009F13000F649C870002E0EDB04EBFA
:100C7000860090ED001AB7EEC11AB0EE410B53ECAE
:100C8000102BEF48401CEFF79FFD38E094ED001A61
:100C9000B7EEC11AB0EE410B53EC102BE848401CE4
:100CA000EFF792FDE748807D01280ADD94ED011AF7
:100CB000B7EEC11AB0EE410B53EC102BE048EFF742
:100CC00083FDE048807D02280ADD94ED021AB7EE2C
:100CD000C11AB0EE410B53EC102BD948EFF774FD5D
:100CE000D848807D03280ADD94ED031AB7EEC11AB7
:100CF000B0EE410B53EC102BD148EFF765FDAFF68A
:100D00002020EFF76DFDD048F0F795F84FE0B8F1EF
:100D1000000F4AD1002E2DDA002F01DD042F02DD55
:100D20004FF0060A43E0002521E004A800EB85000F
:100D300090ED000AB4EEC80AF1EE10FA09D304A847
:100D400000EB850090ED000AB4EEE80AF1EE10FA2F
:100D500002DD4FF0050A08E004A800EB850090EDE5
:100D6000000A04EB850080ED000A681CC5B2BD4294
:100D7000DBDB1CE0012F01D006204FE79DED040ACC
:100D8000B4EEC80AF1EE10FA06D39DED040AB4EEF3
:100D9000E80AF1EE10FA01DD05203FE79DED040AB7
:100DA00004EB860080ED000A01E04FF0070A504690
:100DB00034E7B0EE401B042813DB61280CD0782800
:100DC00004D0792804D07A2808D103E0002007E075
:100DD000012005E0022003E0032001E0002000BF25
:100DE00000BF9A49095C0B293AD2DFE801F0240AD6
:100DF00006343110151A1F070B0000BFB0EE410B6F
:100E0000704700BF9FED920B21EE000BF8E7B2EEAA
:100E1000040B21EE000BF3E79FED8F0B21EE000B8F
:100E2000EEE79FED8F0B21EE000BE9E79FED8E0BB8
:100E300021EE000BE4E78E4901EBC00191ED000BC0
:100E400020EE010B8B4991ED002B20EE020BD7E732
:100E5000B0EE410BD4E79FED882B81EE020BCFE77C
:100E6000B0EE410BCCE7F0B52DED068B83B0B0EEC4
:100E7000409B04460E461746B0EE498B7348055D0D
:100E80000B2D7CD2DFE805F09F13066188313D49C8
:100E90005507140000BF7A4890F83901303079497D
:100EA000887053EC182B0846EFF78EFCB0E000BFBB
:100EB000734890F8390140B2C01E012801DA0120C0
:100EC00004E06F4890F8390140B2C01E30306D49DF
:100ED00088709FED611B28EE011BB0EE410B53ECB7
:100EE000102B0846EFF770FC92E09FED671B28EE91
:100EF000011BB0EE410B53EC102B65A0EFF770FC1B
:100F000086E09FED531B28EE011BB0EE410B53EC26
:100F1000102B61A0EFF764FC7AE09FED510B88EE97
:100F2000001BB0EE41AB53EC1A2B59A0EFF758FC65
:100F30006EE09FED4D0B88EE001BB0EE41AB53EC25
:100F40001A2B53A0EFF74CFC62E04D4890F83901A2
:100F500040B2801E002801DA002004E0484890F8E2
:100F6000390140B2801E30304649887037B9684632
:100F7000B0EE480B71F0C2F8B0EE408B00E041E0FB
:100F80009FED3D1B28EE011BB0EE410B53EC102BE7
:100F90003C48EFF719FC3BE0394890F8390140B282
:100FA000401E012801DA012004E0354890F839019B
:100FB00040B2401E30303349887053EC182B08463D
:100FC000EFF702FC24E02B4890ED001B88EE010BAC
:100FD000334800EBC40090ED001B20EE011B2848B5
:100FE000503030F81400000300EE100AB8EEC00BC9
:100FF00021EE000BB0EE40AB53EC1A2B29A0EFF71B
:10100000EFFB05E02A46214628A0EFF7E9FB00BFE9
:1010100000BF2E480078022869D10D2E58D0202E0E
:101020005AD02C2E5DD158E018000030B8000024B2
:101030002566202566202566202566202566000079
:10104000260000204000002400AF00206407052493
:10105000FCA9F1D24D62503F0000000000408F40DB
:101060006666666666663940A60A462575029A3F38
:1010700078010024D80100240000000000807640A0
:1010800030060524A30000209A9999999999B93FAF
:1010900025362E346C66000025332E346C66000035
:1010A0009801002425322E306C6600004552524FC4
:1010B000523A20756E657865706563746564206466
:1010C000696D20256320256400000000C100002414
:1010D000F8A0EFF785FB09E000BFF7A0EFF780FB72
:1010E00004E03146F5A0EFF77BFB00BF03E031469B
:1010F000F2A0EFF775FBF248EFF79DFE03B0BDECF1
:10110000068BF0BD2DE9F0472DED028B88B08046AF
:101110000D461646B0EE408B4FF0000A032D05DD5C
:10112000012008B0BDEC028BBDE8F08703AA07A838
:1011300006A9CDE901020091E249E34A1288881824
:1011400005AB04AAAFF21811EFF718FD07B2B8F11A
:10115000010F7DD1012F01DD0620E2E7002F08DC21
:10116000DA4890F8390100EE100AB8EE400A8DED29
:10117000040A9DED040AB5EEC00AF1EE10FA08D299
:10118000D24890F8390100EE100AB8EE400A8DED11
:10119000040A9DED040ABCEEC00A10EE100AC4B2A7
:1011A000062C00DD0624C94890F8399180F83941B1
:1011B000002D0DDBE8B206EB850191ED001AB7EECC
:1011C000C11AB0EE410B01220D21FFF74CFE3EE0AB
:1011D00096ED001AB7EEC11AB0EE410B01222021A4
:1011E0000020FFF740FEBA48807D01280ADD96ED19
:1011F000011AB7EEC11AB0EE410B012220211046B0
:10120000FFF731FEB248807D02280ADD96ED021A12
:10121000B7EEC11AB0EE410B012220210220FFF7E8
:1012200022FEAB48807D03280ADD96ED031AB7EE57
:10123000C11AB0EE410B012220210320FFF713FE5B
:10124000AFF66470EFF7CCFA9D48EFF7F4FD00E0DD
:1012500003E09E4880F8399182E0B8F1000F7DD11B
:10126000002D4BDA002F01DD042F01DD062058E7A9
:10127000002440E004A800EB840090ED001AB7EED3
:10128000C11AB0EE410B2046FFF793FDB7EEC00B3D
:1012900004A800EB840080ED000A04A800EB8400A1
:1012A00090ED000AB4EEC80AF1EE10FA07D204A8D5
:1012B00000EB840080ED008A4FF0050A10E004A8DE
:1012C00000EB840090ED000AB4EEE80AF1EE10FAAB
:1012D00006DD04A800EB8400C0ED008A4FF0050A8B
:1012E00004A800EB840090ED000A06EB840080ED7A
:1012F000000A601CC4B2BC42BCDB31E0012F01D04B
:1013000006200EE7E8B29DED041AB7EEC11AB0EE62
:10131000410BFFF74EFDB7EEC00B8DED040A9DEDBE
:10132000040AB4EEC80AF1EE10FA04D28DED048A74
:101330004FF0050A0AE09DED040AB4EEE80AF1EE6A
:1013400010FA03DDCDED048A4FF0050A9DED040A85
:1013500006EB850080ED000A02E0FFE74FF0070A88
:101360005046DEE62DE9FC4704460D4616461F466C
:101370005449554A128888186B4601AA55A1EFF7BF
:10138000FDFB0FFA80F8012C12D1B8F1000F02DD3D
:101390000620BDE8FC87288880001921B0FBF1F900
:1013A00049464EA0EFF71CFA4548EFF744FD1CE014
:1013B000CCB9B8F1010F01D00620EAE70198B0429C
:1013C00002DB0198B84201DD0520E2E7019901EB5B
:1013D000C10202EB0111C81CC11700EB9171C1F3EE
:1013E0008F01298001E00720D3E70020D1E72DE914
:1013F000FC4704460D4616461F463249324A1288BB
:1014000088186B4601AA33A1EFF7B8FB0FFA80F8F2
:10141000012C11D1B8F1000F02DD0620BDE8FC87D8
:101420002888192190FBF1F949462CA0EFF7D8F94B
:101430002348EFF700FD16E09CB9B8F1010F01D089
:101440000620EBE70198B04202DB0198B84201DDCB
:101450000520E3E7019800EBC00101EB00102880B4
:1014600001E00720DAE70020D8E710B501460020A8
:101470001B4A126802F080520AB15920BCE0194A96
:10148000D2780AB11D20B7E0174A127802F00F0295
:101490000AB14A20B0E0154A127802F001020AB1FE
:1014A0004920A9E0114A127802F002020AB149204B
:1014B000A2E01DE00D0A00002000000025630000EE
:1014C00000AF002018000030B800002430060524CA
:1014D00040000024256420256864000025750D0067
:1014E000E00C0020B4020024D80B0020C800002427
:1014F000F84A127802F004020AB149207CE0F54A69
:10150000127802F010020AB1502075E0F14A127808
:1015100002F020020AB150206EE0EE4A127802F08A
:1015200040020AB1512067E0EB4A126802F0200243
:101530000AB9522060E0E84A126802F002020AB9D1
:10154000532059E0E44A126802F008020AB9542014
:1015500052E0E14A126802F001020AB955204BE05C
:10156000DD4A126802F004020AB95C2044E0D94A5C
:10157000128802F480620AB158203DE0D74A92F8FE
:101580004A20D74B93F850321A40D64B1B78D64C92
:10159000247823431A400AB15B202DE0CD4A1288FB
:1015A00002F480420AB14D2026E0CA4A128802F4B1
:1015B00080520AB14C201FE0C64A128802F4005241
:1015C0000AB14C2018E0C34A128802F400420AB162
:1015D0004F2011E0BF4A128802F400620AB14E2087
:1015E0000AE0C24A12780AB11B2005E0B94A126823
:1015F00002F4803202B1472009B1B64A908010BD92
:1016000070B505460E463DB9B248006820F48060CA
:10161000B0490860002070BDAE48808810B1AD4868
:10162000848803E00020FFF720FF04462146B048ED
:10163000EFF7D6F8AF48EFF7FEFBE0B2EBE710B5F7
:1016400004461CB9ACA0EFF7CBF803E02146ACA0F0
:10165000EFF7C6F8A748EFF7EEFB10BD10B504464C
:101660002146AAA0EFF7BCF8572C54D04BDC342C01
:1016700052D020DC0A2C50D008DC0A2C4ED2DFE8F5
:1016800004F0A2A6AAAEB2B7BBBFC3C71B2C46D0FC
:1016900008DCA4F10B000528F0D2DFE800F0C1C59A
:1016A000C9CDD1001D2C66D0202C65D0322C64D041
:1016B000332C33D1D9E0A4F135002228DED2DFE883
:1016C00010F0DC002D002D002D002D00E000E400C6
:1016D0002D002D002D002D002D002D002D002D00A2
:1016E0002D002D00E800EC00F000F400F800FC00F4
:1016F0000001040109030D031103150319031D0360
:10170000210325032903792C71D02CDCA4F1580086
:101710002128B3D204E001E3ABE07DE076E393E07F
:10172000DFE810F00003040308030C0310031403A4
:1017300074037403740374037403740318031C03A5
:101740002003240328032C033003340338037403D9
:101750007403740374037403740374033C0340033D
:10176000440348034C038E2C72D01DDCA4F17A0094
:10177000142891D202E06CE06FE072E0DFE810F034
:1017800026032A032E03320336033A033E034203A1
:101790004603460346034603460346034603460301
:1017A0004603460366056A05A4F1AC00092885D204
:1017B000DFE810F028052C053005340538053C0518
:1017C00040054405480554A0EFF70AF885E255A006
:1017D000EFF706F8FAE757A0EFF702F8F6E75BA095
:1017E000EEF7FEFFF2E75FA0EEF7FAFFEEE7E9E2C1
:1017F00060A0EEF7F5FFE9E764A0EEF7F1FFE5E79B
:1018000069A0EEF7EDFFE1E770A0EEF7E9FFDDE795
:1018100078A0EEF7E5FFD9E784A0EEF7E1FFD5E782
:1018200088A0EEF7DDFFD1E793A0EEF7D9FFCDE773
:1018300097A0EEF7D5FFC9E7A2A0EEF7D1FFC5E765
:10184000AEA0EEF7CDFFC1E7BBA0EEF7C9FFBDE745
:10185000DDE2BEA0EEF7C4FFB8E7C0A0EEF7C0FF20
:10186000B4E7C7A0EEF7BCFFB0E7CCA0EEF7B8FF37
:10187000ACE7D1A0EEF7B4FFA8E7D7A0EEF7B0FF32
:10188000A4E7DAA0EEF7ACFFA0E7DDA0EEF7A8FF33
:101890009CE7E4A0EEF7A4FF98E7E6A0EEF7A0FF30
:1018A00094E7E7A0EEF79CFF90E7EDA0EEF798FF36
:1018B0008CE7EF48EEF794FF88E7EEA0EEF790FF95
:1018C0000BE2F6A0EEF78CFF07E2F9A0EEF788FF37
:1018D00003E20000C8000024D40B0020880300208D
:1018E00030060524B405002070340024AF0D00201C
:1018F000E402010800AF00204F4B2E2E2E0D0000F9
:10190000455252202568750D000000004552524F87
:1019100052202568752C00006E6F206572726F7200
:10192000000000006E6F2076616C69642061786948
:10193000730000006E6F2065786563757461626C7A
:10194000652066756E6374696F6E0000636F6D6D00
:10195000616E64206C696E6520746F6F206C6F6EB1
:1019600067000000756E6B6E6F776E206B65797720
:101970006F7264006E756D626572206F7574736945
:1019800064652072616E67650000000077726F6E9B
:1019900067206E756D626572206F66206172677573
:1019A0006D656E7473000000272127206F72202759
:1019B0003F27206D697373696E67206F72206E6FA9
:1019C0007420616C6C6F776564000000545652207F
:1019D0006E6F7420706F737369626C6520776869CD
:1019E0006C652061786973206973206D6F76696E0C
:1019F00067000000737769746368696E67206178B7
:101A00006973206F6E2F6F6666206E6F7420706F23
:101A1000737369626C65207768696C6520545652EF
:101A200020697320616374697665000066756E6372
:101A300074696F6E206E6F7420636F6E6669677570
:101A4000726564006175746F6D61746963206D6F98
:101A50007665206E6F7420706F737369626C652099
:101A60007768696C65206A6F6767696E67206D616A
:101A70006E75616C000000006C696D69742073778D
:101A80006974636820616374756174656400000043
:101A900066756E6374696F6E206E6F74206578650D
:101AA00063757461626C652062656361757365203E
:101AB000656E636F646572206465746563746564E4
:101AC000000000006572726F7220647572696E6743
:101AD0002063616C6962726174696F6E20286C6941
:101AE0006D697420737769746368206E6F742072F7
:101AF000656C656173656429000000006572726F32
:101B00007220647572696E672063616C69627261CC
:101B100074696F6E20286F70706F73696E67206CC8
:101B2000696D697420737769746368206163747583
:101B3000617465642900000053544F5020696E7031
:101B4000757420616374697665000000616D706C66
:101B50006966696572206F66660000006D6F766564
:101B6000206469736361726465642074617267657F
:101B700074206F757473696465206C696D69740095
:101B80006F6E6520617267756D656E74206F6E6C27
:101B900079206578706563746564000061726775AB
:101BA0006D656E74206973206E6F742061206E7590
:101BB0006D626572000000006B6579776F7264205A
:101BC000424547494E206F7220454F46206D69734C
:101BD00073696E6700000000756E6B6E6F776E2024
:101BE00067656F207479706500000000756E657818
:101BF0007065637465642073657175656E636500F7
